:020000040800F2
:10000000002000106914030885EC0108C95D000890
:1000100081EC01087DEC010879EC0108000000008A
:1000200000000000000000000000000075EC010866
:1000300071EC0108000000006DEC0108B1720008CD
:10004000D1140308D1140308D1140308D1140308F0
:10005000D1140308D1140308D1140308D1140308E0
:10006000D1140308D1140308D1140308194300085C
:1000700009430008F9420008E9420008D942000893
:10008000C5420008B1420008D1140308D114030886
:10009000EDF10108D1140308D1140308D1140308A9
:1000A000D114030845640008E56300086D64000886
:1000B000356400082564000815640008D11403089D
:1000C000D1140308D1140308D1140308D114030870
:1000D000D11403082D750008B174000835740008A8
:1000E000D1140308D11403085DEC0108D1140308EE
:1000F000F5630008D114030805640008D11403084F
:10010000000000000000000000000000D1140308FF
:10011000B97300083D7300080D3A0108F139010870
:100120009D420008894200087542000861420008AB
:100130004D420008D1140308000000000000000038
:10014000D1140308D1140308D114030800000000DF
:10015000000000000000000000000000000000009F
:100160000000000000000000D1140308D1140308AF
:10017000D11403080000000000000000000000008F
:0801800000000000D114030887
:100188000A4B30B503F1140493F900205D78072A6F
:10019800C8BF143A811804338D7213F8025C855471
:1001A80013F8012C0A75A342EED130BDFC3C0308BC
:1001B80003682DE9F041DF691FB13B46BDE8F04116
:1001C8001847002A164611DD04460D460E4400E085
:1001D80023689B68204698470028F9D0236815F8BB
:1001E800011B1B6820469847AE42F1D1BDE8F0815B
:1001F80010B45A21582400220323047041708270DD
:10020800C3705DF8044B7047152303701623C37041
:10021800172383712D2343702E2303712F23C3715A
:10022800704730B4836813B11C689B882385436882
:1002380040F2E93401E0002C37D01D89013C15F06B
:10024800020FA4B2F7D0197303F10C0540F2E9319B
:1002580001E000294BD01C89013914F0010F89B243
:10026800F7D02B78436840F2E93101E000292DD01E
:100278001C89013914F0020F89B2F7D01A7303F1FF
:100288000C0440F2E93201E0002A41D01989013A10
:1002980011F0010F92B2F7D02378836813B11A686E
:1002A8009B889361012030BC704721498B4204D060
:1002B800A1F578418B42D6D101241E4901EB0414E3
:1002C8006189013189B261816189CCE7184A934219
:1002D80004D0A2F578429342DFD10121154B03EBFC
:1002E80001114B8901339BB24B814B89D5E7104CE7
:1002F800A34203D010498B42B4D101210D4B03EB2B
:1003080001114B8901339BB24B814B894368AAE7A2
:1003180007498B4203D0084A9342BED10122054BBC
:1003280003EB0212538901339BB253815389B4E71B
:10033800003001400057002000380040F0B48489A4
:100348004FF6FF764FF47A743BB3002937D00F7815
:10035800013101E0B44219D00589013C15F00205CC
:10036800A4B2F7D007734FF47A7402E0BCB2B44277
:100378000CD0058915F0010504F1FF37F6D0057B8F
:10038800EDB20AB115700132013BDDE70D4B984221
:1003980007D0A3F57843984202D00120F0BC7047FB
:1003A8000125094B03EB05156B8901339BB26B8162
:1003B800688980B2003018BF0120F0BC7047FF2761
:1003C800CAE700BF003001400057002070B505465D
:1003D800806810B104688088208541F080016868D1
:1003E80040F2E93400E0F4B10689013C16F0020F4E
:1003F800A4B2F8D0017300F10C0640F2E93100E034
:1004080011B30489013914F0010F89B2F8D0317899
:1004180068680021FFF792FFAB6813B11A689B88E0
:100428009361012070BD1149884204D0A1F578413B
:100438008842EED101240E4901EB0414618901318F
:1004480089B261816189E4E7084CA04203D0094977
:100458008842DDD10121064800EB011148890130AD
:1004680080B2488149896868D3E700BF00300140FD
:100478000057002000380040002870B51EDB09280E
:10048800044620DD012303EB83035B00B0FBF3F29A
:10049800092AF8D87BB10E4EB4FBF3F00928CCBF7B
:1004A80057223022A6FB03E5024403FB1044EB0865
:1004B80001F8012BF0D100230B7070BD2D230B70B8
:1004C80040420131DBE7303001F8010BF3E700BFB0
:1004D800CDCCCCCC884230B44FF001042ED301FBF4
:1004E80004F4B0FBF4F58D42F9D284B1AAB901E065
:1004F800B0FBF4F5092DCCBF572230222A4404FB67
:10050800150003F8012BB4FBF1F4002CF0D1002204
:100518001A7030BC7047B0FBF4F5092DCCBF3722F8
:1005280030222A4404FB150003F8012BB4FBF1F434
:10053800002CF0D100221A7030BC70470546002A02
:10054800EBD1D7E703685A1C0260197070472DE990
:10055800F047089C2578002B804689460CBF4FF051
:10056800200A4FF0300A661C35B3002A29DD3346CD
:1005780001E0024698B113F8011B501E0029F8D17A
:10058800971E60B13D46013D51464046C8476B1C29
:10059800002BF8DC257827EAE770013055B1041BF9
:1005A80029464046C847301916F8015B002DF7D197
:1005B800BDE8F087BDE8F087002A04DC2846BDE8DE
:1005C800F0870020EBE7571EDCE783684268D0ED30
:1005D800037A00EB83010133934281ED040A8360BF
:1005E80004BF0023836000EB830393ED047A036860
:1005F80070EE277A9A42C0ED037A77EEC77AC0ED9B
:10060800037A0CDA013307EE103AF8EEC76AB7EE50
:10061800007A87EEA60A036030EE070A704707EEF5
:10062800102AB8EEC77A87EE870A704790ED057AE8
:1006380090ED004AD0ED066AD0ED014AD0ED047A7B
:1006480090ED035AD0ED025AA4EE007AB0EE406A5B
:10065800B0EE470AB0EE667AA6EE247A67EEC07A64
:10066800A0EE457AE6EE257A80ED057AC0ED067AA9
:100678007047D0ED057A90ED013AD0ED003AD0ED13
:10068800064A90ED024A90ED077A90ED035A90EDF4
:10069800086AD0ED045AC0ED067AF0EE406A27EEFB
:1006A800830AC0ED056AA3EEA60A80ED087AA4EED7
:1006B800240AA5EE470AA5EEC60A80ED070A704788
:1006C800D0ED007A90ED017A30EE670AE7EE007A15
:1006D800B0EE670AC0ED007A704770470A4491424D
:1006E80014D030B40139551E41F2210211F8014FDE
:1006F800082380EA042004044CBF82EA400040003A
:10070800013B80B2F7D18D42F0D130BC70472DE962
:10071800F04FDFF8FCC1DFF8FCE1BCF80A70DEF846
:100728000060BCF80C30BCF808A03C028BB0361B4B
:100738004FF00004CDE90034009CBCF806304FEAC5
:1007480017654FF0000767EB0507B946B046A4FBED
:1007580006670024CDE90634009C002304FB0977D2
:100768000024CDE90034AAFB0823CDE90223039A2B
:10077800F30D00930AFB09230393009B43EA4723E5
:100788000093029B4FEAD31AFB150193039B4AEA95
:10079800436ADDE9002344464D46CDE90845069CF9
:1007A80012F5FA62A4FB086743F1000304FB09771A
:1007B800CDE90623BCF80440039BBCF802204FEAAD
:1007C800E31B230C059323040493340A44EA0764C7
:1007D8003D12DDE904674FEAC23816EB0A0647EB1B
:1007E8000B0718EB0408DDE906344FEA524949EBD8
:1007F8000509B3F5FA6F74F10004B246BB463CDA5A
:10080800DDE90067BC00B20044EA9673B41847EB10
:10081800030522463C462B4602FB04F406FB034430
:10082800A2FB06232344940844EA83749D105B10BA
:100838004FEA3202B8EB040869EB0509BAEB020A81
:100848006BEB030BDDE90623304C4FF0FF35A2427A
:10085800AB412CDBDDE90856A5FB052305FB06F4B7
:1008680003EB4403D40F44EA4304DD17DDE9062310
:10087800121B63EB0503CDE90623DEF80440A4FB55
:10088800082304FB0933540D44EAC3245D15B4EB73
:100898000A0A65EB0B0B4FEADA3343EA4B4300B124
:1008A800036009B1069B0B600BB0BDE8F08F40F602
:1008B800AC52B4184FF0000347EB03052246A2FBE5
:1008C800022304FB05F403EB4403941843EB0305EC
:1008D800A4185D414FEA850CA6004CEA947CB41A32
:1008E8006CEB0305DF00D6006D104FEA340447EACD
:1008F8005277921B63EB0703B8EB040869EB050911
:100908001AEB020A4BEB030BA4E700BF24FAFFFF24
:10091800D43B0020941E00202DE9F04FDFF81CB2D4
:10092800DFF81CE2BBF80020DEF80860BBF90430F1
:10093800BBF90250BBF90A80C2EB261404FB04F48D
:1009480024135200C2EBE60203FB04F305FB02F298
:100958009B1303EBE223B3F5FA364FEAE37589B04C
:1009680045F1FF373246A6FB0645CDE9024502FBB5
:1009780007F205EB4202CDE90467029EBBF9084085
:10098800039208FB02FC4FEAE87906FB09CC3A46D9
:10099800A8FB0689049ECBF81830E51704FB02F281
:1009A80006FB0522A4FB0667E14417444FEA182218
:1009B80042EA096200924FEA292201923D03DDE9E9
:1009C8000078340345EA16553F19BBF806600690CF
:1009D80048EB05083C1C48F5004503EB8302A4FBE3
:1009E800068906FB0599803213124FEA69064FEA19
:1009F800E977079356EA07038A4600F09280DDE913
:100A08000489BBF90E20DEF80C40BBF910004946FA
:100A1800C4F5801ED317DDE9024502FB01F108FB8E
:100A28000311A2FB08230B444FEA43492B46C11785
:100A380000FB03F304FB0133A0FB0401BBF90C40EA
:100A48001944E30001937346DC170023009349EA35
:100A5800D2394FEA4248DDE9002310EB080041EBA8
:100A68000901E50712184FEACE744B4145EA5E05C5
:100A7800A41A65EB0305221945EB050312196B410E
:100A880099019001801841EA926159418B008200D6
:100A980043EA9073101943EB05018B00820043EA87
:100AA800907310460019194632463B46694130F0AA
:100AB80003FBBBF916204C13450B45EAC14502FB65
:100AC80004F6D31705FB0366A2FB05233344BBF9E1
:100AD800146002FB04F405FB034406FB01FEA2FBC1
:100AE8000523F717234400FB07EE540EA6FB006707
:100AF800774444EAC3144FEAD64800194FEA6365BD
:100B080048EA473869414FEAE74918EB0008BBF95A
:100B1800124049EB01094FEA182646EA0966200106
:100B28003618069B0BB1360A1E60BAF1000F02D0C8
:100B3800079BCAF8003009B0BDE8F08FE43B0020FD
:100B4800941E002070472DE9F041374F374DB7F814
:100B58000AC02A8A3B89B7F91240B7F914E06E69CE
:100B6800B7F90250B7F90E80A2EB0C0203FB02F3AF
:100B7800DA139644E30293FBFEF31344A3F57A6E6B
:100B88000EFB0EF4B7F90CC0FB6122130EFB05F542
:100B9800B7F9044002FB08F8ED1202FB0CF2B7F9B2
:100BA80000C00EFB04F405EBE825B7F920E0FF8848
:100BB800121402EB643205EB8C0505FA0EF50232CD
:100BC800023592104CF25034A6EBA50502F500420E
:100BD80044FA0EF404FB05F407FB02F2D20B002CD6
:100BE800B9BFB4FBF2F252006400B4FBF2F2141283
:100BF80004FB04F50E4E40F6DE3404FB05F403EB6B
:100C0800830306FB02F524145B0004EB2544083338
:100C180004F6CF641B1102EB241200B1026001B18B
:100C28000B60BDE8F08100BFB03B0020941E00209F
:100C380043E3FFFF4FF48053838270474FF48053A0
:100C48008382704770474FF40063838270474FF484
:100C580000638382704790F8203033B1012B03D1B1
:100C68004FF400638382704770474FF48063838238
:100C7800704730B583B00C46C56D0223143001AA05
:100C88001B21A84778B1BDF80430084A43F29031D7
:100C98005BBA11FA83F382FB03121A44DB17C3EB26
:100CA80022232333238003B030BD00BFEBA00EEA1C
:100CB80070B5044682B01430E56D06236A461D21DE
:100CC800A847B0B19DF804009DF800609DF8011098
:100CD8009DF802509DF803209DF8053041EA062151
:100CE80043EA002342EA0522A187E287A4F84030BC
:100CF800012002B070BD70B5044682B01430E56DB5
:100D080006236A464321A847B0B19DF804009DF820
:100D180000609DF801109DF802509DF803209DF891
:100D2800053041EA062143EA002342EA0522A18769
:100D3800E287A4F84030012002B070BD70B50446C7
:100D480082B00830656A06236A463B21A847A8B1E5
:100D58009DF804009DF800609DF801109DF8025070
:100D68009DF803209DF8053041EA062143EA002357
:100D780042EA0522E18222836383012002B070BD2A
:100D88000346407F20B100225A77DA821A835A83B9
:100D98007047704701207047034690F8550030B1FE
:100DA800002283F855209A87DA87A3F840207047F5
:100DB800704770B40468037B2268022101FA03F3C8
:100DC8001A4213D042690A49582000FB02124FF612
:100DD800FE7650685289C5680068296831402960E4
:100DE800C168D24392B20A40C260636070BC704767
:100DF800AC67002030B4094B1C7864B1084B00255F
:100E080003EBC4041A6899885562D0680833014313
:100E1800A342D160F6D130BC704700BFCC6B002034
:100E2800D06B002010B40268047B11680223A34031
:100E3800194209D00649406800240C7001684FF631
:100E4800FE742140016053605DF8044B704700BF99
:100E5800D53D0020F0B4334C00EB800004EB800457
:100E68006468002C5BD0304E49004FF42040CDB26E
:100E7800B061A169090444D460682C4F45F08071C1
:100E8800384041F4903101434FF420406160B06133
:100E980003E0411E002838D00846A1698F07F8D51D
:100EA8004FF42040A262B06102E0421E68B31046CF
:100EB800A2691106F9D562681C4945F0007545F428
:100EC80080350A4015434FF420406560B06102E068
:100ED800421ED0B11046A2699207F9D5A362A36950
:100EE8004FF420409B06B06105D4431E68B11846F4
:100EF800A3699B06F9D52023B061E3610120F0BC0A
:100F08007047411E08B10846B3E7094A1388013300
:100F18009BB24FF0FF31B1611380F0BC704720469F
:100F2800F0BC7047D8560020941E0020009800FCA2
:100F380074330020134600200A4668218AE730B53A
:100F48000446C06C61710368A26823F00103036062
:100F580087B0A379009213F004023DD04FF4805279
:100F680013F00203019244D102934FF480630022EC
:100F7800039311F00103059237D1049308238D07D9
:100F8800694648BF04931EF0BFF86079E36CA17905
:100F980000F00202002A15BF4FF440324FF48032AD
:100FA8004FF40034002410F0010F586808BF22469F
:100FB800CC074CBF024320EA02025A609A6809072C
:100FC8004CBF42F0080222F008029A601A6842F008
:100FD80001021A6007B030BD13F0020301920BD072
:100FE8004FF4005513460295C1E7042304930C23DC
:100FF800C5E74FF40053B7E70293B8E710B50446C6
:10100800C06CA160036823F001030360A37986B074
:1010180013F00402009141D04FF4805213F0020300
:10102800019244D102934FF4806362790393D1070C
:101038004FF000030493059345BF0423049308234A
:101048000C236946920748BF04931EF05DF8607947
:10105800E36CA17900F00202002A15BF4FF4403278
:101068004FF480324FF40034002410F0010F586818
:1010780008BF2246CC074CBF024320EA02025A604E
:101088009A6809074CBF42F0080222F008029A60E9
:101098001A6842F001021A6006B010BD13F002038C
:1010A800019207D04FF4005113460291BDE74FF467
:1010B8000053B7E70293B8E70023262203600270C3
:1010C80027228270012243600271837170472DE9E3
:1010D800F341056906460F467DBBD0F80080C8F38A
:1010E8000A0323B30023D6F80080019329F046FDB4
:1010F800042819D1214C236943F001032361BBB2B1
:10110800A8F8003029F03AFD04282ED108F102038E
:101118000193019B3F0C1F8029F030FD23690428AF
:1011280023F00103236125D06FF0010505E029F0C4
:1011380025FD042805D04FF0FF35284602B0BDE84C
:10114800F0810E4C236943F002032361C4F8148034
:10115800236943F04003236129F010FD2369042823
:1011680023F002032361BDD0E5E7236923F00103DF
:101178002361D9E7336804333360DEE70020024097
:10118800F8B504460D468E180027B54201D12069EE
:10119800F8BDE368591CE160234415F8012B1A7265
:1011A8000429F2D1A1682046FFF791FFE76020618A
:1011B800EBE738B5044600F11405236E80226B2155
:1011C80028469847642005F0D1FF236E072268213E
:1011D80028469847642005F0C9FF236E00226B213A
:1011E80028469847642005F0C1FF236E01226B2131
:1011F800284698470F2005F0B9FF94F85320236E2E
:10120800032A8CBF1A2218221B21284698470F2030
:1012180005F0ACFF236E18221C21284698470F20A2
:1012280005F0A4FF236E94F852201A212846984707
:101238000F2005F09BFF236E94F8542019212846AF
:101248009847642005F092FF236E28461022372124
:1012580098470F2005F08AFF0F20BDE8384005F0B9
:1012680085BF70B5044600F11405236E80226B21FA
:1012780028469847642005F079FF236E2846032204
:101288006B219847236E94F85420192128469847D3
:101298000F2005F06BFF236E94F8522028461A2180
:1012A8009847236E284618221B219847236E284604
:1012B80018221C2198472846236E02223721BDE8B0
:1012C8007040184708B505F0ABFE044B5B68C01AC0
:1012D800C0F5FA5020EAE07008BD00BF4462002063
:1012E80000B5002183B00A2027F0A6FB0F210A20B1
:1012F80027F0A2FB01AA0321102027F0C9FB9DF9C2
:101308000430DFED277ADFED275A06EE103A9DF913
:10131800053006EE903A9DF9063007EE103AB8EE21
:10132800C66AF8EEE66AB8EEC77A76EEE76A36EE8F
:10133800676A37EE677AF7EE007AB0EE675AA6EE7C
:10134800255A194B0021B0EE456AB0EE675AA6EE51
:10135800A55A0A20E7EE257AF3EE0E5A26EE256AFC
:1013680025EE257A67EEA57A83ED006A83ED017A8A
:10137800C3ED027A27F060FB0DF103020121022080
:1013880027F086FB0DF103020121092027F080FBDD
:1013980001210A2027F050FB012003B05DF804FB6F
:1013A800000000430000803B0000002038B50B4CD3
:1013B8002378054653B90A4A6378106849212A46B2
:1013C80000252570FFF702F8012038BDFFF77AFFE6
:1013D8000028F0D005F070FEEDE700BF4462002061
:1013E80040620020F0B54A4C257F012D83B013D010
:1013F80028D3022D0DD1474B1B780646002B77D1F9
:101408006846FFF7D3FF20B19DF8063013F00300BC
:1014180022D0002003B0F0BD3E4E3378002B62D1BD
:101428006846FFF7C3FF9DF8003008B1DB0764D4B6
:101438000023237733784BB100230133002023772F
:1014480003B0F0BD334E3378002BF5D101210220D3
:1014580027F04EFB237FF0E79DF801E09DF8001090
:101468009DF803709DF802209DF805509DF8043002
:10147800207741EA0E2142EA072243EA052309B20E
:1014880012B21BB2494252425B42234806EE901AFE
:1014980007EE102A07EE903A90ED005AD0ED015A67
:1014A80090ED026AF8EEE66AB8EEC77AF8EEE77AE7
:1014B80066EE856A27EE257A67EE867AFDEEE66A9D
:1014C800BDEEC77AFDEEE77A16EE901A17EE102AEF
:1014D80017EE903A31807280B38001210A2027F0FC
:1014E800ABFA03B0F0BDFFF7EDFE002898D090E707
:1014F800FFF7E8FE00288CD182E7337823B907216B
:10150800032027F0F5FA257F0135257781E700BF0D
:10151800941E00204462002000000020F8B53E4ED2
:10152800777F0446C7B100F11405A06923F0DAFCFF
:1015380094F852201A212846FEF773FE012005F080
:10154800BBFDA06923F0BCFC2046FFF7D4FB94F94F
:101558003E30013357D0F8BD04F11405806923F0FB
:10156800C1FC80226B212846FEF75BFE962005F021
:10157800FDFD032268212846FEF753FE962005F05C
:10158800F5FD03226B212846FEF74BFE0F2005F0E0
:1015980093FD10226A212846FEF743FE0F2005F02E
:1015A8008BFD3A466C212846FEF73BFE0F2005F0DE
:1015B80083FD94F8542019212846FEF732FE0F20A7
:1015C80005F07AFD18221B212846FEF72AFE0F2077
:1015D80005F072FD10221C212846FEF722FE0F207E
:1015E80005F06AFD102237212846FEF71AFE0F2063
:1015F80005F062FDA06923F063FC012005F05CFDA5
:101608000123737791E794F93C300133A3D1BDE806
:10161800F8402DF0C3BA00BF941E002010B5044650
:101628000120A269138823F040031B041B0C1380BC
:1016380013889BB223F0380343F0300313801388D8
:101648009BB243F04003138005F036FD2046FFF7B8
:10165800B0FD10226A2104F11400FEF7E2FD6420B7
:1016680005F084FDA06923F02BFC0120BDE81040A3
:1016780005F022BD70B5044600F11405192005F0E7
:1016880075FD2846236E00221521984708B926F0D3
:10169800CDFD94F85220236E42F0180216212846F8
:1016A8009847236E0022172128469847236E012267
:1016B8003D2128469847236E284601223E21BDE851
:1016C8007040184770B582B004466946143027F058
:1016D8005FF9B0B19DF805009DF801609DF8021012
:1016E8009DF803509DF804209DF8063041EA062134
:1016F80043EA002342EA0522A187E287A4F84030A2
:10170800012002B070BD10B490E80600047B406967
:101718000223A3404B6013685DF8044B4FF6FE713B
:101728000B40136005F03CBF03685B6A03B11847C0
:10173800704703681B6A03B11847704703682DE9AF
:10174800F041DF691FB13B46BDE8F0411847002A68
:10175800164611DD04460D460E4400E023689B68DA
:10176800204698470028F9D0236815F8011B1B6804
:1017780020469847AE42F1D1BDE8F08103689B69E5
:1017880018470368DB68184703689B6818470368AD
:101798005B68184703681B681847014B1868F9E726
:1017A800FC760020054B53F8203033B11A689B882B
:1017B800918A0B4218BF1B0493617047345700206D
:1017C80003682DE9F04F03F13845644EAD0A012452
:1017D800755D05F01F066D09022D04FA06F400F088
:1017E800A280032D00F0A480012D52D08088B0FA89
:1017F80080F4C4F11F04A4B2E50803EB850504F0E6
:1018080007042E6AA4000F27A74026EA07062E62BF
:101818002E6A01F0030702FA04F47A1E3443012AFF
:10182800C1F3810CC1F300182C62C1F3411135D901
:10183800C60700F19780850700F1A380440700F1EF
:10184800B180020700F1BF80C60600F1CD80850691
:1018580000F1DB80440600F1E980020600F1F78020
:10186800C60500F10581850500F11381440500F1E5
:101878002181020500F12F81C60400F13D81850414
:1018880000F14B81440400F15981020455D4BDE8AC
:10189800F08F334D6E6934436C61A7E7002422460C
:1018A8004FF0010E4FF0030904E00132102A04F151
:1018B8000204ECD00EFA02F636EA0005F5D1D3F8A8
:1018C80008A009FA04F5ED430AEA050AC3F808A0D6
:1018D800D3F808B00CFA04FA4AEA0B0AC3F808A0CD
:1018E800B3F804A01FFA8AFA2AEA06069E80B3F81B
:1018F80004A008FA02F646EA0A06B6B29E801E68F6
:101908002E401E60D3F800A007FA04F646EA0A063D
:101918001E60D3F80CA001FA04F605EA0A0A46EAA2
:101928000A05DD60C1E70E4DAE693443AC615DE781
:101938000B4DEE693443EC6158E71A6822F04042D7
:101948001A601A6842EA87771F60DA6822F0404214
:1019580042EA8171D960BDE8F08F00BF6462030874
:10196800001002401A6822F003021A601A683A430B
:101978001A60DA6822F003020A438507DA607FF505
:101988005DAF1A6822F00C021A601A6842EA8702F0
:101998001A60DA6822F00C0242EA81024407DA602F
:1019A8007FF54FAF1A6822F030021A601A6842EACF
:1019B80007121A60DA6822F0300242EA0112DA608D
:1019C80002077FF541AF1A6822F0C0021A601A6850
:1019D80042EA87121A60DA6822F0C00242EA8112EB
:1019E800C606DA607FF533AF1A6822F440721A60CF
:1019F8001A6842EA07221A60DA6822F4407242EA58
:101A080001228506DA607FF525AF1A6822F4406264
:101A18001A601A6842EA87221A60DA6822F4406279
:101A280042EA81224406DA607FF517AF1A6822F489
:101A380040521A601A6842EA07321A60DA6822F4D9
:101A4800405242EA0132DA6002067FF509AF1A68AD
:101A580022F440421A601A6842EA87321A60DA6849
:101A680022F4404242EA8132C605DA607FF5FBAED5
:101A78001A6822F440321A601A6842EA07421A6069
:101A8800DA6822F4403242EA01428505DA607FF5DD
:101A9800EDAE1A6822F440221A601A6842EA8742B8
:101AA8001A60DA6822F4402242EA81424405DA6088
:101AB8007FF5DFAE1A6822F440121A601A6842EA0B
:101AC80007521A60DA6822F4401242EA0152DA60D8
:101AD80002057FF5D1AE1A6822F440021A601A682E
:101AE80042EA87521A60DA6822F4400242EA8152D6
:101AF800C604DA607FF5C3AE1A6822F040721A6035
:101B08001A6842EA07621A60DA6822F0407242EA0A
:101B180001628504DA607FF5B5AE1A6822F040628A
:101B28001A601A6842EA87621A60DA6822F040622C
:101B380042EA81624404DA607FF5A7AE1A6822F0AF
:101B480040521A601A6842EA07721A60DA6822F08C
:101B5800405242EA0172DA6097E6036803F13842BC
:101B68002DE9F04F920A584DAA5C02F01F05520960
:101B78000124022A04FA05F400F08C80032A00F0FC
:101B88008E80012A3CD001F003077A1E012AC1F396
:101B9800810CC1F300188088C1F3411135D9C607FB
:101BA80000F19680850700F1A280440700F1B0801B
:101BB800020700F1BE80C60600F1CC80850600F160
:101BC800DA80440600F1E880020600F1F680C605D6
:101BD80000F10481850500F11281440500F120819E
:101BE800020500F12E81C60400F13C81850400F154
:101BF8004A81440400F15881020455D4BDE8F08FAD
:101C0800324A55692C435461BDE7002422464FF0FF
:101C1800010E4FF0030904E00132102A04F1020416
:101C2800ECD00EFA02F636EA0005F5D1D3F808A092
:101C380009FA04F5ED430AEA050AC3F808A0D3F83F
:101C480008B00CFA04FA4AEA0B0AC3F808A0B3F879
:101C580004A01FFA8AFA2AEA06069E80B3F804A0AE
:101C680008FA02F646EA0A06B6B29E801E682E40B8
:101C78001E60D3F800A007FA04F646EA0A061E60BA
:101C8800D3F80CA001FA04F605EA0A0A46EA0A059E
:101C9800DD60C1E70D4A95692C43946173E70B4AEF
:101CA800D5692C43D4616EE71A6822F040421A6065
:101CB8001A6842EA87771F60DA6822F0404242EAEF
:101CC8008171D960BDE8F08F64620308001002409A
:101CD8001A6822F003021A601A683A431A60DA682E
:101CE80022F003020A438507DA607FF55EAF1A68BF
:101CF80022F00C021A601A6842EA87021A60DA684F
:101D080022F00C0242EA81024407DA607FF550AF04
:101D18001A6822F030021A601A6842EA07121A603A
:101D2800DA6822F0300242EA0112DA6002077FF52F
:101D380042AF1A6822F0C0021A601A6842EA871293
:101D48001A60DA6822F0C00242EA8112C606DA6036
:101D58007FF534AF1A6822F440721A601A6842EAB2
:101D680007221A60DA6822F4407242EA01228506E4
:101D7800DA607FF526AF1A6822F440621A601A68A2
:101D880042EA87221A60DA6822F4406242EA812233
:101D98004406DA607FF518AF1A6822F440521A60D8
:101DA8001A6842EA07321A60DA6822F4405242EAB4
:101DB8000132DA6002067FF50AAF1A6822F440425F
:101DC8001A601A6842EA87321A60DA6822F44042D6
:101DD80042EA8132C605DA607FF5FCAE1A6822F461
:101DE80040321A601A6842EA07421A60DA6822F436
:101DF800403242EA01428505DA607FF5EEAE1A68A4
:101E080022F440221A601A6842EA87421A60DA68A5
:101E180022F4402242EA81424405DA607FF5E0AECE
:101E28001A6822F440121A601A6842EA07521A60C5
:101E3800DA6822F4401242EA0152DA6002057FF5BC
:101E4800D2AE1A6822F440021A601A6842EA87522F
:101E58001A60DA6822F4400242EA8152C604DA6063
:101E68007FF5C4AE1A6822F040721A601A6842EA16
:101E780007621A60DA6822F0407242EA0162850459
:101E8800DA607FF5B6AE1A6822F040621A601A6806
:101E980042EA87621A60DA6822F0406242EA8162A6
:101EA8004404DA607FF5A8AE1A6822F040521A603E
:101EB8001A6842EA07721A60DA6822F0405242EA67
:101EC8000172DA6098E610B50409013C052C17D8B0
:101ED8000C4B33F8142000F00F0042FA00F313F013
:101EE80001030DD0012303FA00F0013810402FF050
:101EF80033F9054A054B125D104403EBC00010BDD1
:101F0800002010BDD8660308E4660308A06300201B
:101F18002DE9F04F4A484B4B4B4C4FF090414FF056
:101F2800010A4FF002094FF004084FF0080C4FF077
:101F3800100E20274026802530F8022B12F0010FC2
:101F480003D01960A3F804A0083312F0020F03D0DD
:101F58001960A3F80490083312F0040F03D0196035
:101F6800A3F80480083312F0080F03D01960A3F80F
:101F780004C0083312F0100F03D01960A3F804E06E
:101F8800083312F0200F02D019609F80083312F036
:101F9800400F02D019609E80083312F0800F02D0E3
:101FA80019609D80083312F4807F05D04FF4807B40
:101FB8001960A3F804B0083312F4007F05D04FF479
:101FC800007B1960A3F804B0083312F4806F05D0C1
:101FD8004FF4806B1960A3F804B0083312F4006F53
:101FE80005D04FF4006B1960A3F804B0083312F45D
:101FF800805F05D04FF4805B1960A3F804B0083304
:1020080012F4005F05D04FF4005B1960A3F804B028
:10201800083312F4804F05D04FF4804B1960A3F8B1
:1020280004B00833D20B04D04FF4004219609A80F0
:10203800083301F58061A1427FF47EAFBDE8F08FDF
:10204800D8660308A063002000180048002867D05D
:1020580003682DE9F04F03F138445C4EA40A0125CA
:10206800345D04F01F066409022C05FA06F558D001
:10207800032C00F0A580012C58D08088B0FA80F499
:10208800C4F11F04A4B2E50803EB850504F00704B6
:102098002E6AA4000F27A74026EA07062E622E6A9A
:1020A80001F00307A2407C1E3243012CC1F3810CCE
:1020B800C1F300182A62C1F341113CD9C60700F1E7
:1020C8008980850700F19580440700F1A380020705
:1020D80000F1B180C60600F1BF80850600F1CD8011
:1020E800440600F1DB80020600F1E980C60500F134
:1020F800F780850500F10581440500F1138102058B
:1021080000F12181C60400F12F81850400F13D8191
:10211800440400F14B81020400F15981BDE8F08FBD
:1021280070472B4CA6693543A561A6E7284C66691C
:1021380035436561A1E7002422464FF0010E4FF0B8
:10214800030904E00132102A04F10204E6D00EFA71
:1021580002F636EA0005F5D1D3F808A009FA04F525
:10216800ED430AEA050AC3F808A0D3F808B00CFA48
:1021780004FA4AEA0B0AC3F808A0B3F804A01FFA45
:102188008AFA2AEA06069E80B3F804A008FA02F63C
:1021980046EA0A06B6B29E801E682E401E60D3F834
:1021A80000A007FA04F646EA0A061E60D3F80CA057
:1021B80001FA04F605EA0A0A46EA0A05DD60C1E7FB
:1021C800034CE6693543E56157E700BF64620308DD
:1021D800001002401A6822F003021A601A683A4393
:1021E8001A60DA6822F003020A438507DA607FF58D
:1021F8006BAF1A6822F00C021A601A6842EA87026A
:102208001A60DA6822F00C0242EA81024407DA60B6
:102218007FF55DAF1A6822F030021A601A6842EA48
:1022280007121A60DA6822F0300242EA0112DA6014
:1022380002077FF54FAF1A6822F0C0021A601A68C9
:1022480042EA87121A60DA6822F0C00242EA811272
:10225800C606DA607FF541AF1A6822F440721A6048
:102268001A6842EA07221A60DA6822F4407242EADF
:1022780001228506DA607FF533AF1A6822F44062DE
:102288001A601A6842EA87221A60DA6822F4406201
:1022980042EA81224406DA607FF525AF1A6822F403
:1022A80040521A601A6842EA07321A60DA6822F461
:1022B800405242EA0132DA6002067FF517AF1A6827
:1022C80022F440421A601A6842EA87321A60DA68D1
:1022D80022F4404242EA8132C605DA607FF509AF4E
:1022E8001A6822F440321A601A6842EA07421A60F1
:1022F800DA6822F4403242EA01428505DA607FF565
:10230800FBAE1A6822F440221A601A6842EA874231
:102318001A60DA6822F4402242EA81424405DA600F
:102328007FF5EDAE1A6822F440121A601A6842EA84
:1023380007521A60DA6822F4401242EA0152DA605F
:1023480002057FF5DFAE1A6822F440021A601A68A7
:1023580042EA87521A60DA6822F4400242EA81525D
:10236800C604DA607FF5D1AE1A6822F040721A60AE
:102378001A6842EA07621A60DA6822F0407242EA92
:1023880001628504DA607FF5C3AE1A6822F0406204
:102398001A601A6842EA87621A60DA6822F04062B4
:1023A80042EA81624404DA607FF5B5AE1A6822F029
:1023B80040521A601A6842EA07721A60DA6822F014
:1023C800405242EA0172DA6002047FF5A7AE1A6849
:1023D80022F040421A601A6842EA87771F60DA687A
:1023E80022F0404242EA8171D960BDE8F08F0028AE
:1023F80052D0036803F138422DE9F04F920A514D4B
:10240800AA5C02F01F0552090124022A04FA05F405
:1024180043D0032A00F09080012A43D001F003073B
:102428007A1E012AC1F3810CC1F300188088C1F318
:1024380041113CD9C60700F18980850700F19580D4
:10244800440700F1A380020700F1B180C60600F13D
:10245800BF80850600F1CD80440600F1DB800206CE
:1024680000F1E980C60500F1F780850500F10581D6
:10247800440500F11381020500F12181C60400F131
:102488002F81850400F13D81440400F14B81020451
:1024980000F15981BDE8F08F70472B4A95692C43AC
:1024A8009461BBE7284A55692C435461B6E7002478
:1024B80022464FF0010E4FF0030904E00132102AC2
:1024C80004F10204E6D00EFA02F636EA0005F5D168
:1024D800D3F808A009FA04F5ED430AEA050AC3F897
:1024E80008A0D3F808B00CFA04FA4AEA0B0AC3F8B1
:1024F80008A0B3F804A01FFA8AFA2AEA06069E8002
:10250800B3F804A008FA02F646EA0A06B6B29E80B4
:102518001E682E401E60D3F800A007FA04F646EAAB
:102528000A061E60D3F80CA001FA04F605EA0A0AA6
:1025380046EA0A05DD60C1E7034AD5692C43D46140
:102548006CE700BF64620308001002401A6822F0BA
:1025580003021A601A683A431A60DA6822F0030222
:102568000A438507DA607FF56BAF1A6822F00C0220
:102578001A601A6842EA87021A60DA6822F00C02C6
:1025880042EA81024407DA607FF55DAF1A6822F0FB
:1025980030021A601A6842EA07121A60DA6822F0F2
:1025A800300242EA0112DA6002077FF54FAF1A687B
:1025B80022F0C0021A601A6842EA87121A60DA68C2
:1025C80022F0C00242EA8112C606DA607FF541AF06
:1025D8001A6822F440721A601A6842EA07221A60DE
:1025E800DA6822F4407242EA01228506DA607FF551
:1025F80033AF1A6822F440621A601A6842EA8722E6
:102608001A60DA6822F4406242EA81224406DA60FB
:102618007FF525AF1A6822F440521A601A6842EA18
:1026280007321A60DA6822F4405242EA0132DA606C
:1026380002067FF517AF1A6822F440421A601A683A
:1026480042EA87321A60DA6822F4404242EA81326A
:10265800C605DA607FF509AF1A6822F440321A60BD
:102668001A6842EA07421A60DA6822F4403242EAFB
:1026780001428505DA607FF5FBAE1A6822F4402234
:102688001A601A6842EA87421A60DA6822F440221D
:1026980042EA81424405DA607FF5EDAE1A6822F419
:1026A80040121A601A6842EA07521A60DA6822F47D
:1026B800401242EA0152DA6002057FF5DFAE1A687D
:1026C80022F440021A601A6842EA87521A60DA68ED
:1026D80022F4400242EA8152C604DA607FF5D1AEA4
:1026E8001A6822F040721A601A6842EA07621A6091
:1026F800DA6822F0407242EA01628504DA607FF506
:10270800C3AE1A6822F040621A601A6842EA876209
:102718001A60DA6822F0406242EA81624404DA60B0
:102728007FF5B5AE1A6822F040521A601A6842EA7C
:1027380007721A60DA6822F0405242EA0172DA60DF
:1027480002047FF5A7AE1A6822F040421A601A68A0
:1027580042EA87771F60DA6822F0404242EA8171D4
:10276800D960BDE8F08F10B1036882881A85704778
:1027780010B1036882889A617047F0B5174F83B02B
:102788000646386AFFF7EFFFE82022F06BFB6C463D
:102798000DF10605002022F065FB04F8010BAC42A0
:1027A800F8D1386AFFF7E4FF9DF804009DF800505F
:1027B8009DF801109DF802409DF803209DF8053012
:1027C80041EA052143EA002342EA04220120B187B5
:1027D800F287A6F8403003B0F0BD00BF941E002079
:1027E80038B5284B284C00211C2518469D71D971F5
:1027F800236221F0E5FF216A0846FFF7B9FF234A63
:10280800138823F040031B041B0C138013889BB20E
:1028180023F0380343F00803138013889BB243F076
:10282800400308461380FFF79EFF242022F01AFB7E
:10283800802022F017FB206AFFF79AFF642004F03B
:102848003BFC206AFFF78FFF202022F00BFBAF2014
:1028580022F008FB206AFFF78BFF012004F02CFC14
:10286800206AFFF780FF232022F0FCFA602022F084
:10287800F9FA206AFFF77CFF6420BDE8384004F0CD
:1028880075BC00BFB8650020941E002000300140D0
:1028980038B100298388026814BF002110218B40B9
:1028A8009361704710B40A4B0A4A1C78012383408D
:1028B800234052F8200029B9B3FA83F149095DF899
:1028C800044BE5E7191C18BF01215DF8044BDFE74D
:1028D800305700203457002030B1036882881B8AA3
:1028E8001A4214BF01200020704703685B6A18472A
:1028F8002DE9F041044618460D46164698462DF037
:1029080031FF2768E6722844A07229467D6943464C
:1029180032462046AC46BDE8F0416047036810B532
:1029280004461B689847236820469B689847A37B02
:102938000133A37310BD10B5036804469B6898471C
:10294800FF2301226373227310BD08B5FFF7BBFA9A
:1029580038B12C2282710022C2712021BDE80840C2
:1029680045E508BD40F2E93300E09BB10289013B2F
:1029780012F0020F9BB2F8D0017340F2E93300E085
:1029880043B10289013B12F0010F9BB2F8D0007BE2
:10299800C0B27047094A904205D0094B984201D00D
:1029A800FF2070470123074A02EB03135A890132BB
:1029B80092B25A815889C0B2704700BF00300140B6
:1029C800003800400057002010B5014600BF074CF2
:1029D80023689868FFF7C7FE23685868FFF7C2FFA7
:1029E80023689868FFF7C4FE00BF10BD4C62002042
:1029F800F8B5574C0601A7190546387A21F0C2FEEA
:102A08003B7A03F01F015B090122022B02FA01F253
:102A180078D0032B71D0012B67D0A3190135187911
:102A2800FFF751FAEDB2074610B11223C571837151
:102A3800A3195879FFF747FA10B11323C5718371A9
:102A4800A3199879FFF73FFA10B11423C571837160
:102A5800A5190E21EA793846FFF7F8FA6879FFF7E1
:102A680032FAEA790E21FFF7F1FAA879FFF72BFA83
:102A7800EA790E21FFF7EAFAA359364A934251D070
:102A8800354A934259D0354A934240D03444227B48
:102A9800002A2FD1012002249A8822F4805212049D
:102AA800120C9A80998889B241F4805199801A88C9
:102AB80002F4415242F44572024322431A809A8832
:102AC80022F470621204120C42F4E0629A809A8B2B
:102AD80022F400621204120C07219A8319821A88C0
:102AE80092B242F040021A80F8BD1D4B996A0A431F
:102AF8009A6292E700200446CEE7194B19690A4307
:102B08001A618AE7164BD9680A43DA6085E702F545
:102B1800EA32116941F400411161116921F400415F
:102B28001161B3E702F56042D16841F48051D16088
:102B3800D16821F48051D160A8E702F5EC3211691F
:102B480041F480411161116921F4804111619DE7CF
:102B5800005700200030014000380040003C004091
:102B680000100240427A02B9704710B50446036863
:102B7800406804F10A0198470023637210BD437A44
:102B88005A1C0344D2B242729972037A934200D813
:102B980002B9704710B504460368406804F10A0199
:102BA80098470023637210BD30B40B4D002305F124
:102BB800140101E0272B0BD011F8132082424FEAB1
:102BC800430403F10103F5D12C44607D30BC704708
:102BD800002030BC704700BFFC3C030870B5448837
:102BE80006460D46C4F30B0422460021284630F061
:102BF800CCFF3369094A934209D3094A934206D262
:102C0800224628461946BDE870402EF03FBD23B144
:102C180021462846BDE87040184770BDFCA403084B
:102C2800F3A50308064B07498B4202D30023184635
:102C380070471A88C2F30B029042F8D01433F3E7B6
:102C480060A00308FCA40308024A136823EA0000F2
:102C580010607047505B0020F8B5174D2B78A32BF8
:102C680028D16B78BE2B25D1022229464FF6FF705A
:102C7800FDF734FD114FAC1C22884AB1A618BE429C
:102C880018D2052A16D92146FDF728FD3446F3E760
:102C980021460222FDF722FD0222A118FDF71EFDA2
:102CA8000634074B641B1C8041F60F53C31A584265
:102CB8005841F8BD0020F8BD00F0030800000408E2
:102CC800763300202DE9F04FDFF848914C4F8BB058
:102CD8000326A7EB09071822002104A830F055FFA6
:102CE800484BCDF8109005971A69120604D5464A44
:102CF8005A6002F188325A6001228DF82420342269
:102D0800DA60424B424C1B88ADF80030022269461B
:102D180004A8FEF735FA022269464FF6FF70FDF760
:102D2800DDFCDFF8F4A080464FF0000B544536D3A5
:102D38000AAC002524F8245D0222214604A8FEF7E7
:102D48001FFA022221464046FDF7C8FC40BAC0439C
:102D5800ADF80800022202A904A8FEF711FA0798A4
:102D680060B106ABC0F104022946184430F00DFFEB
:102D7800069904A8FEF7ABF9079508909DF824304A
:102D8800089A23B11F490B6943F080030B61013E88
:102D98002DD0002A9FD1FFF75FFF50B32CE0658844
:102DA8008DF80DB0C5F30B05AB1DADF808302388C1
:102DB800C3F30B02ADF80A201B0B062202A904A8D4
:102DC8008DF80C30FEF7DCF9062202A94046FDF723
:102DD80085FC616880462A4604A8FEF7D1F9616837
:102DE80040462A46FDF77AFC143480469EE7002ABE
:102DF800D1D0052003F0FAFC0BB0BDE8F08F00BF7E
:102E08000000040800200240230167455E3D0308D6
:102E180060A0030800F00308FCA403080378202B33
:102E2800024600F10100F9D0092BF7D02D2B2CD048
:102E38002B2B03BF5378B7EE000A0246B7EE000A01
:102E4800A3F13001C8B209289FED467A10D8F2EEF6
:102E5800046A07EE901AF8EEE77A12F8013FE7EEF7
:102E6800267AA3F13001C8B20928B0EE677AF0D902
:102E78002E2B4CD003F0DF03452B0BD0F7EE007A56
:102E880067EE276A20EE260A70475378BFEE000ADD
:102E98000246D5E710B451782D2959D02B290ABFFD
:102EA8009178501C901C0024A1F13003092B53D8B1
:102EB800002303EB830301EB430310F8011FA1F187
:102EC8003002092AA3F13003F3D9B3F59A7F28BF5A
:102ED8004FF49A73072B42D9DFED236A1A46F7EEAF
:102EE800007A083A072A67EEA67AFAD803F00703A9
:102EF8002BB1F2EE046A013B67EEA67AFBD124B34C
:102F0800C7EE276A5DF8044B20EE260A704753780F
:102F1800A3F13001C8B2092802F10102AAD8F2EEE1
:102F2800046AF0EE665A07EE901AF8EEE77A12F89D
:102F3800013F87EEA66AA3F13001C8B2092866EE00
:102F4800A56A37EE067AEED994E767EE276AD9E7DD
:102F5800901C91780124A7E7F7EE007ACFE7F7EE07
:102F6800007AC5E70000000020BCBE4CB5EEC00AE0
:102F7800DFED317AF1EE10FACCBF30EE270A30EEF1
:102F8800670ADFED2E7A20EE270A30B5FDEEC07A0B
:102F980087B017EE904A054684EAE470002303A937
:102FA800A0EBE4700193009302931DF055F8002CF8
:102FB800ACBF20232D2303A88DF800302DF0D2FBC1
:102FC800012803A924D002282DD0032805BF3023C7
:102FD800684668468DF8013030F0FDFD68462DF0F2
:102FE800C1FB0338C4B222466946284630F051FE78
:102FF80000232B5528462DF0B5FB2E22431C2A54BE
:103008000DEB0401E81830F003FE284607B030BD88
:10301800302368468DF801308DF802308DF8033082
:1030280030F0D9FDDAE7302368468DF801308DF8A5
:10303800023030F0D0FDD1E76F12033A00007A4435
:103048002DE9F041064615460846B6FBF2F43CB9B0
:1030580005FB1464124B1B5D00F8013BBDE8F081D1
:10306800B4FBF2F767B90E4B05FB174705FB146471
:10307800DA5D00F8012B1B5D00F8013BBDE8F0812B
:10308800B7FBF2F8B8F1000F02D04046FFF7D8FFBF
:1030980005FB1878024B13F8082000F8012BE3E72A
:1030A800586B030830B402681146531C036011F8CA
:1030B800024B0160D31C517803609378151D05609D
:1030C8001B0443EA0123D078234343EA006030BC61
:1030D80070470368591C1A46016012F8021B026007
:1030E800587841EA0020704703685A1C0260187833
:1030F800704738B50446006815462EF0C7FA2268AE
:103108002A44226038BD036810B40A0A5C1C0460B3
:103118001A7003685A1C026019705DF8044B7047F6
:1031280003685A1C026010B4197003680A0A5C1C10
:1031380004601A7003680A0C5C1C04601A70036847
:10314800090E5A1C026019705DF8044B7047036839
:103158005A1C026019700368090A5A1C0260197027
:1031680070472DE9F047002488B080460F461E4678
:10317800A14605AD531C0393117839B3252933D1E2
:10318800931CCDF810900393507830284ED04FF010
:10319800000AA0F13003DBB2092B42D96C2819D000
:1031A800642800F0938024D825281CD063D9582897
:1031B80076D063281BD131784046B847039A531C10
:1031C80003931178043601340029D7D1204608B07A
:1031D800BDE8F087039B5A1C03921B78642B7CD0B4
:1031E8002AD8252B54D1252140460134B847039AC3
:1031F800C0E7732833D044D975284FD106F1040E9F
:1032080030682B4600220A217646FDF763F9049AB6
:103218000095534639464046FDF799F9039A044408
:10322800A8E704AA03A91CF0F3FEB7E7D31C03938D
:1032380090784FF0010AACE7732B10D05BD9752B4F
:103248003AD0782B96D1A3F15802B2FA82F23068BC
:1032580052092B4610210436FDF73CF9D7E73368AD
:10326800049A0093394600234046FDF770F9043666
:103278000444039A7EE70028B9D1204608B0BDE887
:10328800F0876E28B3D1039A336804361C6071E75F
:103298002AD9582BD7D0632B8DD06BE77828A6D1A5
:1032A800A0F15802B2FA82F2306852092B46102176
:1032B800FDF710F90436AAE706F1040E30682B462C
:1032C80000220A217646FDF705F9A0E7331D30688C
:1032D80029461E46FDF7D0F899E7331D3068294680
:1032E8001E46FDF7C9F892E7002B7FF443AF20464E
:1032F80008B0BDE8F0876E2BC6D03BE70EB400B52A
:1033080084B005AB019053F8042B0649039301A838
:10331800FFF727FF019B00221A7004B05DF804EB49
:1033280003B070474D0500080FB430B583B006AB45
:103338000B490C4853F8042B096800680193FFF700
:1033480010FF094C0546206803685B699847002808
:10335800F9D0284603B0BDE8304004B0704700BF3C
:10336800C4320020C8320020FC760020DFED2B7A22
:10337800B4EEE70AF1EE10FA4ADDDFED296A9FEDB7
:10338800297A01E0B0EE670AB4EEC70AF1EE10FA46
:1033980070EE667AF6DC9FED247AF4EEC77AF1EEE9
:1033A80010FA38D5DFED1E6A9FED207A01E0F0EEC5
:1033B800407AF4EEC77AF1EE10FA37EEA60AF6D4A0
:1033C800DFED1B7AB4EEE70AF1EE10FA14DDDFED5B
:1033D800137A37EEC00A60EE006A9FED166A9FED19
:1033E800167ADFED167AA6EE867A20EE266AE6EEE3
:1033F800877AA6EE270A7047DFED117AB4EEE70A5E
:10340800F1EE10FA44BFDFED087A37EEC00AE2E7C2
:10341800F0EE407ABFE7B0EE670AD1E7DB0F49402C
:10342800DB0FC940E4CB1641DB0F49C0E4CB16C122
:10343800DB0FC93F92E741B99730083C15A82ABE6F
:10344800DB0FC9BF80EAE073A3EBE0738B4205DBB7
:10345800002801DD401A704702D1704700207047EC
:103468000844704709B909E0194690FBF1F301FBDC
:1034780013030846002BF7D1084670470146FBE7BF
:103488009FED317A70EE077AFDEEE76A16EE903A14
:103498002033402B02D99FED2D0A7047B4EEC70A9E
:1034A800F1EE10FA0FDDB0EE677A9FED296ADFEDD5
:1034B800296A01E0B0EE677AB4EEE67AF1EE10FA26
:1034C80077EEC67AF6DC9FED247AF4EEC77AF1EE51
:1034D80010FA0FD5B0EE677A9FED1D6ADFED1F6A0F
:1034E80001E0B0EE677AB4EEE67AF1EE10FA77EE24
:1034F800867AF6D49FED147AF4EEC77AF1EE10FAD4
:103508001DDC9FED177AF4EEC77AF1EE10FA44BF8E
:103518009FED117A77EE677A27EEA76ADFED115AE9
:10352800DFED116A9FED117AE6EE256A67EE865A9D
:10353800A6EE267AE5EE877AB0EE670A70479FED29
:103548000C7A77EE677AE7E7DB0FC93F00000000E7
:10355800DB0FC940E4CB1641DB0F49C0E4CB16C1F1
:10356800DB0FC9BF92E741B99730083C15A82ABEBE
:10357800DB0F494010B507EE901A2DED028BB8EE1F
:10358800678ADFED217A28EE008A044628EE278A2A
:10359800B0EE480A2EF03AFAF0EE408AB0EE480A49
:1035A8002EF096F9F7EE007A9FED187AF0EE675A4A
:1035B800E8EE875A0023A361B0EE676AC7EEA56AF2
:1035C80063612362E361A8EEC76ABDEC028B77EE04
:1035D800C07AB6EE007AF8EE005A27EE877A20EE27
:1035E800250A27EE267A26EE266A67EEA67A20EEC8
:1035F800260A84ED046AC4ED017A84ED007A84ED2C
:10360800027A84ED030A10BD27D4D236F304353F7D
:1036180010B44C09012250F8243001F01F0102FABD
:1036280001F10B4340F824305DF8044B70474B0917
:1036380001F01F0150F82320012303FA01F1114280
:1036480014BF184600207047074A084B10781B78AB
:10365800074A834296BFC31AC3F180030020126849
:1036680018441044704700BF646F0020E16E0020CA
:10367800183B0020064A074B10781B7883428ABF04
:10368800C3F18003C01AC018C0F17F00704700BFA3
:10369800646F0020E16E002030B5144C237883B0AD
:1036A8001BB90120237003B030BD052200238DF81B
:1036B80000208DF8013000BF0D4D2B689868FFF78A
:1036C80052F82B6801AA6946586825F0ADF82B68AE
:1036D8009868FFF74DF800BF9DF8053003F0010327
:1036E80083F00100237003B030BD00BF5E6200208C
:1036F8004C62002070B5064C0646256803E0236836
:103708005B1BB34203D8FFF7C7FF0028F7D070BD93
:10371800685700202DE9F04F89B0B2F1000A0290F5
:103728000491039340F3B0800B46002201EB8A0119
:1037380053F8040B8B420244FAD1039B0592002BE9
:1037480000F09A80059B002B6AD0544B059A1B68A1
:10375800DFF85C9100920099DAB25118B1F5807FD8
:103768008CBFC2F58072009A01924D4A92689A42C3
:103778006DD9190C1A0A4FF0020406208DF81F3073
:103788008DF81E208DF81D108DF81C40FFF7B2FF34
:103798000620FFF719F9434A0123137000BFD9F82F
:1037A80000309868FEF7DFFFD9F8003007A958689D
:1037B800002224F0F1FF0024049D029E019FA346ED
:1037C80029684FEA840800220B46013471B1B942D6
:1037D8002AD2D9F8000031684068FCF7AFFD2A68A2
:1037E800336813443360BF1AC5F800B0A24505F129
:1037F800040506F10406E3D1D9F800309868FEF70D
:10380800B7FF00BF254B019900981B68421A009228
:10381800224A0B441360039A32B3009A002A9AD1C1
:10382800059809B0BDE8F08F029CD9F8003054F82B
:103838000810586800223B46FCF780FD54F8082021
:103848002B683A44DF1B44F808202F60D4E705981A
:10385800009C1549154A001B0590059800230B701C
:10386800137009B0BDE8F08F059B009A9B1A059369
:10387800059809B0BDE8F08FFFF70EFF00287FF428
:1038880061AF039B0593CBE7039C1CB9FFF704FFCB
:103898000594C5E700230593C2E700BF183B002045
:1038A800D80D00205E620020646F0020E16E0020C9
:1038B8004C62002070B5104D104E2B7831788B4239
:1038C80084B016D00E4A03921A4402928CBF0C465A
:1038D800CA1A04A98CBFC3F180020024012341F84D
:1038E800102D02A802220194FFF714FF0023337061
:1038F8002B7004B070BD00BFE16E0020646F002023
:10390800E46E002070B5194C194D23782978994236
:1039180084B027D0174A03921A44029234BF0E4645
:10392800CA1A04A934BFC3F180020026002341F853
:10393800102D02A802220196FFF7ECFE2378184406
:10394800C0B203062B7848BF80F080008342207005
:1039580002D0002004B070BD002301202B7023701A
:1039680004B070BD012004B070BD00BFE16E00203E
:10397800646F0020E46E002008B545F20820FFF7C8
:10398800B9FE0620FFF720F8064B0122C7201A705F
:10399800FFF71AF804480549054A002303700B701D
:1039A800136008BD5E620020646F0020E16E002095
:1039B800183B00202DE9F04182B00346060C050AA9
:1039C800032406208DF80730884617468DF80560D1
:1039D8008DF806508DF80440FFF78CFEC0B100BF8B
:1039E8000D4C23689868FEF7BEFE236801A9586845
:1039F800002224F0D1FE23684246002158683B4645
:103A0800FCF79CFC23689868FEF7B2FE00BF3846B6
:103A180002B0BDE8F08100BF4C620020F0B5124B47
:103A28009D6885B00DB905B0F0BDED0A14D000272A
:103A380004AE7C196410E00210226946FFF7BAFF51
:103A48000F2809DD6B4653F8042B01320AD1B34223
:103A5800F9D12546AF42ECDBFFF72CFF034BED0213
:103A68001D60E0E7671CF5E7D80D0020183B002033
:103A7800704770B50446806815460E46FEF773FE1B
:103A8800012003F019FB31466068FEF76BFF2946F9
:103A98006068FEF767FFA068FEF76AFE012003F082
:103AA8000BFB012070BD2DE9F04383B00F4615468E
:103AB8000446FFF7DEFF642003F0FEFA1B4E47F0D2
:103AC80080084FF01509A068FEF74DFE012003F0AD
:103AD800F3FA41466068FEF745FF01230DF107023E
:103AE80000216068FCF72AFCA068FEF741FE01206F
:103AF80003F0E2FA9DF80730AB422A4639462046E1
:103B080010D0F3880133F380FFF7B3FF642003F08C
:103B1800D3FA09F1FF3010F0FF09D4D1484603B0B9
:103B2800BDE8F083012003B0BDE8F08324740020D1
:103B3800F8B54F4E96F824700446002F2ED0A06991
:103B48004C4B98426CD0A3F57843984279D021F039
:103B5800B7F92046FDF7CFF894F93E30013308D085
:103B6800A369444A934262D0A2F5784293426AD04C
:103B7800F8BD94F93C300133F2D1A3693D4A934230
:103B880072D0A2F5784293426BD02AF05FFD3A4991
:103B98003A4B3B483B4A0860DA60F8BD04F114052B
:103BA800806921F09FF980226B212846FFF761FF89
:103BB800322003F0DBFA01226B212846FFF773FF5E
:103BC80094F85330042B34BF18221A2228461B219C
:103BD800FFF769FF94F85230042B3BD0032B94BFB6
:103BE80007223A461A212846FFF75DFF94F8542029
:103BF80019212846FFF757FF10221C212846FFF7F6
:103C080052FF122237212846FFF74DFFA06921F005
:103C180057F9012386F82430A069164B984292D1AF
:103C28000022194B03EB021300225A818FE7164B2F
:103C38005A8992B2A2B1002203EB021300225A81E0
:103C4800A3E70122EDE7104B5A8B92B2002A8FD0DE
:103C58000122F1E701221A212846FFF724FFC5E7D0
:103C6800F8BD0122084BE7E70022074BE4E700BF55
:103C7800941E002000300140FC9F002000ED00E071
:103C8800EFBEADDE0400FA0500570020B0F1FF3F9B
:103C98000AD0022810B403DC5DF8044BFDF7DAB84B
:103CA80000205DF8044B70470020704710B40446AC
:103CB800134690F904000A4661795DF8044BE5E77C
:103CC8000278012A00D070474821EFE70278012ADC
:103CD80000D070475821E9E70378012B00D07047DE
:103CE8003122F421E2E7044B93F820209201343288
:103CF80002F0FC02F421D9E7B03B00202E22F42187
:103D0800D4E7002310B52A2204461C211846FFF7E1
:103D1800BDFF02230E221C210020FFF7B7FF03235B
:103D28000F221C210020FFF7B1FF12232B221C2198
:103D38000020FFF7ABFF02232C221C210020FFF7F5
:103D4800A5FF01232D221C210020FFF79FFF002340
:103D580018462E221C21FFF799FF05232A221C2131
:103D68000020FFF793FF4FF48073A38210BD10B5B6
:103D780080232422192104460020FFF787FF6420AE
:103D880003F0F4F99723202219210020FFF77EFF82
:103D98000A2003F0EBF91023232219210020FFF752
:103DA80075FF642003F0E2F94FF48053A38210BD3D
:103DB80010B590F852304E2B1DD05D2B19D0362BF4
:103DC8000CBF4F240F24642003F0D0F9F0232322E2
:103DD80068210020FDF73EF808B924F027FA0520ED
:103DE80003F0C4F92346202268210020BDE81040D2
:103DF8004CE7CF24E7E78F24E5E710B5082304460E
:103E08000F2218210020FFF741FF0E23102218214E
:103E18000020FFF73BFF4FF48053A38210BD38B555
:103E2800194B1C78054608232D22532194B92046A6
:103E3800FFF72CFF0A23312253212046FFF726FFE4
:103E48000A2320462C225321FFF720FF4FF48073CA
:103E5800AB8238BD0020FFF719FF0A233122532116
:103E68000020FFF713FF0C232C2253210020FFF71B
:103E78000DFF9023382253210020FFF707FF4FF44E
:103E88008073AB8238BD00BF04460020F0B55B4BA1
:103E98005B4A97B01968914200AF00F0A380594976
:103EA800594A00234FF47000C1F888003B607B60DA
:103EB800136843F48033136003E03B68B3F5A04F05
:103EC80009D0136803F400337B603B6801333B601F
:103ED8007B68002BF1D04C4B1B6813F4003318BFE0
:103EE80001237B607B68012B52D0464C464B474AE6
:103EF800E260474A596A11605A6A42F080725A620F
:103F08005A6942F4FC025A610025032207F10801AC
:103F1800012341F6FF764FF09040FD60BE603A7392
:103F2800BB731FF063FF4FF6FF7307F108013948B1
:103F3800BB601FF05BFF07F108013748374E1FF0E1
:103F480055FF07F1080136481FF050FF07F1080137
:103F580034481FF04BFF07F1080133481FF046FFB4
:103F680007F108001FF052FDBB683049304AA1FB39
:103F7800031330499B0CF0204FF0070E5C370B60A1
:103F8800566084F823009560C2F800E0BD46F0BD95
:103F9800294A1D4B122111605A685A605A685A60A2
:103FA8005A6842F480625A605A6822F47C125A6055
:103FB8005A6842F4E8125A601A6842F080721A602D
:103FC8001A689201FCD559680F4A21F0030159601B
:103FD800596841F002015960536803F00C03082B3B
:103FE800FAD182E700221A6062B6144B1B6883F389
:103FF8000888134B1B689847FEE700BFFC9F00200A
:10400800EFBEADDE00ED00E0001002400005FA054D
:10401800AC46002000040048000800483F19010091
:10402800000C0048001000480014004883DE1B43C1
:1040380010E000E06C5700200020024000D8FF1F6D
:1040480004D8FF1F70B50F4C0F4DC0EBC00004EB38
:104058008004686926693043686182B09209667B8A
:10406800A1600025012101A863618DF804608DF825
:1040780005208DF806508DF807101FF0F1FB02B0EF
:1040880070BD00BF3C06002000100240074BC0EB8B
:10409800C00030B403EB8000054C056963692B430D
:1040A80063610176427630BC704700BF3C06002051
:1040B800001002402DE9F04F5E4C54F8204083B0C8
:1040C800002C71D0666D984691465B4B7268E2642D
:1040D800A160236004F15A014FF4807304F5AD72B6
:1040E8006161A261E36023610746307E20F04AFBEC
:1040F800F068A8B1514B00215A68904203F11C03A3
:1041080000F0928001310C29F6D100207A1CD2B23D
:104118000C21FFF7BBFFE36CF26822632433A3642E
:10412800B068D8B1454B00215A68904203F11C038E
:1041380078D001310C29F7D100257A1CD2B20B2195
:104148002846FFF7A3FF2346F27E3D492846FFF79E
:1041580079FFE36CB26862632833636494F85900AA
:10416800FDF7B1FE054694F85800FDF7ACFE18F0CF
:10417800080F824696F819B01AD0CDB118F0110F71
:104188004FF00B0307F1010714BF4E213E21EF71D9
:104198005A46AB712846FDF759FF18F0010F45D074
:1041A800236B5BB3636B4BB3204603B0BDE8F08F62
:1041B80018F0010F0CBF4FF02E084FF04E0819F001
:1041C800020F09D045B10B227B1CAA71EB7128465E
:1041D8005A464146FDF73AFF19F0010FE0D0BAF10F
:1041E800000FDDD001370C238AF807705A46414684
:1041F8008AF806305046FDF729FFD1E7337FB27EB3
:104208008DF804209B090021012201A88DF80530B2
:104218008DF806108DF807201FF022FB204603B00A
:10422800BDE8F08FCDB288E7C8B26FE72846FEF741
:104238009AFAB5E7D0320020603D03083C0600201A
:104248000F1700080348D0F83C3113B100F59A70F5
:10425800184770473C0600200348D0F8203113B1B6
:1042680000F58C70184770473C0600200348D0F8CA
:1042780004310BB1FC301847704700BF3C060020E2
:104288000348D0F8E8300BB1E0301847704700BF5A
:104298003C0600200348D0F8CC300BB1C430184796
:1042A800704700BF3C0600200348D0F8B0300BB17F
:1042B800A8301847704700BF3C0600200348D0F8D4
:1042C80094300BB18C301847704700BF3C06002073
:1042D8000248836F0BB17030184770473C060020C6
:1042E8000248C36D0BB15430184770473C06002094
:1042F8000248036C0BB13830184770473C06002061
:104308000248436A0BB11C30184770473C0600202E
:104318000248836803B11847704700BF3C06002075
:10432800F0B53E4C059D00EB800004EB800464680A
:10433800002C71D03A4E49004FF42040CFB2B06102
:10434800A169090454D46068DFF8E0E047F49031CB
:1043580000EA0E0001434FF420406160B06103E0C1
:10436800411E002848D00846A1698907F8D54FF4AE
:104378002040A262B06103E0421E00283CD01046F3
:10438800A2695206F8D5274A6168DFF8A0E0B06153
:1043980042EA0342174301EA0E0217436760C3B1BA
:1043A800013BDBB201332B44A0694FF4204210F0EB
:1043B800040002F1FF3207D1511C26D0A06910F089
:1043C800040002F1FF32F7D0626A05F8012B9D4222
:1043D800EAD14FF42040B06102E0431E60B11846B4
:1043E800A3699B06F9D52023B061E3610120F0BDE4
:1043F800411E08B10846A3E70B4A138801339BB254
:104408004FF0FF311380B161F0BD0749B2610B88ED
:1044180001339BB20B80F0BD2046F0BDD85600207A
:10442800941E00200024000274330020009800FC31
:1044380070B590F904506C1C82B00AD0022D08DCCB
:1044480016460A46417900962846FFF769FF02B0EA
:1044580070BD002002B070BD00B50378012B83B099
:1044680004D1032301AA0021FFF7E2FF9DF80530DC
:104478009DF804209DF806001B0243EA02431843F6
:1044880003B05DF804FB08B5FFF7E6FF014B586081
:1044980008BD00BF941E002008B5FFF7DDFF014BE3
:1044A800186008BD941E002070B50378012B82B0F7
:1044B80004D106236A46F721FFF7BAFF9DF80120C9
:1044C8009DF804309DF800609DF803509DF8024067
:1044D8009DF80500074912011B0142EA063243EA2A
:1044E800053342EA141243EA1013CA608B6002B023
:1044F80070BD00BF941E002010B582B001AA03232E
:10450800F621FFF795FF9DF80530094A9DF804400C
:104518009DF80600B2F9202006491B0243EA04432D
:104528000343C2F10802D3404B6102B010BD00BF83
:10453800B03B0020941E002000B583B001AA0223DE
:10454800F621FFF775FF9DF804109DF80530034A22
:1045580043EA0123138203B05DF804FB941E002094
:10456800F0B585B002AB04460093032206231E2152
:104578000020FFF7D5FE00283CD09DF808509DF894
:1045880009109DF80A709DF80B209DF80C609DF8A5
:104598000D3041EA052142EA072243EA062309B21F
:1045A80012B21BB2144D06EE901A07EE102A07EE4F
:1045B800903AF8EEE66A95ED035AD5ED055A95ED71
:1045C800046AB8EEC77AF8EEE77A66EE856A27EEEF
:1045D800257A67EE867AFDEEE66ABDEEC77AFDEECD
:1045E800E77A16EE901A17EE102A17EE903A218005
:1045F800A280638005B0F0BD000000202DE9F043E3
:10460800322083B002F0B2FD0022104611231E2191
:10461800FFF73CFB602301221E210020FFF736FB39
:10462800642002F0A3FD6846FFF79AFF0024DFF834
:104638005481254626460A27012302221E210020EE
:10464800FFF724FB322002F091FD6846FFF788FF50
:10465800BDF902E0BDF90410BDF900208E4573468E
:10466800A8BF0B469342A8BF134643454FF001002D
:1046780075440C44164479DBFDF794F8013FDBD10F
:104688004FF001090022104612231E21FFF7FEFAFF
:10469800DFF8F0800A27012302221E210020FFF7FD
:1046A800F5FA322002F062FD6846FFF759FFBDF9BE
:1046B80002E0BDF90410BDF900208E457346A8BF7D
:1046C8000B469342A8BF134643454FF00100A5EBA4
:1046D8000E05A4EB0104A6EB02064ADBFDF762F81F
:1046E800013FD8D107EE906AF8EEE76A07EE905AD4
:1046F800B8EEE77A07EE904ADFED1F5A9FED1F5A92
:104708001F4EF8EEE77A85EEA66A0022104670235F
:104718001E21C5EE876A85EE277AB0EEC66AF0EEEE
:10472800E66AF0EEC77A86ED036AC6ED046AC6ED5E
:10473800057AFFF7ABFA202301221E210020FFF79C
:10474800A5FA0023184602221E21FFF79FFA6420CB
:1047580002F00CFDB9F1000F04D14FF07E53F36065
:1047680033617361012003B0BDE8F0834FF00009A5
:1047780088E74FF00009B5E700406F4601C05E4684
:104788000000002001F0FFFFF0B587B00DF10F0326
:1047980005460093022201230C210020FFF7C0FDEB
:1047A80018B19DF80F30DB0703D40024204607B06A
:1047B800F0BD04AB0093032206230C210020FFF771
:1047C800AFFD0DF10F030093092201230C210020F6
:1047D800FFF7A6FD04460028E7D09DF80F0010F06B
:1047E8000C00E2D19DF811E09DF810109DF81370AF
:1047F8009DF812209DF815609DF8143041EA0E21AD
:1048080042EA072243EA0623C1EB8131C2EB823236
:10481800C3EB8333890092009B0029806A80AB80B8
:104828000A2201230C21FFF731FABFE710B5002354
:1048380084B018460A220C21FFF728FA142002F047
:1048480095FC0F230A220C210020FFF71FFA0A20EB
:1048580002F08CFC03AB0093102203230C210020F0
:10486800FFF75EFD0A2002F081FC002318460A22A9
:104878000C21FFF70BFA0DF10B040A2002F076FC6D
:104888000094012302220C210020FFF749FD009427
:10489800012309220C210020FFF742FD01230A22EF
:1048A8000C210020FFF7F2F9012004B010BD00B57B
:1048B80083B0002000920A466821FFF731FD03B05B
:1048C8005DF804FB10B584B002AB044600930122E6
:1048D80006231C210020FFF723FD30B39DF8082094
:1048E8009DF809309DF80A1043EA022343F38D032B
:1048F800002BB8BF03339DF80B209B1042EA01221E
:10490800E3829DF80C109DF80D3042F38D0243EAC6
:104918000123002A43F38D03B8BF0332002BB8BF2D
:10492800033392109B102283638304B010BDF0B54B
:1049380085B002AB04460093A82206231921002063
:10494800FFF7EEFC00B39DF809709DF808109DF87C
:104958000B609DF80A209DF80D509DF80C3041EA37
:10496800072142EA062243EA052309B212B21BB222
:1049780001EBD17102EBD27203EBD37349105210E1
:104988005B10E1822283638305B0F0BDF0B585B08A
:1049980002AB04460093A822062368210020FFF7F3
:1049A800BFFCA8B19DF808709DF809109DF80A6031
:1049B8009DF80B209DF80C509DF80D3041EA072119
:1049C80042EA062243EA0523A187E287A4F8403099
:1049D80005B0F0BDF0B585B002AB044600930222E5
:1049E800062318210020FFF79BFCB8B19DF8091099
:1049F8009DF80B209DF80D309DF808709DF80A6011
:104A08009DF80C50090212021B0201EB970102EB00
:104A1800960203EB9503E1822283638305B0F0BD20
:104A28002DE9F04F364B1B7885B08146002B3FD0DF
:104A380000242546264627460DF1080800E043B322
:104A48000134CDF800800823322253210020E4B23B
:104A5800FFF766FCA8B39DF809B09DF808109DF80B
:104A68000BA09DF80A209DF80DC09DF80C309DF80C
:104A78000FE003EB0C2301EB0B2102EB0A22202CA5
:104A880005FA83F507FA81F706FA82F60EF07F0336
:104A9800D5D197FBF4F796FBF4F6A9F8167095FBB9
:104AA800F4F4A9F81860A9F81A4005B0BDE8F08F29
:104AB80002AA18460092062332225321FFF730FC3F
:104AC80018B9002005B0BDE8F08F9DF809609DF881
:104AD80008109DF80B509DF80A209DF80D409DF890
:104AE8000C3001EB062102EB052203EB0423A9F8A5
:104AF8001610A9F81820A9F81A3005B0BDE8F08FEB
:104B0800044600201749184B184A194810B4D1F820
:104B1800884044F47004C1F888401C6844F00104DB
:104B28001C605C6822405A601A6822F0847222F481
:104B380080321A601A6822F480221A605A6822F4B5
:104B4800FE025A60DA6A22F00F02DA621A6B002457
:104B580010404FF0006218639C608A605DF8044B57
:104B6800704700BF00ED00E0001002400CC07FF865
:104B7800CCFC00FF38B50B4C23688BB15A68821AFD
:104B8800002A054604DA0CE05A68AA1A002A07DB4C
:104B98009A68226018461A6890472368002BF3D158
:104BA80038BD38BD144200200B4B002210B40272ED
:104BB80003F58274112102E0072A09DC9979890733
:104BC80002D51979815401329C4203F11403F3D1BF
:104BD8005DF8044B704700BF6C620308282303701C
:104BE800704700BF30B401233025332431213222ED
:104BF8004570C4714171C270037083710371837011
:104C080030BC70472C22022302704370704700BFEB
:104C1800436A8269D154436A0169426B01338B420A
:104C280028BF00234362002A2FD0EFF311815023BD
:104C380083F31288436B1A68D2072CD470B45E6869
:104C48006EB9456A826A954217D084691444DC605B
:104C58000ED9AA1A5A608562002280F850201A6874
:104C680042F00102C9B21A6081F3118870BC704722
:104C78000469A21A5A608662EEE7012380F8503070
:104C8800C9B281F3118870BC7047C26C136843F0D5
:104C9800800313607047C9B281F31188704700BF61
:104CA800026B10B462B1036CC2684469D11A013B4B
:104CB800615C5DF8044B08BF13460364C8B27047D3
:104CC800016A4369C4685B5C0131A14228BF11468F
:104CD80001625DF8044BD8B2704700BF436B13B153
:104CE80090F850007047836A406A181AB0FA80F04A
:104CF80040097047416A836A99420AD3CB1A416BCB
:104D0800026961B14968501E0B4483420AD2C01A35
:104D1800704702691144CB1A416B0029F2D1501E29
:104D2800C01A704700207047036B43B1026C5B6880
:104D380093422FBF981AC0689B1AC0187047C2695F
:104D4800036A9A422FBFD01AC0688018C01A7047E9
:104D580008B514F01DFC024B024ADA60FEE700BFFA
:104D680000ED00E00400FA05024A034B12781978B6
:104D78001CF028BEFF1E0020001F00202DE9F04770
:104D88000569C3681D4028D00F4606464FF0004805
:104D98004FF00009B5FA85F328FA03F2D2431B3B1A
:104DA80032611540042B16D8DFE803F031292119A8
:104DB80003007B6A002B32D003F1FF3A1FFA8AFA0C
:104DC800C7F824903C6A34B1236820465146984776
:104DD8006468002CF8D1002DDCD1BDE8F087386874
:104DE800716B036889B29847002DD3D1F5E77868CD
:104DF800B16B036889B29847002DCBD1EDE7B8684D
:104E0800F16B036889B29847002DC3D1E5E7F868CC
:104E1800316C036889B29847002DBBD1DDE7F36A8E
:104E28001FFA83FACEE700BF2DE9F04F2DED028B74
:104E3800A0F10A0389B00C46E72B00F24C86DFE8A4
:104E480013F01C014A064A064A064A064A064A065A
:104E58004A064A064A064A064A064A064A064A06CA
:104E68004A064A064A064A064A064A064A064A06BA
:104E78004A062D014A064A064A066B054A064A06AC
:104E88004A064B014A0658014A065D024A062C02A8
:104E98004A0624024A06D3034A06FC014A064A0681
:104EA8004A06F501EE014A06E7014A064A06E0010C
:104EB8004A06B8014A064A064A069C014A064A06B4
:104EC8004A064A06E1054A06FC004A064D04010660
:104ED8004A064A064A064A064A064A064A0629056C
:104EE8004A06EC044A06B8044A0664044A06100254
:104EF8004A064A064A064A06B6057B05D905250626
:104F0800E8004A064A069A031A034A06E302C70259
:104F18004A064A064A064A06BC024A064A069B024E
:104F28004A064A064A068C027502860344034A0664
:104F38004A064A0635034A0626032D044A064A0647
:104F48004A064A064A064A064A064A064A064A06D9
:104F58004A064A064A064A064A06B6054A064A065E
:104F68004A064A064A064A064A064A064A064A06B9
:104F78004A064A064A064A064A064A064A064A06A9
:104F88004A064A064A064A064A064A064A064A0699
:104F98004A064A064A064A064A064A064A064A0689
:104FA8004A064A064A064A064A064A064A064A0679
:104FB8004A064A064A064A064A064A064A064A0669
:104FC8004A064A064A064A064A064A064A064A0659
:104FD8004A064A064A064A064A064A064A064A0649
:104FE8004A064A064A064A064A064A064A064A0639
:104FF8004A064A064A064A064A064A064A064A0629
:105008004A064A064A064A064A064A064A06220442
:10501800F803A74E337853B1A64F002537F8021F7F
:105028002046FEF794F833780135AB42F6DC0120D0
:1050380009B0BDEC028BBDE8F08F9D4E3378002B94
:10504800F5D09D4F0025B846236817F81520591C40
:1050580021601A7098F8011001EB810101EB8101C0
:1050680001F2EE2189B22046FEF771F83378013556
:10507800AB4208F10208E7DCD9E7904D28462BF04F
:1050880071FB0028D3DD2B460544226813F8011B69
:10509800501C9D4220601170F7D1C8E7884D05F17A
:1050A8005006287829F0B8FA2368027A591C21603A
:1050B8001A7023686A78591C21601A702368AA78C4
:1050C800591C21601A702368EA780435591CAE42CD
:1050D80021601A70E5D1AAE70B687A4A581C117842
:1050E8002060197023685278591C216001201A70B9
:1050F8009EE7754D0B682A7A591C21601A70A98B96
:105108002046FEF724F8298B2046FEF720F8698B05
:105118002046FEF71CF82368EA7C591C21601A70A7
:10512800A98C2046FEF713F8E98C2046FEF70FF805
:105138002368AA7F591C21601A70236895F82020DB
:10514800591C21601A70698C2046FEF700F8236804
:10515800EA7A591C21601A70E9682046FDF7E0FFD9
:1051680023682A7C591C21601A70236895F821202D
:10517800591C216001201A705AE7FEF78DFA23683E
:10518800524D002803F101010CBF022203222160C5
:105198001A7029882046FDF7C3FFA9682046FDF745
:1051A800BFFFFEF751FA01462046FDF7B9FF01207F
:1051B8003EE70B68434A464D1178464A581C206022
:1051C800197011682046FDF7ABFF23683E4A591C49
:1051D800127A21601A7029882046FDF7B8FFA9883D
:1051E8002046FDF7B4FF29892046FDF7B0FF0021CE
:1051F8002046FDF7ACFF20460021FDF7A8FF01205F
:1052080016E7084608223049FDF773FF01200FE72B
:105218000B68314A581C91782060197062E70B6856
:1052280001229918216010461A7001E72B4B084695
:105238001968FDF775FF0120FAE6294D294E05F199
:10524800300795F90210284B93F906208A4203F19A
:10525800080300F043849E42F6D10835BD42F0D1E0
:10526800E5E60B68214A2249D078224A5D1C256070
:10527800187023684979581C206019702368D278FF
:10528800591C216001201A70D2E60B680E4A591C7D
:10529800527D216001201A70CAE6174D05F180067B
:1052A80055F8041F2046FDF73BFFAE42F8D1BEE695
:1052B8002C5500204A530020CC59002030380020BB
:1052C800343B0020303B0020AC6D0020D80D00207E
:1052D800FC320020505B0020EC780020143C0020B9
:1052E80064620020A86D0020786D0020F44500203D
:1052F8002C400020A03B0020843C0020A94D05F153
:105308004006B5F880102046FDF721FF236895F880
:105318008220591C21601A70236895F8832004356F
:10532800591CAE4221601A70EBD180E60A689E4B88
:105338009E491878551C2560107022685878551CAD
:105348002560107022689B78501C206013702046DE
:10535800C988FDF7FCFE01206AE6944D08462988B5
:10536800FDF7F5FE69882046FDF7F1FE2046A9887D
:10537800FDF7EDFE01205BE68D4D05F16006A9887D
:105388002046FDF7E4FEE9882046FDF7E0FE29897E
:105398002046FDF7DCFE2368AA7A591C21601A70A2
:1053A8002368EA7A591C21601A7055F80C1B2046AC
:1053B800FDF7B6FEAE42E2D139E67E4952232268B5
:1053C800501C2060137011F8013F002BF7D12EE616
:1053D800794800232268056803EB4301561C6D5C7D
:1053E80026601570026825680A446E1C527826608B
:1053F8002A70026825680A4401339278691C0A2BCE
:1054080021602A70E6D112E66C4D0B682A68591C97
:10541800127821601A702B6822689978531C2360CF
:10542800002311702A6821681A4401335279481CF4
:10543800032B20600A70F5D123682A68591C127A58
:1054480021601A7023682A68591CD27821601A7062
:1054580023682A68591C127921601A702B68204623
:105468005989FDF774FE2A682368527A591C21600D
:105478001A702A6836E6524B08461968FDF750FE3E
:10548800504B20461988FDF762FE0120D0E54E4BAF
:105498004E49B3F9003081FB0321DB17C3EBA101AF
:1054A800204689B2FDF753FE0120C1E5484D084664
:1054B800A98AFDF74CFEE98A2046FDF748FE2046FA
:1054C800298BFDF744FE0120B2E5DFF818E100273B
:1054D800FEB2714600232268501C206016702268B4
:1054E800501C20601370226811F8010F0133551CFD
:1054F800062B25601070EED10137062F0EF1060E2F
:10550800E6D1344900232268501C206017702268B5
:10551800501C20601370226811F8010F0133551CCC
:105528000B2B25601070EED123681E4A581C0721EA
:105538002060197023680021581C206019702368A6
:1055480092F8F020591C216001201A7070E50B6850
:10555800214A224910781C4A5D1C2560187023686E
:105568008978581C2060197023689278591C21602A
:1055780001201A705CE51A4D08462988FDF7E7FDF9
:1055880069882046FDF7E3FDB5F904300F4AD917BD
:1055980082FB0323C1EBA301204689B2FDF7D7FDA7
:1055A800012045E5883C00208C3400200C38002080
:1055B80030730020883D03088054002000560020E6
:1055C800B834002020200020A03B002067666666D3
:1055D800806700206B3D0020146C0020F4450020FB
:1055E80004550020473D0020A34B03F15A052268CB
:1055F8005979501C2060117022681978501C20605D
:10560800117022685978501C2060117022689978AE
:10561800501C206011702268D978501C20601170CD
:10562800226819790633501C9D4220601170DED122
:10563800FDE4924B03F1700522681978501C206034
:10564800117022685978501C20601170226899786E
:10565800501C206011702268D978501C206011708D
:1056680022681979501C2060117022685979501CE1
:1056780020601170226899790733501C9D42206080
:105688001170D9D1D3E47E4D0846E989FDF75FFD55
:105698002046A989FDF75BFD0120C9E40B68794F15
:1056A800591C3A7821601A703B78002B3FF4BFAC44
:1056B8000025EEB2304627F039FE23684278591C9F
:1056C800216030461A7027F031FE01892046FDF727
:1056D8003EFD3B780135AB42EBDCA8E40B680025C6
:1056E8005A1C0A601D700B685A1C0A601D700B68F2
:1056F8005A1C0A60204629461D70FDF711FD2046F8
:105708002946FDF70DFD012092E400212046FDF712
:105718001EFD00212046FDF71AFD00212046FDF759
:1057280016FD2368584D00265A1C22601E702368F7
:105738002A68591C92F82C2021601A7023682A685C
:10574800591C92F8362021601A7023682A68591C5F
:1057580092F8372021601A7023685A1C22601E7044
:1057680023685A1C22601E7023685A1C22601E700F
:105778002B682046598FFDF7EAFC2B682046198FC5
:10578800FDF7E5FC23682A68591C92F82E20216051
:105798001A7023685A1C22601E702B682046598E86
:1057A800FDF7D5FC2B682046998EFDF7D0FC01202B
:1057B8003EE4364E0B687279334D591C21601A70DD
:1057C8002B682046198CFDF7C2FC2B682046D98B24
:1057D800FDF7BDFC71892046FDF7B9FCB18920466B
:1057E800FDF7B5FC2B682046598CFDF7B0FC2B68FB
:1057F8002046998CFDF7ABFCF1892046FDF7A7FC04
:10580800318A2046FDF7A3FC2A68236892F82620EF
:10581800591C216001201A700AE41C4EF378002BF1
:1058280000F046820B680822591C21601A70236810
:105838000122991821601A702368154D591C2A797C
:1058480021601A702368AA78591C21601A70298867
:105858002046FDF77CFC698A2046FDF778FC236822
:10586800F279591C21601A702368EA78591C216062
:1058780001201A70FFF7DCBBE43500209870002087
:10588800F44500200174002080540020146C00208E
:10589800806700201CF07AF8FF28064600F0168280
:1058A80008A9002501F8125D0DF10D008DF80D50C5
:1058B8001CF04CF808A800F8115D1CF03BF808A88B
:1058C80000F8105D1CF02AF808A820F8085D1CF004
:1058D80019F823685A1C22601E7023689DF80D2051
:1058E800591C21601A7023689DF80E20591C2160EC
:1058F8001A7023689DF80F20591C21601A702368BC
:105908009DF81020591C21601A702046BDF8181007
:10591800FDF71DFCFFF78BBB9F4D08462988FDF757
:1059280016FCA9882046FDF712FC20462989FDF7B8
:105938000EFC0120FFF77CBB984B9B8AB3F5006FE8
:1059480000F2C281B3F5806F00F2E381B3F5007F06
:1059580034BF01270227924D05F10C0655F8041BA8
:1059680091FBF7F1204689B2FDF7F1FBAE42F5D184
:105978008C4D8D4F05F10C06B5EC010AD7ED087A70
:1059880080EE270A2BF0F6FF81B22046FDF7DFFBF9
:10599800B542F1D1854D05F10C0655F8041B20469A
:1059A80089B2FDF7D4FBAE42F7D1FFF740BB002523
:1059B8008146DFF82482DFF824B205950495069520
:1059C800079501214FF6FF7A05E001350B2D00F010
:1059D800A38018F9011F4F1C4AFA05F3F5D0DE071A
:1059E800F3D5BBF800302B41D807EED506A8FDF754
:1059F8000FFEEAE7084610226D49FDF77AFB012001
:105A0800FFF716BB0B686B4D591C2A7921601A7079
:105A180023686A79591C21601A7029882046FDF785
:105A280096FB2368AA79591C21601A706988204658
:105A3800FDF78DFB2368EA79591C216001201A7053
:105A4800FFF7F6BA0B685C4E01255A1C0A601D70F8
:105A58000B68B278591921601A7014F0F1FC2368A8
:105A6800564A57495F1927601870B1F90010B2F902
:105A78000000FDF7F7FC23685A1922601870318876
:105A88002046FDF764FB2846FFF7D2BA4D4D4E4E2F
:105A9800DFF84C81DFF84C919FED4C8A05F1200727
:105AA80008E020460435FDF752FBAF4206F1180620
:105AB8003FF4BDAA717C0029F3D098F80030D5EDE9
:105AC800007A012B00F00981FCEEE77ACDED017A2E
:105AD800BDF80410E5E70020FFF7AABA23685A1CAE
:105AE8002260197029882046FDF731FB2368EA787F
:105AF800591C21601A7023682A79591C21601A7070
:105B08002368AA79591C21601A7023686A79591C7C
:105B180021601A70FFF7A1BBDFF8CCA000254FF079
:105B280008080135C5F1200208FA02F2A5F12003A0
:105B38002AFA05F6164328FA03F31E43252D06F024
:105B480001024FF000030BD01343EAD0E8B21DF076
:105B5800FDFA0028E5D0294606A8FDF759FDE0E73B
:105B68001B4B1B78DA0700F1C4800025194E2F461D
:105B780002E00135252D39D029463046FDF757FD7D
:105B88000028F6D0294606A8FDF751FD002840F068
:105B98008A800137EDE700BFFC320020AC540020BA
:105BA800E45400202C6C0020BC5F0020F45400203A
:105BB800F438002028380020365B00205A390020AD
:105BC8005C39002004390020606600200000404253
:105BD8003556002074770020B83D0308FC3D0020AE
:105BE800A8670020386C002090E33FF46C4B6D4DA3
:105BF800B3F850102046FDF7AAFA6B4B19882046D7
:105C080089B2FDF7A4FA694B19684B0103F0200229
:105C1800C1F340031343C1F3800243EA4203C1F3D3
:105C2800C00243EA8203C1F3401243EAC20301F00F
:105C3800100119432046FDF78AFA04A904222046D8
:105C4800FDF757FA23682978594A581C20601970BB
:105C580011886429A8BF64212046FDF778FAB9F1B4
:105C6800960F4BD000212046FDF771FA2168B7F155
:105C7800190348BFA7F11203A3F3C4034A1C226007
:105C880020461A460B7005A9FDF733FA2368494ADE
:105C9800581C10212060197020461188FDF740FA21
:105CA8000120FFF7C5B9394604A8FDF7B1FC70E734
:105CB8000B68B178404A581C206019702368127824
:105CC800591C21601A70B7E5082744E623685A1C56
:105CD800226001201E70FFF7ABB9D9F80030DB0451
:105CE80019D5F5EE407AF1EE10FA1CD140F2DC51EC
:105CF800D7E6069B43F00103069336E723680322A1
:105D0800591C21601A7023686A78591C21601A701E
:105D1800ACE704271FE6F4EEC87AF1EE10FA1FDAB2
:105D28004FF47A71BDE6F4EEC87AF1EE10FADDD4DC
:105D38009FED227AF4EEC77AFDEEE77AF1EE10FADB
:105D480017EE901A1DD86FF4F973303903FB01F17F
:105D580040F2E73391FBF3F101F2DB5189B2A0E69F
:105D6800FDEEE77A40F2E73317EE901A303903FB7D
:105D780001F140F2CF7391FBF3F101F2E93189B2FD
:105D88008FE640F2F313A1F5836103FB01F140F2C2
:105D9800E73391FBF3F101F2DD5189B281E600BFEF
:105DA800900000207454002074330020A854002070
:105DB80078330020C83D00204872002000E082446B
:105DC80008B501210220FCF76DFD094B1B7803F093
:105DD8000503052B08D000210120FCF763FD0021F5
:105DE8000846FCF75FFDFEE713F02CFCF3E700BF65
:105DF800CC320020022828BF022010B4084C094BDE
:105E0800207000EB8002C0EBC20207495DF8044B2A
:105E1800013003EB4203C0B20B6029F0DBBD00BFC9
:105E2800745400201A5A00208054002008B520F02D
:105E380077F9FCF747FFBDE8084020F059B900BFE3
:105E480038B5434B5A899989914224BF00225A8117
:105E5800198ADA89914224BF0022DA81DA788AB372
:105E6800072A2FD03B493C4D91F8570001240021C7
:105E78000A282C709C70D9713DD00C2865D0DFEDB4
:105E8800377A8ABB364C9FED370AA278002918BFAB
:105E9800F0EE407A062A04D8334901EB820191EDED
:105EA8000F0A217959B3013A032A4DD8F7EE007A3F
:105EB80087EE800A2BF05EFD2388984228BF18469B
:105EC800208038BDD97921B198780428B8BF04203A
:105ED8009870204890F857000A280CD00C28CED18A
:105EE800DFED227A002ACDD0072ACBD00A282CD180
:105EF800DFED1F7AC6E70A20DFED1E7AC1E79B783F
:105F0800154A07EE103A1178B8EEC77A27EE277AC5
:105F180007EE901AF8EEE77A67EE877AB4EEE70AAA
:105F2800F1EE10FA10DDC0EE077AFDEEE77A17EE13
:105F3800903A102BA8BF1023012BB8BF0123DBB266
:105F48008B4238BF0B46137038BDDFED0B7A99E7EB
:105F5800146C0020BC5F0020487200206F120339C7
:105F6800806700206F120338883D03080AD7A339D9
:105F78000F506E3A5304E9386F12833A38B50C4C17
:105F88000C4DAC4206D2616820461434FCF726FE5C
:105F9800AC42F8D3084A094B094C1460002209495D
:105FA8001A705A7008480860BDE8384016F092BD6B
:105FB80060A00308FCA40308805400207454002047
:105FC8001A5A0020005600208454002008B5FFF714
:105FD800D5FF20F0A5F8FCF775FEBDE8084020F0D5
:105FE80087B800BFF0B50C292BD8DFE801F06F2A7D
:105FF8002A2A4C2A2A2A2B2A2A2A0700046AB2F8B3
:106008000CE097881668674D24F480540462036A8C
:106018004468C16923F4005343EA0E3321F4E6418E
:10602800A84243EA073341EA062100F0B58005F5A6
:106038000065A84200F0B08092684460C1610264C3
:106048000362F0BD046A96899588D2F800E0554F3E
:1060580024F480740462036A4468C16923F40073F9
:1060680043EA062321F07301B84243EA052341EAD3
:106078000E017ED04C4DA8427BD092684460C1612D
:10608800C2630362F0BD046A96899588D2F800E07D
:10609800444F24F010040462036A4468816923F0C1
:1060A800200321F0807143EA061321F4E641B84247
:1060B80043EA051341EA0E2148D03B4DA84245D09A
:1060C80092684460816182630362F0BD046A9389C7
:1060D800B2F804E01768334E24F001040462056A3C
:1060E8004468816943EA0E0321F4803125F00205F2
:1060F8009BB221F07301B04243EA050341EA07016C
:1061080014D0294DA84211D005F54065A8420DD0FC
:1061180005F58065A84209D005F58065A84205D037
:1061280092684460816142630362F0BDD689158A32
:10613800578A23F0080333433D43D68824F4407438
:1061480023F00403ADB233432C43E9E7D589178A1A
:10615800D68823F0800343EA051324F44064558A63
:1061680023F0400344EA870443EA061344EA85041B
:10617800A6E7D589178AD68823F4006343EA05235E
:1061880024F44054558A23F4806344EA071443EA0C
:10619800062344EA051470E7158A24F4804444EA87
:1061A800851449E7002C0140003401402DE9F04FE7
:1061B8004FF48C72002183B07848794CDFF8049250
:1061C800784D794E794FDFF800822DF0DEFC784863
:1061D8007849DFF8F8E1DFF8F8C100221359834263
:1061E80000F0C280B3F1804F00F0C080AB4200F0F5
:1061F800C980B34200F0C880BB4200F0C780734535
:1062080000F0C680634500F0C580434500F0C480B7
:10621800DFF8C0A153457FD00AF5806A534508BF0F
:1062280009237AD01432B2F58C7FD7D15C4C624DF9
:10623800624E604F04F58C7802E01434A04568D0B3
:10624800A379002BF9D023794FEA131909F1FF3903
:10625800B9F1050F03F00F03EFD835F8190040FA2C
:1062680003F2D207E9D54FF0010A0AFA03F3013B1A
:1062780018402AF071FF16F809305149184411EBFB
:10628800C002DAD051F83000DFF84CE1217A00F191
:1062980038439B0A1EF8033003F01F0E5B09022BDC
:1062A8000AFA0EFA69D0032B62D0012B03D17B695D
:1062B8004AEA03037B6193880093B3FA83F3C3F13B
:1062C8001F039BB2DA0800EB820203F00703D2F83F
:1062D80020E09B004FF00F0C0CFA03FC2EEA0C0E8A
:1062E800C2F820E0D2F820E001FA03F343EA0E03F3
:1062F800136269460023022214348DF804208DF8B5
:1063080005308DF806308DF807301DF06FFDA0457B
:1063180096D103B0BDE8F08F082309EBC3034FF013
:10632800010B93F85CA00AF01F034FEA5A1ABAF15E
:10633800020F0BFA03F30BD0BAF1030F0ED0DA45B4
:106348007FF470AFD1F814A043EA0A034B6169E700
:10635800D1F818A043EA0A038B6163E7D1F81CA0BF
:1063680043EA0A03CB615DE70023D6E70123D4E7BC
:10637800FB694AEA0303FB619DE7BB694AEA030339
:10638800BB6198E70223C8E70323C6E70423C4E7F1
:106398000523C2E70623C0E70723BEE78C240020B5
:1063A8006C62030800040040000800400010004030
:1063B800002C014000100240D8660308E466030878
:1063C800A0630020883D03080040014000140040FD
:1063D8000034014000440140646203080149024856
:1063E800FEF7CCBC7C25002000480140014902484A
:1063F800FEF7C4BC2C2500200034014001490248A6
:10640800FEF7BCBC2C25002000340140014902489D
:10641800FEF7B4BC042500200008004001490248EA
:10642800FEF7ACBCDC2400200004004002494FF019
:106438008040FEF7A3BC00BFB424002010B5064C72
:1064480006482146FEF79AFC04F1C8010448BDE855
:106458001040FEF793BC00BF8C240020002C0140A4
:106468000044014001490248FEF788BC8C24002002
:10647800002C01402DE9F0410468514DA30AAB42BC
:1064880000F084800AD94F4DAB4277D00135AB423A
:106498005FD0053DAB426DD0BDE8F0814A3DAB42CF
:1064A80070D00135AB4258D0B3F5801FF4D14FF00E
:1064B800480E012647794FEA970C00296AD0B000A8
:1064C800634685190227D4F80C809F400CEB4503DE
:1064D800BFB23D4D03F1040C47EA080745F8231005
:1064E80045F82C20E760EFF31181502282F31288DF
:1064F800821905EBC2021369002B32D013620433F0
:10650800821905EBC202576917B11F60536904333A
:10651800821905EBC202976917B11F6093690433AA
:10652800821905EBC202D76917B11F60D36904331A
:106538000027CAB21F6082F31188304405EBC000FF
:10654800036A8BB9E3684FF6FE721340E360BDE857
:10655800F0814FF4887E0626ACE74FF0980E0326AC
:10656800A8E705EB0E03CBE7E36843F00103E3601C
:10657800BDE8F0814FF0C00E04269BE74FF0E80E0F
:10658800052697E74FF0700E022693E74FF0200E8E
:1065980000268FE7BF08022306FA03F0BB40DB435F
:1065A800E768094D9BB23B4087190CEB470CE36049
:1065B8000CF1040345F82C1045F8232093E700BF9D
:1065C8004B001000510010008C24002030B50368E7
:1065D8005C4D18885C4CB4FBF2F20139013AAB42CD
:1065E80094B283B089B282B266D05848834263D0ED
:1065F800B3F1804F60D0A0F5983083425CD000F5AD
:106608008060834258D0524883425BD000F5806056
:1066180083427DD022F4407200F58C3092B28342DE
:106628001A80D9621C850ED0484A93420BD002F5D5
:106638004062934207D002F58062934203D002F58C
:106648008062934201D100221A8601225A611A8877
:106658003C4992B242F001028B421A8062D0B3F1F7
:10666800804F61D03B4A934260D002F580629342EA
:106678005ED002F5006293425CD002F580629342DC
:106688005AD002F59032934258D002F540629342B4
:1066980056D002F5806293421ED002F58062934282
:1066A80008BF092219D002A84FF0012340F8043D81
:1066B8001DF0D6F803B030BD254822F070028342A1
:1066C80092B2A3D101201A80D9621C8558611A8818
:1066D80092B202431A80C5E708221F4B03EBC2039C
:1066E80001A893F85D408DF80440012300228DF83D
:1066F80005308DF807308DF806201DF0B1F81B2CF9
:10670800D8D1164B019301A81DF0AAF803B030BDEB
:1067180001201A80D9621C8558611A8892B20243F6
:106728001A809CE70022D8E70122D6E70222D4E7A4
:106738000322D2E70422D0E70522CEE70622CCE7DF
:106748000722CAE7002C014000A24A040034014095
:106758000010004000040040883D030819010001B2
:10676800204B98422DD0B0F1804F2CD0A3F5943314
:1067780098422AD003F58063984228D003F5006335
:10678800984226D003F58063984224D003F59033CD
:10679800984222D003F54063984220D003F58063E5
:1067A800984207D003F58063984208BF092202D0B7
:1067B8000020704708220C4B03EBC20393F85C00DF
:1067C80070470022F7E70122F5E70222F3E70322E8
:1067D800F1E70422EFE70522EDE70622EBE70722BF
:1067E800E9E700BF002C0140883D03082DE9F04F80
:1067F800013085B0C3B203938E4D8F4F8F4C904EAE
:106808000A230293DFF840921EF01CFD4FF4FA7A37
:106818004FF0100C4FF47A70D9F80430C3F3080322
:10682800002B40F0C880EFF31183002B40F0C380A9
:106838002968A26800BF2B689942F9D1D7F800E00F
:1068480000FB0EF39B1AB3FBFEF300FB01314FF084
:10685800010E0191D9F80430C3F30803002B40F06E
:106868008E80EFF31183002B40F089802B68A1689C
:1068780000BF2A689342F9D1D7F800B000FB0BF2A9
:10688800521AB2FBFBF200FB0323019A9B1AB3F5E1
:106898007A7FDFD3BAF1010ABED1039B002B40F007
:1068A800C4804FF47A7ADFF8A09150464FF0100C6C
:1068B800D9F80430C3F30803002B40F09980EFF3B4
:1068C8001183002B40F094802968A26800BF2B68D0
:1068D8009942F9D1D7F800E000FB0EF39B1AB3FBFD
:1068E800FEF300FB01314FF0010E0191D9F804309D
:1068F800C3F308033BBBEFF3118323BB2B68A168E9
:1069080000BF2A689342F9D1D7F800B000FB0BF218
:10691800521AB2FBFBF200FB0323019A9B1AB3F550
:106928007A7FE3D3BAF1010AC2D1029B013B0293F9
:106938007FF468AF4349444B4448454A0860DA60ED
:1069480005B0BDE8F08FEFF311888CF31288A168C9
:106958002368DB0344BFC6F800E0A1682B683268EF
:106968005FFA88F888F31188D7F800801A4400FB8A
:1069780008F35B1AB3FBF8F300FB0233CDE7EFF340
:1069880011888CF31288A1682368DB0344BFC6F81A
:1069980000E0A1682B6832685FFA88F888F31188EC
:1069A800D7F800801A4400FB08F35B1AB3FBF8F32E
:1069B80000FB023369E7EFF311828CF31288D4F8F5
:1069C80008E02368D90303D501233360D4F808E02D
:1069D8002B683168D2B282F311883A68194400FBF7
:1069E80002F3A3EB0E03B3FBF2F300FB01312EE736
:1069F800EFF311828CF31288D4F808E02368D903E6
:106A080003D501233360D4F808E02B683168D2B28B
:106A180082F311883A68194400FB02F3A3EB0E03D2
:106A2800B3FBF2F300FB01315DE718461EF06EFA86
:106A380037E700BF685700206C57002010E000E0DF
:106A480064570020FC9F002000ED00E0EFBEADDEA3
:106A58000400FA052DE9F047AF4FB04E1FF060FB78
:106A6800BE421ED2DFF83C83DFF83C9344462588BB
:106A780062197DB14A450DD2052D0BD9338861883D
:106A8800C3F30B03994200F0F58014462588621978
:106A9800002DEFD1716830461436FCF79FF8BE42DE
:106AA800E4D39F4A1378A3F1170102290FD99D490E
:106AB80011F83300002840F0FF80D80001444978DD
:106AC80029B1994911F83330002B00F01D81974CFA
:106AD8006378022B84BF002363702378022B84BF62
:106AE80000232370924B9A78042A00F0048132B96B
:106AF8001A88B2F5F07F84BF4FF4F0721A808D4D7A
:106B08008D4A2B681A40002A00F00181D80700F14D
:106B1800ED80590400F1E5801A0700F1DD809B043F
:106B280000F1D380854D2B685A8C998C914224BFF3
:106B380000225A84FFF784F923F09AFD10B980489F
:106B480028F016FB4020FCF77FF88020FCF77CF843
:106B58004FF48020FCF778F84FF40010FCF774F835
:106B68004FF00070FCF770F84FF08060FCF76CF89D
:106B78006378022B06D8734A734903EB430302EB8D
:106B880083030B602378022B07D803EB83016F4A3A
:106B9800C3EBC10302EB43032B601CF04FFB002146
:106BA80030226B482CF0F1FF286825F0C9FD694BAD
:106BB8002E6803F1500102E0043399427AD01A7822
:106BC800002AF9D19C78D8788442F5D26249634B7F
:106BD80091F804E06248634D5C6B634B2860C827FA
:106BE800642111FB0E71DFF8C4E159605F4F30F882
:106BF800061C5F4DAEF8001000219960D96019613C
:106C080059619961D96183F8201083F821103A708D
:106C18002E600CB117F0DAFB564B9FED575A1B88C4
:106C2800564A9FED576A5579564C57495748086058
:106C380006EE903AF8EEE66A1388C5EE265A07EE95
:106C4800103A53881279C4ED005A07EE903AB8EE1C
:106C5800C77A4F4BF8EEE77A1D725A7227EE067A1A
:106C680067EE867ABDE8F04783ED017AC3ED007AD6
:106C78001FF03EBA63799B077FF407AF716894F8F9
:106C880004A03046FBF7AAFF3388BAEB133F04D0C1
:106C98001436BE42FFF4EAAE03E773887068AA1F91
:106CA800C3F30B039A4204F10601A8BF1A462AF05F
:106CB800EDFCEDE7012289E7D8000C186468002C88
:106CC8007FF4FCAE17241470F8E63248FBF7BCFFDB
:106CD8004020FBF7B9FF25E72F48FBF7B5FF2B68E6
:106CE8001DE72E48FBF7B0FF2B6815E72C48FBF78C
:106CF800ABFF2B680DE71A8BB2F57A7FBFF4FFAEB6
:106D08004FF47A721A83FAE618231370DFE643F415
:106D180000532B60FAE600BFFCA4030860A0030838
:106D2800303B0020BC5D0308F06703087454002062
:106D380080670020505B002009600002805400201A
:106D48006462002084540020005600201A5A002053
:106D580088220020343B002028380020AC54002032
:106D6800FA4500204C770020A43D0020D4050020DF
:106D7800BC220020C4340020C0C9FB48EC1E0020FF
:106D880017B7D138C8340020A03500203661023D3D
:106D98007C35002009400002016000020920000241
:106DA8000860000202F0030800000408844500207F
:106DB80008B51FF0B5F9FBF785FF1FF099F9FFF744
:106DC80049FE0120BDE8084028F004BE2DE9F04F37
:106DD800013085B0C3B203930B4602918B4C8C4EA5
:106DE800002B00F099808B4D8B4FDFF830921EF00E
:106DF80029FA4FF4FA7A4FF0100C4FF47A70D9F858
:106E08000430C3F30803002B40F0DE80EFF3118356
:106E1800002B40F0D9802968A26800BF2B689942EE
:106E2800F9D1D7F800E000FB0EF39B1AB3FBFEF391
:106E380000FB01314FF0010E0191D9F80430C3F382
:106E48000803002B40F08780EFF31183002B40F0FC
:106E580082802B68A16800BF2A689342F9D1D7F8CD
:106E680000B000FB0BF2521AB2FBFBF200FB03234B
:106E7800019A9B1AB3F57A7FDFD3BAF1010ABED122
:106E8800039B002B40F0BD804FF47A7ADFF88C9199
:106E980050464FF0100CD9F80430C3F30803002B08
:106EA80075D1EFF31183002B71D12968A26800BF57
:106EB8002B689942F9D1D7F800E000FB0EF39B1A32
:106EC800B3FBFEF300FB01314FF0010E0191D9F83D
:106ED8000430C3F3080313BBEFF31183FBB92B682A
:106EE800A16800BF2A689342F9D1D7F800B000FB27
:106EF8000BF2521AB2FBFBF200FB0323019A9B1A16
:106F0800B3F57A7FE3D3BAF1010AC4D1029B013BFE
:106F18000293002B7FF467AF05B0BDE8F08FEFF365
:106F280011888CF31288A1682368DB0344BFC6F874
:106F380000E0A1682B6832685FFA88F888F3118846
:106F4800D7F800801A4400FB08F35B1AB3FBF8F388
:106F580000FB0233D2E7EFF311888CF31288A168A3
:106F68002368DB0344BFC6F800E0A1682B683268D9
:106F78005FFA88F888F31188D7F800801A4400FB74
:106F880008F35B1AB3FBF8F300FB023370E7EFF387
:106F980011828CF31288D4F808E02368D90303D54A
:106FA80001233360D4F808E02B683168D2B282F349
:106FB80011883A68194400FB02F3A3EB0E03B3FBF4
:106FC800F2F300FB01317FE7EFF311828CF31288B3
:106FD800D4F808E02368D90303D501233360D4F833
:106FE80008E02B683168D2B282F311883A681944F4
:106FF80000FB02F3A3EB0E03B3FBF2F300FB01313A
:1070080018E718461DF082FF3EE700BF10E000E0D9
:1070180064570020685700206C57002000ED00E0FE
:10702800204B5B68C3F3080330B4BBB9EFF311839B
:10703800A3B91D4B1D4C1868A16800BF1A6890427F
:10704800F9D11B4B1C684FF47A7202FB04F3591AEE
:10705800B1FBF4F130BC02FB00107047EFF3118272
:10706800102383F3128811498C680B6813F4803F4E
:10707800104B02D0012018608C680B49D2B20D6801
:10708800186882F311880A4B19684FF47A722844F9
:1070980002FB01F31B1B30BCB3FBF1F302FB003016
:1070A800704700BF00ED00E06857002010E000E0E6
:1070B8006C570020645700202DE9F84F8046FFF7F1
:1070C800AFFF254E2549DFF8A0E0254A254D844627
:1070D80010274FF47A740120DEF80430C3F3080354
:1070E800D3B9EFF31183BBB90B68D2F808A000BF7E
:1070F800D1F800904B45F7D1D6F800B004FB0BF956
:10710800A9EB0A09B9FBFBF904FB0393A3EB0C03F6
:107118004345E1D3BDE8F88FEFF3118A87F312886E
:10712800D2F808B01368DB0344BF2860D2F808B06F
:107138000B68D5F800905FFA8AFA8AF31188D6F8B6
:1071480000A0994404FB0AF3A3EB0B03B3FBFAF387
:1071580004FB0933DAE700BF6C57002068570020AA
:1071680010E000E06457002000ED00E02DE9F04F4A
:10717800DFF830C1474A4849484E494D80461027F4
:1071880018F1FF38C0F08480DCF80430C3F308033A
:10719800002B5CD1EFF31183002B58D10B68946856
:1071A80000BF08688342F9D1D6F800904FF47A708E
:1071B80000FB09FEAEEB040EBEFBF9FE00FB03EE7E
:1071C800DCF80430C3F308034FF47A740120FBB9E8
:1071D800EFF31183E3B90B68D2F808A000BFD1F828
:1071E80000904B45F7D1D6F800B004FB0BF9A9EB9A
:1071F8000A09B9FBFBF904FB0393A3EB0E03B3F5F0
:107208007A7FBDD2DCF80430C3F30803002BDFD04B
:10721800EFF3118A87F31288D2F808B01368DB03FA
:1072280044BF2860D2F808B00B68D5F800905FFA20
:107238008AFA8AF31188D6F800A0994404FB0AF365
:10724800A3EB0B03B3FBFAF304FB0933D5E7EFF326
:10725800118487F31288D2F808901368D80303D5ED
:1072680001232B60D2F808900B682868E4B284F3F5
:107278001188D6F800A04FF47A7400EB030E04FBD3
:107288000AF3A3EB0903B3FBFAF304FB0E3E97E7FB
:10729800BDE8F08F10E000E0685700206C57002030
:1072A8006457002000ED00E030B4EFF311831022A2
:1072B80082F312880649074C0A68074801320025FC
:1072C8000A602560DBB2026883F3118830BC70471E
:1072D800685700206457002010E000E00F4B1B881F
:1072E800014643B90E4B0F4A1B7810680BB981F061
:1072F8000101FBF7CDBA0C4B5A691AB118B91A68D3
:10730800106058747047094A18681188084A92FB37
:10731800F1F2012102605974704700BF4057002004
:10732800425700204457002048570020605700204B
:1073380020A107001D4B70B51C69E36C226BDD6949
:10734800C2B1636B2BB12B0702D5E36C08221A621A
:1073580070BD2A06F7D5A26A616A8A421FD0511CFD
:10736800A069A162825C2069E66C81423285EAD319
:10737800A362E8E7A906E4D5E26A1AB1988C80B25C
:107388009047DEE7E1699B8C6069DBB24E1CE661E1
:107398004354E169E368994228BFE261D1E7E26CAE
:1073A800136823F080031360CDE700BFD0320020BC
:1073B8001D4B70B5DC68E36C226BDD69C2B1636B91
:1073C8002BB12B0702D5E36C08221A6270BD2A067E
:1073D800F7D5A26A616A8A421FD0511CA069A162CE
:1073E800825C2069E66C81423285EAD3A362E8E7D1
:1073F800A906E4D5E26A1AB1988C80B29047DEE714
:10740800E1699B8C6069DBB24E1CE6614354E1691B
:10741800E368994228BFE261D1E7E26C136823F080
:1074280080031360CDE700BFD03200201D4B70B53C
:107438009C68E36C226BDD69C2B1636B2BB12B07CF
:1074480002D5E36C08221A6270BD2A06F7D5A26A33
:10745800616A8A421FD0511CA069A162825C2069BE
:10746800E66C81423285EAD3A362E8E7A906E4D54F
:10747800E26A1AB1988C80B29047DEE7E1699B8C8A
:107488006069DBB24E1CE6614354E169E3689942E6
:1074980028BFE261D1E7E26C136823F08003136030
:1074A800CDE700BFD03200201D4B70B55C68E36C9F
:1074B800226BDD69C2B1636B2BB12B0702D5E36C7C
:1074C80008221A6270BD2A06F7D5A26A616A8A4242
:1074D8001FD0511CA069A162825C2069E66C8142C0
:1074E8003285EAD3A362E8E7A906E4D5E26A1AB1CD
:1074F800988C80B29047DEE7E1699B8C6069DBB2CB
:107508004E1CE6614354E169E368994228BFE26191
:10751800D1E7E26C136823F080031360CDE700BF66
:10752800D03200201D4B70B51C68E36C226BDD69FE
:10753800C2B1636B2BB12B0702D5E36C08221A6228
:1075480070BD2A06F7D5A26A616A8A421FD0511C0B
:10755800A069A162825C2069E66C81423285EAD327
:10756800A362E8E7A906E4D5E26A1AB1988C80B26A
:107578009047DEE7E1699B8C6069DBB24E1CE661EF
:107588004354E169E368994228BFE261D1E7E26CBC
:10759800136823F080031360CDE700BFD0320020CA
:1075A80070B4EFF31186502383F31288436B1A6883
:1075B800D20720D45D686DB9446A826A944217D0B4
:1075C80081691144D9600ED9A21A5A6084620022D6
:1075D80080F850201A6842F00102F1B21A6081F373
:1075E800118870BC704701698A1A5A608562EEE793
:1075F800012380F85030F1B281F3118870BC7047D4
:107608002DE9F04F95B0B0F908500D81EDB2442D39
:1076180000AF0C46904600F04784064643D9812DBA
:1076280000F07D8300F29880542D00F0CC8040F269
:1076380062836E2D00F00684802D40F0CD80734B60
:1076480093F800A00AF1020A1AF0FF0A00F09780E6
:107658006F4BDFF8EC816F4EDFF8E8B19A4403F125
:1076680001090A2516E0322D01F00683A5F13C0038
:10767800C0B2132841F2078300232268511C2160FD
:1076880015702268D14502F101012160137076D08E
:1076980019F8015B0A2DE6D1BBF80030FF2BA8BF13
:1076A800FF23DBB2E9E7052D00F0EC8320D8022D9B
:1076B80000F0818040F20C83032D00F0B783042D85
:1076C80040F08A802A4654492046FBF712FD0021E3
:1076D8002046FBF73CFD22680021531C012523604E
:1076E80028462B46543711706381BD46BDE8F08F9C
:1076F800242D5ED040F2A282282D00F05983382D27
:107708006AD10A68454B0125511C21601570226811
:10771800052150192060117022680A215019206033
:1077280011702268002150192060117022681978A0
:107738005019206011702268597850192060117012
:1077480022689978531923602B46117028465437BC
:107758006381BD46BDE8F08FA02D18D040F28D8220
:10776800B82D00F06183FE2D36D12D4D05F10806A8
:1077780035F8021B2046FBF7EAFCB542F8D1012593
:107788002B46284654376381BD46BDE8F08F254B0C
:1077980008461968FBF7C4FC234B20461968FBF719
:1077A800BFFC224B196820460125FBF7B9FC2B4684
:1077B800E7E71F4BF6E704221E4920460125FBF7A1
:1077C80098FC2B46C2E70B681B491022581C206006
:1077D8001A702268097880E721462846FDF724FBBD
:1077E80003460028CBD1742D00F08B82772D2BD146
:1077F8003268716891421EBF531C336011780F4A7A
:1078080008BF1946204626F0B3FEB8E701740020E9
:10781800303E03080426002079540020055A002031
:1078280024740020ACF7FF1FB0F7FF1FB4F7FF1F49
:10783800505B0020806B0308FC1E0020A9DA0208B8
:10784800676666662C260020F52D01F0C382472D59
:1078580000F05683292D336801F08282392D01F01A
:107868006C82212D01F0498271680B3DCA1AEF2DF7
:1078780000F2C18401A050F825F000BFAB860008D3
:10788800FF810008FF810008FF810008FF810008D0
:10789800FF810008FF810008FF810008FF810008C0
:1078A800FF810008FF810008FF810008FF810008B0
:1078B800FF810008FF810008FF810008FF810008A0
:1078C800FF810008FF810008FF810008FF81000890
:1078D800FF810008FF810008FF8100085786000823
:1078E800FF81000835860008FF8100080B86000824
:1078F800FF810008FF810008FF810008B1870008A8
:10790800FF8100083B870008FF81000809870008FD
:10791800FF810008E3860008FF810008F985000858
:10792800FF810008A1850008FF810008198500086B
:10793800FF810008FF810008FF810008FF8100081F
:1079480087770008FF810008FD840008FF81000890
:10795800FF810008618C0008FF810008CB8B0008BC
:10796800FF810008FF810008FF810008FF810008EF
:10797800BF8B0008FF810008FF810008FF81000815
:107988007F8B0008FF8100089F890008FF8100089D
:10799800FF81000861890008FF810008FF81000855
:1079A800FF810008FF810008FF810008FF810008AF
:1079B800FF8100088D880008FF810008D98700082A
:1079C800FF8100089D8A0008FF810008ED890008F2
:1079D800FF810008578B000863810008FF810008B9
:1079E800FF810008FF810008FF810008FF8100086F
:1079F800FF810008FF810008FF810008FF8100085F
:107A0800FF810008FF810008FF810008FF8100084E
:107A1800FF810008FF810008FF810008FF8100083E
:107A2800FF810008FF810008FF810008FF8100082E
:107A3800FF810008FF810008FF810008FF8100081E
:107A4800FF810008FF810008FF810008FF8100080E
:107A5800FF810008FF810008FF810008FF810008FE
:107A6800FF810008FF810008FF810008FF810008EE
:107A7800FF810008FF810008FF810008FF810008DE
:107A8800FF810008FF810008FF810008FF810008CE
:107A9800FF810008FF810008FF810008FF810008BE
:107AA800FF810008FF810008FF810008FF810008AE
:107AB800FF810008FF810008FF810008FF8100089E
:107AC800FF810008FF810008FF810008FF8100088E
:107AD800FF810008FF810008FF810008FF8100087E
:107AE800FF810008FF810008FF810008FF8100086E
:107AF800FF810008FF810008FF810008FF8100085E
:107B0800FF810008FF810008FF810008FF8100084D
:107B1800FF810008FF810008FF810008FF8100083D
:107B2800FF810008FF810008FF81000839810008F3
:107B3800FF8100081D810008FF810008FF810008FF
:107B4800FF810008FF810008FF810008FF8100080D
:107B5800FF810008FF810008FF810008FF810008FD
:107B6800FF810008FF810008FF810008FF810008ED
:107B7800BF800008FF81000887800008FF81000897
:107B88003F84000825840008E1840008FF8100087C
:107B98000B840008FF810008E3830008D1830008F4
:107BA80071830008FF81000841830008FF810008F5
:107BB800FF810008A7820008798200083182000846
:107BC80009820008E1810008B7810008FF810008E8
:107BD8009F810008FF810008FF810008FF810008DD
:107BE800FF810008FF810008FF810008FF8100086D
:107BF800FF810008FF810008FF810008FF8100085D
:107C0800FF810008FF810008FF8100087F810008CC
:107C1800FF810008FF810008E9820008FF81000851
:107C2800FF810008FF810008FF810008FF8100082C
:107C3800FF810008FF810008D1820008202D7FF411
:107C4800CBAD0B689C4D591C6A7821601A7023686B
:107C58002A78591C21601A702368AA78591C216057
:107C68001A7029892046FBF772FA23686A79591C29
:107C780021601A702268A9792FE5822D7FF4ACADB6
:107C88000B688E4A8E4D11788B4A581C20601970EB
:107C980011892046FBF75BFA8A4B22681B88FF2B69
:107CA80002F10101A8BFFF2321601370A96881F3C5
:107CB800100189B22046FBF74AFA296801F30F013F
:107CC80089B22046FBF743FA7F4B2268197804E50E
:107CD800012D7FF481AD0B680022591C21601A70B8
:107CE80023685A1C22601D7022682421531C2360BB
:107CF8002B4611702AE5522D7FF46EAD22680021C3
:107D0800EBE43268716891421EBF531C33601178EE
:107D18006E4A08BF1946204626F02AFC2FE56C4B10
:107D28001E78033616F0FF063FF429AD694BDFF8DD
:107D3800C8811E4403F1010A4FF00A0920E0B9F195
:107D4800500F00F09687B9F1320F00F0B287A9F111
:107D58003C00C0B2132840F2B087002529462368AA
:107D68005A1C2260204683F80090FBF7F0F9294658
:107D78002046FBF7ECF956453FF401AD1AF8019B94
:107D8800B9F10A0FDBD1544B9D68196805EB8505DD
:107D98004FF6FF736D009D42A8BF1D469942A8BFCC
:107DA800194625EAE57521EAE171ADB289B2D6E74F
:107DB8000B68DFF84891494E591C022221601A705D
:107DC80023684FF006085A1C226083F80080236855
:107DD8000A22591C21601A70236801255A19226049
:107DE8001D70B9F800102046FBF7B1F9B9F8021078
:107DF8002046FBF7ACF923685A19226083F8008003
:107E080023685022591921601A70236800225919D1
:107E180021601A7031882046FBF799F9718820464D
:107E2800FBF795F92B4691E42D4BBBE40B685A1CE4
:107E38000A601D700B680222591C21601A702268A2
:107E480000214AE41F4B0A681B881D4DFF2BA8BF61
:107E5800FF23511C21601370A96881F3100189B2B6
:107E68002046FBF774F91F4B20461988FBF76FF97A
:107E7800296801F30F0189B220460125FBF767F94C
:107E88002B4663E40B2218492046FBF732F90822F7
:107E980016492046FBF72DF90125072214492046EB
:107EA800FBF727F92B4651E4002A3FF468AC114B45
:107EB800136001252B4649E4943D00201E750020DF
:107EC800CC740020D87400208F3D002019E40208EB
:107ED80001740020403E0308B8250020EC2500204E
:107EE800D83500208C3D0020886B0308946B03086C
:107EF800A06B0308594D0008FC25002028350020F8
:107F0800726835687B623046551BFBF7CBF8052D48
:107F180038627B6A00F2DD878026B346012594E843
:107F28000600521A103A9642C8BF1FFA82FBC34A8B
:107F3800396A92683A61521A9345396A7B622046D7
:107F4800FA6088BF1FFA82FBFBF7EAF87B6A002B0E
:107F580000F09D87002D40F01C872368C7F800D0EB
:107F68005D71C0B00533C7F808D0FB61BBF1000FE5
:107F780001F08E803B6A3A69934281F04F80AA46AD
:107F88003E6A7D627C6080255446FB681C1BAB4BB7
:107F9800B4F5807F28BF4FF480749B6832199A42E9
:107FA80088BF9C1BFBF786FC2246BC6830462146EE
:107FB800FBF700FDF969B86104EB000C0B787B61F5
:107FC800644530D2DFF89C920CF1FF3C04F1FF3E8F
:107FD8001EF8013F09EB830219F823405688FCB1CB
:107FE80000234FF4004204F1FF3816424FEA5202D0
:107FF80002D00878284308706D0806D10AF1010AF2
:108008004D701FFA8AFA01318025D34505D8F44509
:1080180000F26A864345C0F2678601339C42E4D188
:10802800E645D5D1F9617B6ABA6913449BB2D34559
:108038007B6206D97B6A3A6A1C46D6183B699E421F
:10804800A3D37C68802D1CBF0AF101031FFA83FAB1
:108058000AF1020189B22046FBF779F82368796AA8
:1080680001255A19226020461D70FBF770F8236815
:10807800534423602B46D7F800D0FFF767BB704AFC
:108088001068DA1C01462133951E356012F8035C2E
:108098000D70551E356012F8025C4D70326012F892
:1080A800015C8D700332934201F10301ECD124F09D
:1080B800B3FCFFF764BBC2F34705122D00F29B80A7
:1080C800C5B107F1500307F12A0903EB450AC84671
:1080D800AAF1260A3046FAF7FCFF28F8020FC24533
:1080E800F8D1584B39F8022F23F8022FC845F9D197
:1080F800112D09D8544A6B00023B13440021223247
:1081080023F8021F9A42FBD1504A01231D461370DF
:10811800FFF71CBBDFF8508100233046C8F8003059
:10812800FAF7C0FF0125C8F800002B46FFF70EBB81
:108138001A46591C316012F8025B3260DA1C587812
:1081480032609978002D00F0D987012D7FF417ABA4
:108158000BF066FC2B46FFF7F9BA3D4A127812F08D
:10816800010148D15A1C3260187801250BF09AFB9E
:108178002B46FFF7EBBA3046FAF7ABFFDFF8DC80A7
:10818800A8F80E003046FAF7A4FF0125A8F80C005D
:108198002B46FFF7DBBA3046FAF79BFF2D4A00EB78
:1081A80080004300012513802B46FFF7CFBA3046E5
:1081B800FAF78FFFDFF8B480A8F814003046FAF712
:1081C80088FFA8F816003046FAF783FF0125A8F8BB
:1081D80018002B46FFF7BABA1A46591C316012F834
:1081E800020B3260DA1C597832609A7814F000FC7D
:1081F80000287FF4C4AA4FF0FF352B46FFF7A6BA34
:108208001A46591C3160144912F8020B0870326082
:1082180012495A788A70DA1C32600E4A9B78937039
:1082280001252B46FFF792BA054B0D4918684E22D7
:10823800012529F02BFA2B46FFF788BAD80D002024
:1082480080540020A2570020A4570020C8570020BF
:1082580035560020A03B0020146C0020F445002077
:1082680068550308503E0308D83500208067002071
:1082780019465A1C3260BB4A11F8020B1070316063
:1082880059785170D91C31609B7893703046FAF751
:1082980020FFB54B0125D8802B46FFF757BA30464B
:1082A800FAF717FFDFF8C082A8F800003046FAF79F
:1082B80010FFA8F802003046FAF70BFF0125A8F8CE
:1082C80004002B46FFF742BAA84B1B78DB0792D471
:1082D8000125FDF7ABFDFEF7BDFB2B46FFF736BAD0
:1082E8005A1C32601A780F2A85D8991C3160C2EB63
:1082F800C2029F4958788854D81C30600A4499783B
:108308005170191D3160D9789170591D31601979F2
:10831800D170991D316059791171D91D31609979E0
:10832800517103F108013160DB799371012523F064
:10833800C1FF2B46FFF70ABADFF84C9299F80030D4
:10834800002B3FF41CAADFF8448200253046FAF7D8
:10835800C0FE11F09BF899F80030A8EC010A01352D
:108368009D42F3DBFFF70BBA0D2A7FF444AF5A1C8A
:1083780032601D78072D3FF63EAFDFF81492304685
:108388004FF00C08FAF7A5FE08FB05F809EB0805FD
:10839800A8803046FAF79DFEE8803046FAF799FE45
:1083A800336828811A46591C316012F8021BA972D9
:1083B80032605B78EB723046FAF774FE012549F8B3
:1083C80008002B46FFF7C2B93046FAF782FE694B20
:1083D800012518802B46FFF7B9B95A1C3260187866
:1083E800060600F11F86614B1B78DD073FF5C7A91C
:1083F800032828BF00200125FDF7FCFC2B46FFF7CA
:10840800A5B95A4B1B78D8073FF5B9A90125FDF73F
:10841800DDFDFEF71FFB2B46FFF798B9534B1B7882
:10842800D9073FF5ACA9544B4FF4C87201251A80FF
:108438002B46FFF78BB9092A7FF7DDAEDFF85481A9
:108448001A46591CD8F80050316012F8021B2970DE
:1084580032605A78AA70DA1C32609A78642A03F17A
:108468000401A8BF64226A713160DA78642A03F1D2
:108478000501A8BF6422AA7131601A79EA719A1DB0
:1084880032605A79642A03F10701A8BF64222A726C
:1084980031609A79EA7003F108023260DB792B7156
:1084A8003046FAF716FE726833686881D11A0029D7
:1084B8000CDD591CD8F800003160521A002A1978CE
:1084C800417203DD9A1C32605B78437001251AF013
:1084D800B5FE2B46FFF73AB9244B1B78DA073FF570
:1084E8004EA9264A1378012543F0040313702B463E
:1084F800FFF72CB9591C1A463160214912F8020BB2
:10850800887032605B784B7001252B46FFF71EB9E7
:108518000721B2FBF1F1C1EBC105521B7FF46BAE31
:10852800C9B201F1FF395FFA89F900293FF427A997
:10853800DFF850A009F1010915465A1C326093F979
:108548000010104B4FF0000893F902208A4203F103
:10855800080300F0E08408F10108B8F1060FF3D130
:1085680049E600BF8C3400200C3800203556002026
:108578009870002088340020E87800204C390020CA
:10858800EC7800206462002001740020103700207D
:1085980030730020005600205A1C32601A780E2AC8
:1085A8003FF629AE991C31605D78032D3FF623AE66
:1085B800A848062101FB02F1421803F1030E557188
:1085C800C6F800E09D784554191D3160D97851707E
:1085D800591D316019799170991D31605979D1709F
:1085E800D91D31609B79137101252B46FFF7AEB871
:1085F8005A1C3260984A1B78537501252B46FFF7A1
:10860800A5B83046FAF765FDDFF86C82C8F80000B7
:108618003046FAF75EFDC8F804003046FAF759FD0F
:108628000125C8F808002B46FFF790B8DFF84C8200
:108638000023C8F800303046FAF734FDD8F8003087
:1086480001250343C8F800302B46FFF77FB85A1CB2
:1086580032601D78132D3FF6CEAD9A1C32605878E3
:108668007B6225F0BFFF00283FF4C5AD7B6A7B4ADB
:10867800017802F82510D91C316002EB850299783F
:108688005170191D3160D8789070581D3060744948
:108698001B79D370086801251AF05EFD2B46FFF799
:1086A80055B87049102A13464FF0000228BF10230E
:1086B8000A604A608A60CA600A74002B3FF45FA8A7
:1086C8003268013913440132326012F8010C01F8A2
:1086D800010F9A42F7D1FFF752B8591C31601D7843
:1086E8001F2D3FF688AD052A7FF485AD3046FAF791
:1086F800D9FC5D4B43F8250014F0ECF9FFF73FB8BF
:10870800594D05F140083046FAF7E3FC3368A5F8FF
:108718008000591C1A46316012F8021B85F8821035
:1087280032605B7885F883300435A845EBD1FFF7D4
:1087380026B85A1C3260484D1B782B723046FAF71F
:10874800C8FCA8833046FAF7C4FC28833046FAF7F9
:10875800C0FC32686883531C33601278EA7472680C
:10876800D31A032B00F374843368D11A05290EDD5C
:108778005A1C32601B78EB723046FAF793FC336868
:10878800E8605A1C32601B782B7433687268D21AFE
:10879800002A7EF7F4AF5A1C32601B7885F8213026
:1087A80001252B46FEF7D2BF581C30602F4A1D7892
:1087B8001570091A00297EF7E2AF991C31605B78C1
:1087C800003318BF0123012553702B46FEF7BEBFA7
:1087D8001A46591C3160DFF8A88012F8021B88F885
:1087E8000210326022495A780A70DA1C3260214D30
:1087F8009A782A711A1D3260DB78092BA8BF0923E1
:108808003046AB70FAF765FC336872682880D11A75
:10881800012905DD3046FAF75CFC33687268688226
:108828009A4207D05A1C32601B78003318BF0123C4
:1088380088F80730FDF704FB336872689A423EF403
:108848009EAF5A1C32601B78EB7001252B46FEF751
:108858007DBF00BFE4350020AC6D0020343B002014
:108868008054002030380020883C0020303B002015
:108878004872002080670020FC320020505B0020F6
:10888800146C00203046FAF724FC054619F07EF8EF
:10889800FF283EF474AF3F2D00F2FF8307F1500824
:1088A800002308F8243D4FEAD509414607F12B007B
:1088B80087F82B3009F1010919F048F897F82B309F
:1088C8005FFA89F905F007054B4505F1010503D164
:1088D80097F82C30AB4203D02946484619F042F8A5
:1088E80033687268D21A012A7EF749AF5A1C07F119
:1088F8005000326000221D7800F8252D19F01AF872
:1089080097F82B30AB420AD0C44B1B683BB19A791D
:10891800AA4204D31B681B690BB1284698473368E1
:108928005A1C3260404600221D7887F82C2018F027
:10893800F5FF97F82C30AB423EF421AFB74B1B68DC
:10894800002B3EF41CAF1B685B69002B3EF417AF8D
:1089580028469847FEF713BFB14A1278012A3EF617
:108968000EAF18465A1C3260DFF8E08210F8022B6E
:1089780088F80220DA1C891A306001295878326098
:1089880040F3A1833046FAF7A4FB0125A8F80000BC
:108998002B46FEF7DBBE5A1C326093F80080B8F114
:1089A800110F3FF628AC9A1C32609E4D5B7805F893
:1089B80018303046FAF78DFB40F6CA039842A8BF34
:1089C800184640F2EE23984205EB4801B8BF184616
:1089D8000125A0F2EE222B46192092FBF0F24A70F4
:1089E800FEF7B4BE3046FAF774FB3046FAF771FB6F
:1089F8003046FAF76EFB3046FAF776FB33688A4D55
:108A08001946581C2A68306011F8020B82F82C00AD
:108A18003160597882F83610D91C31609B7882F819
:108A280037303046FAF760FB3046FAF75DFB3046E0
:108A3800FAF75AFB3046D5F80080FAF74AFBA8F84F
:108A48003A003046D5F80080FAF743FB336872687D
:108A5800A8F83800D11A01290ADD591C2A683160A2
:108A68001B7882F82E303046FAF73EFB336872687E
:108A7800D31A032B0BDD3046D5F80080FAF729FB13
:108A8800A8F8320030462E68FAF723FBB08628682B
:108A9800FFF70DBB5A1C3260634DDFF8B4811B78B9
:108AA80088F805303046D5F80090FAF712FBA9F897
:108AB80020003046D5F80090FAF70BFB726833684F
:108AC800A9F81E00D11A072919DD3046FAF701FB6B
:108AD800A8F80A003046FAF7FCFAA8F80C00304665
:108AE800D5F80090FAF7F5FAA9F822003046D5F83B
:108AF8000090FAF7EEFA33687268A9F82400D11AE0
:108B080003290BDD3046FAF7E4FAA8F80E003046E0
:108B1800FAF7DFFA33687268A8F81000D21A002A48
:108B280005DD591C2A6831601B7882F82630FDF76C
:108B380087F921F0EFF93D4B1B68002B00F07D828F
:108B48002868012523F04AFC2B46FEF7FFBD1A468C
:108B5800591C3160364912F8020BC8703260354929
:108B68005A784A71DA1C3260334A9B78D3700125EF
:108B78002B46FEF7EBBD1A46591C304D316012F8F2
:108B8800021B297132605B786B713046FAF7A1FAE3
:108B9800336828805A1C32601B78AB713046FAF76C
:108BA80098FA336868805A1C32601B78EB7101258B
:108BB8002B46FEF7CBBD0125FAF7DEFE2B46FEF766
:108BC800C5BD5A1C32601E4A1B78DFF888801370B6
:108BD8000023C8F800303046FAF764FA3368D8F84A
:108BE80000201849184D10435A1CC8F8000032607C
:108BF8001B780B723046FAF76CFA28603046FAF7A1
:108C080068FA68603046FAF764FAA8603046FAF7FE
:108C180060FA3046FAF75DFAFEF7B1BD3855002024
:108C2800335B0020CC59002080540020143B0020E6
:108C3800F44500202C400020A03B002028380020CC
:108C4800303B0020AC6D0020FC320020365B002059
:108C5800146C0020505B0020C64A03F10801013360
:108C6800336013F8010C02F8010F8B42F7D1FEF7BD
:108C780086BDC14BFFF788B83388FF2BA8BFFF23F9
:108C8800DBB2FEF7FABC24F051FB00283EF4F4AC4A
:108C980003780A2B2FD8B0F9023088FB0312DB17B0
:108CA800C3EBA2039BB2FF2BA8BFFF23DBB2FEF7E7
:108CB800E4BC98E82200FFF769B824F037FB0028E5
:108CC8003FF44BA803780A2B3FF647A8B0F90430C5
:108CD800B0F9061003EB830383F3500521EAE17131
:108CE800ADB289B2FFF73BB8FB697C681A463B7D99
:108CF8001370FFF7A7B90023D8E71A46591C31604B
:108D08009E4D12F8021B697032605A782A70DA1C7C
:108D180032609B78AB703046FAF7DBF9336828810C
:108D2800591C1A46316012F8021B697132605B786F
:108D3800AB7101252B46FEF709BD5A1C32601A7823
:108D48000A2A00F0D9803046FAF7CEF93046FAF709
:108D5800CBF901253046FAF7C7F92B46FEF7F6BCE2
:108D68005A1C32601B780A2B00F0C080502B7FF40D
:108D78004DAF3046FAF7ADF9DFF81C82A8F80000CD
:108D88003046FAF7A6F90125A8F802002B46FEF7A7
:108D9800DDBC7B4B3A6A9B68D4F800905A449A42EF
:108DA80000F22981FAF786FD5A464946386AFAF7E9
:108DB80001FE23680344236086427EF7E0AC00216D
:108DC80000E0236801305A1C864222601970F8D1ED
:108DD800FEF7D5BC336872689A4240F0E380694B6D
:108DE800FF22DA704FF0000A674D09F0DFFD5146A7
:108DF8003022664885F800A02AF0C7FE87F82CA024
:108E080097F82C300B2B00F20781DFF890915F4E1A
:108E1800524697F82C3003EB430309EBC3035B7C02
:108E2800E3B197F82C3003EB430309EBC30320218C
:108E38005B699BB197F82C3003EB430309EBC30341
:108E4800586946F82200F9F7D2FA2B7856F8230029
:108E5800F9F78EFC2A780132D2B22A7097F82C30B2
:108E68000133DBB287F82C3097F82C300B2BD0D994
:108E78002368591C21601A70B8F1000F3EF47FACCA
:108E8800434BC8F8003001252B46FEF75FBC002D88
:108E98007FF47FAF59462046FAF759F923685A1CE0
:108EA80022601D70364B26689D683B6A0BEB0302F7
:108EB800AA4240F215813B6AED1AFAF7FBFC2A46F2
:108EC8003146386AFAF776FD236803442360FEF7D3
:108ED80056BC3046FAF7FDF8326871687B6A9142F1
:108EE80083463DD106461D46FFF719B83046FAF7C6
:108EF800F0F8DFF8AC8041E79A1C3260254A5978CF
:108F08001170D91C316099785170191D3160DB7866
:108F18009370FEF734BC0AEBC80B30468BF802108E
:108F2800FAF7D7F832682AF838001346511C31602E
:108F380013F8021B8BF80310336053788BF8043056
:108F4800D31C336093788BF80630131D33600135DA
:108F5800D2788BF805204D457FF4EFAAFEF70FBCB9
:108F6800511C316012781D46131C064618BF012398
:108F7800FEF7D5BFAB6D0020F0250020943D002002
:108F8800D80D0020FC1E0020776F0020E858002034
:108F9800FDBB0208055A0020EC2500206066002071
:108FA800283500205A1C19463260574811F8022B00
:108FB800C27031605B780371042A03D9FF2A7EF4FA
:108FC8009DAE0FE751490978994205D8022A7EF4E7
:108FD80095AEFF2B7EF492AE236801255A192260C4
:108FE8001D70B8F1000F3EF4CAAB494BC8F8003009
:108FF8002B46FEF7ABBB3A6AA3EB0208FAF75AFC1A
:1090080042464946386AFAF7D5FC23680344236088
:10901800002D3EF4B4ABCFE6524629E77D62AA465E
:10902800FFF716B800F07F00032828BF00200125AD
:109038000AF012FD2B46FEF789BB36483649374AF7
:10904800374B036001250B6013602B46FEF77EBB90
:109058003046FAF73EF8A8843046FAF73AF833680B
:109068007268E884D11A03297FF77FAB1A46591C26
:10907800316012F8021BA97732605B7885F82030DE
:109088003046FAF726F8336872686884FFF76DBBD4
:10909800DA46C7F824B0FEF7DBBF07F12C084046D4
:1090A80018F030FCBB8DAB423FF41AAC1D4B1B686B
:1090B800002B3FF415AC1B689B69002B3FF410ACE8
:1090C800284698470CE4184A99781288012512FB1B
:1090D80000F22B4692FBF1F2A8F80020FEF736BB0F
:1090E800FAF7E8FB5A463146386AFAF763FC236810
:1090F8000125034423602B46FEF728BB012523F0F6
:1091080003FB2B46FEF722BBFC1E00200174002047
:10911800714D000888710020DC7100204472002025
:10912800E3060008385500205A3900202DE9F04F91
:109138002DED028B93B0834613F0B2F9AD4B1D7839
:1091480025B113B0BDEC028BBDE8F08FAA4B1B68AC
:109158005E05F6D5A94FAA4E3B68002B5BD0A94CFB
:109168003168D4F810218A1A7C2A54D994F8142129
:10917800DFF8E0829FEDA48AC4F81011013284F868
:1091880014214FF0240A5E20984750463B689847C0
:109198009E4BF8EC016A9B8A07EE103AF8EEE66AF5
:1091A800B8EEC77A0AF1010AC6EE877A5FFA8AFA38
:1091B80067EE887AFDEEE77ACDED027ABDF9089080
:1091C8005FFA89F024F04AFCC9F3072024F046FC32
:1091D800BAF1270F3B68D6D15E2098473B6830200C
:1091E8009847D4F818815FFA88F024F037FCC8F360
:1091F800072024F033FC3B685E20984794F814312C
:1092080013F0030800F06E8113F0070801F03A82AA
:10921800282B01F0F0827E4B1B78002B6BD0794C09
:109228007C4AD4F82031ABEB0303934200F26D87FC
:1092380094F8285195BB784F3868F8F7A8FAC0B267
:1092480001280FD9022841F06F83744B1A78002A3D
:1092580041F09E85D4F82C21ABEB0202B2F57A6F6F
:1092680081F05986D4F83031002B44D094F8283155
:10927800BBB96B4B1B689B7801211E3B00228B42BC
:1092880084F8281184F83C2141F20E8638680221BE
:10929800043024F059FB94F8343110E0D4F830311C
:1092A8004BB3D4F8383140F6B732ABEB03039342F3
:1092B80021D994F83431002B01F08782564F013BB5
:1092C800DBB284F83431002B00F07887D4F83051C1
:1092D80094F83C2115F8011B94F83D313868C4F81E
:1092E80030510A44013384F83C2184F83D31F8F7C1
:1092F80051FAC4F838B14B4B35681B7843B14A4F23
:10930800386828B1494B1B78013B012B40F265872F
:10931800474B1B7863B1474D2B684BB1394CD6F896
:1093280000A0D4F85431AAEB0303632B00F25A8649
:10933800414B1B7873B1414D2B685BB1314CFDF744
:109348006FFED4F85C31029044F61F62C31A934250
:1093580000F214813A4B1B78002B7DD1394B1B78D6
:1093680043B1284CD4F8AC3203F5C333A0339B4542
:1093780080F08C86344B1B78002B3FF4E2AE214EF4
:10938800324C334D06F2CD272068F8F700FA002852
:109398003FF4D7AE2068F8F7F4F92B7880465A1EC8
:1093A80033B120682A70F8F7F2F90028F2D1C8E63C
:1093B80003223946781E2AF0CEFB96F8CC3296F86E
:1093C800CD2286F8CF8283F47F4383F0FF039B1A74
:1093D8001FFA88F89BB2B8EB132FD5D196F8CE2296
:1093E800DBB29A42D0D1781E24F018F82B781844B2
:1093F8002870C9E76F540020386C0020E4760020FC
:1094080068570020081F002000007A44AC54002050
:109418009A3E00203F0D0300DC7600202900002042
:10942800E07600209C3E0020C4740020A43E00206A
:10943800AC3E0020584F0020B43E0020B83E00202B
:10944800F83E0020093F0020BE3E0020C43E002018
:10945800C83E0020E45400203C4C2278A2B13C4B8A
:109468009B7A53B1FDF7DCFD3A4B1B68C31AA3F591
:109478007A73B3F5FA6F07D82278374B37491868EB
:10948800F8F75CF900232370354CD4F8A43203F5BF
:10949800C333A0339B45FFF461AF324DC4F8A4B287
:1094A8002B78002B41F0F8822F4D2B78002B41F0C0
:1094B800F1812E4994F8A8228D5CE90701F1AA846C
:1094C800AA0701F16A846B0701F16183284A94F8BD
:1094D800A8321178013393FBF1F201FB123384F8BF
:1094E800A8323BE7D4F8102141F288339A4201F2BE
:1094F800E6813B685E2098473B68142098471D4BDF
:109508001D4AB3F9043082FB03124FEAE378C8EB33
:10951800A2080FFA88F85FFA88F024F09FFAC8F3D7
:10952800072024F09BFA3B685E2098473B681C2084
:109538009847002024F092FA002024F08FFA3B6824
:109548005E20984794F814315EE600BF8C3E0020F8
:10955800AC6D002094580020FC3E00204C3E0020BA
:10956800081F0020003F0020013F0020043F00208A
:10957800083F0020045500206766666694F862314B
:10958800002B41F07681DB4B1A6802F00803002BB0
:1095980048F603414AF60B404BF60F4349F6074796
:1095A80004BF03460F4612F0040F4FF0190118BF0D
:1095B8001F46920684F8621103D547F4804747F0A6
:1095C8002007CD4B5A79C7F30909002A41F0F084E6
:1095D8009B79002B41F04D85984664204FF0FF3A67
:1095E8004FF0000C0A970B97ADF834C0CDF83AC08D
:1095F800CDF83EC0CDF842C0CDF83090ADF83680F9
:10960800ADF838A08DF846000AAF0FCFDFF800E3B9
:1096180084F805C0AEE80F0097E80F00AEE8070031
:109628002EF8023B71464FF0010C1B0CFE271F2041
:10963800C82201F81E39A770A27184F807C0E0702B
:1096480094F87201207180F0F10383EA0313DAB20F
:10965800130983F0E70343EA022383EAC2031BB238
:1096680083EA0312D2B2C3F3072383EA121343EA4D
:10967800022383EAC2031BB283F0C80282EA021201
:10968800D2B2C3F3072383EA121343EA022383EA1D
:10969800C2031BB283EA0C0787EA0717FFB2C3F3BA
:1096A800072282EA171242EA072200EB0C0382EA39
:1096B800C7070EEB0C0084F87231278011F8013BC4
:1096C8007B4083EA0313DBB21A0982EA172242EAD3
:1096D800032282EAC3031BB29FB281422780EDD1E5
:1096E80083F07C0383EA0313DBB24FEA131E8EEA8E
:1096F800172E8EEA032E8EEAC30E0FFA8EFE1FFA7D
:109708008EFADFF810C2A4F800A05FFA8EFE4FEAC6
:109718001A2A84F828A084F827E00CF5CD7804F1FB
:109728002209DCF80000DCF80410DCF80820DCF87A
:109738000C3047460FC70CF1100CCC45B846F0D199
:10974800DCF8000038606D4F9CF8043088F804306D
:1097580007F1270884F8C1E184F8C2A117F8011FAE
:109768002868F8F717F8B845F8D194F86331002B52
:1097780041F07A806249326809780A2084F86301E6
:10978800002901F0FA815F4F01293888069041F2DB
:1097980060840229B7F802E001F02284B8880590B5
:1097A800032901F06D84F8880490042901F0748479
:1097B8000529388901F06B840629B7F80A9001F069
:1097C80054840729B7F80C8001F04C84FB89039373
:1097D80094F872110A920B4683F0300282EA021260
:1097E800D2B217094849079387F07A0747EA022750
:1097F8000988237187EAC202444FC1EB012187FB24
:10980800013A069B4FF0000C63F30F0C059B6EF3B7
:109818001F4C4FF0000E63F30F0E049BCDF82CC0C5
:1098280012B28A440027C91763F31F4EC1EB6A2A94
:10983800039BCDF830E082EA021160F30F070020A5
:10984800C9B268F30F00C2F3072269F31F4782EA1F
:10985800111263F31F404FF000090D978DF83DA0DA
:109868000E908DF83C9042EA01220DF1280C82EA14
:10987800C107BCE80F003FB287F0C80888EA08189B
:10988800DFF88CE084F805905FFA88F8C7F30727BB
:10989800AEE80F0087EA181747EA08239CE8030098
:1098A80083EAC8031BB283F023024EF8040B82EA52
:1098B8000212D2B2C3F30723079F83EA121370463A
:1098C80043EA022383EAC20207F1010C20F81419C3
:1098D8004FF023081621FE27C82384F872C122807E
:1098E80084F807800EF1020EA770E170A37111468B
:1098F80012E000BFA8540020943D0020A3200020BF
:109908002C5500204C5300208C3D0020030820805B
:10991800101F00200A1F002010F8013B4B4083EA6B
:109928000313DBB21A0982EA112242EA032282EA0D
:10993800C3031BB299B270452180EDD183F0F403C3
:1099480083EA0313DBB24FEA131E8EEA112E8EEA66
:10995800032E8EEAC30E0FFA8EFE1FFA8EF8E44F1E
:10996800A4F800804FEA182C5FFA8EFE84F81EE0F7
:1099780084F81FC07968BA683868FB6807F5CD783D
:10998800A8E80F0038697969BA6904F29B17A8E852
:10999800070004F2B91884F8B9C184F8B8E117F8D7
:1099A800011F2868F7F7F6FEB845F8D194F86AC1A0
:1099B800BCF1000F40F06887CE4B94F87271B3F990
:1099C8000010B3F90220B3F904309FEDCB6ADFF839
:1099D80044E384F805C007EE103A33680A9387F029
:1099E8006A0383EA031306EE901AD9B20B0983F0CF
:1099F800D50343EA012383EAC1031BB283EA0311B7
:109A08005242C9B207EE902AC3F3072383EA11131F
:109A180043EA0123F8EEE77AF8EEE66AB8EEC77A89
:109A280083EAC1031BB267EE867A66EE866A27EE82
:109A3800067A002083F0C808CDED0C7ACDED0B6ACC
:109A48008DED0D7A0E900F90109088EA08160DF1A2
:109A58002809F6B2C3F30728B9E80F0088EA1618F0
:109A680048EA062888EAC6080FFA88F8AEE80F0020
:109A780088F01E0699E8070086EA0616F6B2C8F3CB
:109A8800072383EA161343EA06238EE8070083EACE
:109A9800C6061C20C8214FF005084FF01E0CFE23F7
:109AA8007A1CE070A17184F86A8184F807C0A370F9
:109AB800AEF1100127710EF10C00268084F8722196
:109AC80011F8013B734083EA0313DBB21A0982EAF7
:109AD800162242EA032282EAC3031BB29EB28142E3
:109AE8002680EDD183F0270383EA0313DBB24FEA24
:109AF800131E8EEA162E8EEA032E8EEAC30E0FFA76
:109B08008EFE1FFA8EFC7A4FA4F800C05FFA8EFE14
:109B18004FEA1C2C84F825C084F824E007F5CD789A
:109B280004F1220938687968BA68FB6846460FC6A6
:109B380010374F45B046F5D1704E3B88A8F8003035
:109B480006F1240784F8BEE184F8BFC116F8011FA6
:109B58002868F7F71FFEB742F8D194F86BA1BAF15D
:109B6800000F40F08B86664B1B68052213F0140F1C
:109B780084F86B2140F0DF86DFED627A94F872C1D9
:109B88005C4B614AB3F90410B2F906205F4E604895
:109B9800CDED0C7A8CF0220383EA0313DFB23B0984
:109BA80083F0590343EA072383EAC703B2F5FA6F40
:109BB8001BB2A8BF4FF4FA6283EA0317FFB2B2F5EB
:109BC8007A7FC3F3072383EA1713B8BF4FF47A7277
:109BD8004FF0640E43EA0723A2F57A720EFB02F2F5
:109BE80083EAC70386FB02E680FB01E01FB2D217B7
:109BF800C9174FF00008C2EBA612C1EBA00187F00D
:109C0800C806ADF83A20ADF83810CDF82880CDF860
:109C18002C80CDF834800DF1280E86EA0616BEE8B1
:109C28000F00F6B2C7F3072787EA161747EA062791
:109C380087EAC606374FDEF800E084F804C00FC78D
:109C480036B286F04A0383EA0313DBB2C6F3072170
:109C580081EA13113A4641EA03210CF1010C81EA29
:109C6800C303142042F810E9FE264FF04A0E0021E3
:109C780084F872C14FF0C80CE0702380043784F870
:109C880007E0A670617184F806C0184612F8011B37
:109C9800414081EA0111C9B20B0983EA102343EA62
:109CA800012383EAC10109B288B2BA422080EDD10A
:109CB80081F0140181EA0111C9B24FEA111E8EEA3E
:109CC800102E8EEA012E8EEAC10E0FFA8EFE1FFAB2
:109CD8008EF6074F26804FEA16295FFA8EFE84F823
:109CE8001D9084F81CE079683868BA68FB6813E04E
:109CF8000A1F00200455002088C3E43AA32000204E
:109D0800A8540020000000004C530020D34D6210DE
:109D180067666666101F0020B7F8188007F5CD7CC7
:109D2800ACE80F0038697969ACE8030004F29B16C7
:109D3800ACF8008084F8B791B04684F8B6E104F234
:109D4800B71918F8011F2868F7F724FDC145F8D19D
:109D5800C54BC64A1B781278013B12F00100DBB2F2
:109D680014BFC0214021172B03D8C14A134493F8CC
:109D780024A0C04B1A8893071ABF002341F0100192
:109D8800012312F4027F18BF022312F0100F18BF2C
:109D9800062312F0200F18BF1023002841F0B180CD
:109DA8004FF0030C94F872910A9389F0460383EA02
:109DB8000313DAB2130983F0920343EA022383EA16
:109DC800C2031BB283EA0310C0B2C3F3072282EABC
:109DD800101242EA002282EAC00212B282F0C80ED1
:109DE8008EEA0E1E5FFA8EFEC2F30722002382EA75
:109DF8001E1203208DF82CA08DF82FC08DF82D3061
:109E080042EA0E2C8DF82E108DF830000AAA07CAE7
:109E18008CEACE0E0FFA8EFEDFF864A2E3718EEAAA
:109E28000E1CAAE803005FFA8CFCCEF3072E8EEA1C
:109E38001C1E4EEA0C2181EACC0C94F808E08AF842
:109E480000200FFA8CFC8EEA0C0E8EEA0E1E5FFACA
:109E58008EFECCF3072282EA1E1242EA0E22607AB4
:109E6800A17A94F80BC0637182EACE0212B2504014
:109E780080EA001E5FFA8EFEC2F3072080EA1E10F9
:109E880040EA0E2080EACE0000B2414081EA01118A
:109E9800C9B2C0F3072282EA111242EA012282EA19
:109EA800C10212B28CEA020C8CEA0C1C5FFA8CFC20
:109EB800C2F3072282EA1C1242EA0C2294F80CE050
:109EC800607BA17B94F8108084F8049082EACC022D
:109ED80012B28EEA020E8EEA0E1E5FFA8EFEC2F3F0
:109EE800072282EA1E1242EA0E2282EACE0212B249
:109EF800504080EA0010C0B2C2F3072282EA101272
:109F080042EA002282EAC00212B2514081EA0111FB
:109F1800C9B2C2F3072282EA111242EA012282EA96
:109F2800C102E17B13B281EA030282EA0212D2B2D1
:109F3800C3F3072383EA121343EA022383EAC20323
:109F48001BB288EA030282EA0212D2B2C3F30723E1
:109F580083EA121343EA022383EAC2031BB283F0A3
:109F6800320282EA0212D2B2C3F3072383EA12133F
:109F780043EA022383EAC2031BB29AB24FF0FE0CF3
:109F88004FF0090EC82009F10101DBB284F802C0C4
:109F980084F803E04FEA122CA07184F87211228031
:109FA80084F812C0637438687968BA68B7F80C9096
:109FB8000AF5C67EAEE807000AF5CE7A8EF802806A
:109FC800AEF8009084F8ACC184F8AB3116F8011FE4
:109FD8002868F7F7DFFBB245F8D1029BC4F85C317B
:109FE800FFF7B8B9DFF89C90234FDFF89C80412039
:109FF80023F058FCB9F9023087FB0320DB17C3EBC9
:10A00800A00080B223F034FCB9F9003087FB0320AC
:10A01800DB17C3EBA00080B223F02AFCB9F90430A7
:10A0280087FB0320DB17C3EBA00080B223F020FCE2
:10A0380098F800102868F7F7ADFB94F8583113F03A
:10A04800010700F09D840D4AC4F854A10133DBB226
:10A05800A2FB0312D20802EB8202A3EB420384F8AC
:10A068005831FFF765B900BF303B00203556002056
:10A0780054420308FC3D002067666666CDCCCCCC14
:10A08800101F0020045500205254002094F8B032CC
:10A09800BC4AC4F8ACB202EB8302D26B42B312AD35
:10A0A80004F2B723B84E45F8203D002104F2C92335
:10A0B80031800B9380211523A52784F8B6322846D2
:10A0C80084F8B51284F8B472904728463188F9F7B5
:10A0D8003EF80A9DAD4804F52D716D1A152DA8BFDF
:10A0E80015252A4627F0D2FAA94A94F8B0321570F5
:10A0F800A84A013382FB0312A2EBE37202EB42028D
:10A108009B1A84F8B032FFF735B9A34BA34AD4F8A9
:10A11800241130681288DF7AA14B401A4FF47A7103
:10A12800D5B201FB07F1120A9D771D7588424FF0E1
:10A138000005DA775A759D701D7180F0B283994ACF
:10A148009949DFF874E212680D688868974FC4F877
:10A1580020B18EFB02C1D217C2EB6112D4F81811DC
:10A168008EFB01CE87FB058C87FB0087C017C0EBF1
:10A17800A70002F5FA72CF1792B2C7EB6E1EED1761
:10A1880001F5EA47C5EBAC0530379A76120A0EF1AD
:10A19800780E3F123031DA764FEA252C02121D77FD
:10A1A80083F81DC083F8200083F8212083F824E079
:10A1B80083F8237083F82210FFF73AB894F83C111B
:10A1C80094F83D3138684A1C013384F83C2184F8FE
:10A1D8003D31F7F7DFFAFFF78CB8754CDFF8DC8113
:10A1E8004FF0010A4FF0000908E01B2B00F0E48251
:10A1F8000D2B00F0118288F801A03868F7F7C7FA2C
:10A20800002838D03868F7F7BCFA83B27E2B32685A
:10A218002AD098F801100029EFD194F83E21002A9D
:10A22800E3D07D2B00F0098294F84CE1BEF1000FD9
:10A2380004D080F02003DBB284F84C11511CC9B261
:10A248002244092984F83E1182F8403100F0EB815C
:10A258000829D2D8B4F84A21134403EB132303F096
:10A26800FF03A4F84A31C8E784F83E9184F83F9187
:10A2780088F80190C1E794F84D3133B194F8413131
:10A2880084F84D01302B00F0308694F83F213D4B87
:10A29800DFF82CC1DFF800A1DFF828E1DFF828910A
:10A2A8000127002A3FF434A83168491B012900F22C
:10A2B800AE8194F84E81B8F1000F40F0918294F885
:10A2C8004F1133F8110010B984F84F71E9E70131E3
:10A2D800B0F5826F84F84F1100F002811ED9B0F5F5
:10A2E800E26F00F0C08034D9B0F5046F00F0C98087
:10A2F800B0F5116F00F04781B0F5E46FD1D12D4A68
:10A30800156C918A642303FB05F393FBF1F123F0A9
:10A3180001FB002384F83F31FEF7FABFB0F5007F58
:10A3280000F0BB8052D8B0F5807F00F04681B0F5D0
:10A33800887FB6D1DCF800104907B2D5D4F81811D7
:10A348004FF4887023F0E6FA002384F83F31FEF7D3
:10A35800DFBFB0F5C06F00F0B380B0F5E06FA0D1FB
:10A36800144A906B918A642303FB00F34FF4E06076
:10A3780093FBF1F123F0CEFA002384F83F31FEF786
:10A38800C7BF00BF54420308083E00200C4100200C
:10A39800214100205655555510750020D8740020CD
:10A3A800CC3E0020B8340020CC7400206766666676
:10A3B800081F0020AC5400201F85EB512900002005
:10A3C800A8540020943D00201E750020B0F5047F9D
:10A3D80000F00381B0F5806F7FF463AF94F85031DB
:10A3E8000133DBB2032B00F22D8142F2107184F8A5
:10A3F800503101FB03F1964B1B88002B40F0208164
:10A408000131944B1B78DF07934B1B8848BF0431FD
:10A41800DD0748BF0A31980748BF14311A0648BFFC
:10A428002831DF0548BF28315D0748BF6431180768
:10A4380048BFC8319A0548BF01F5C8719F0648BF93
:10A4480001F57A71DD0648BF01F5FA61580648BF83
:10A4580001F57A614FF4806023F05CFA002384F8F8
:10A468003F31FEF755BF7D4AD56B918A642303FBC4
:10A4780005F393FBF1F123F04DFA84F83F81FEF7E1
:10A4880047BF774BB3F9041001EB8101490023F072
:10A4980041FA84F83F81FEF73BBF9EF80610002979
:10A4A8003FF4FFAE6F4B70491B6881FB0321DB173C
:10A4B800C3EBA10123F02EFA84F83F81FEF728BFF1
:10A4C8009EF8061000293FF4ECAE664B4FF4C060CE
:10A4D800996823F01FFA002384F83F31FEF718BF6C
:10A4E800DCF8001011F020087FF4DBAE5F49086843
:10A4F800010600F1E1849AF80C1000293FF4D1AE6E
:10A5080094F85111032900F27885DFE801F0322828
:10A518001902574B1B6859799A79DB7901F1407117
:10A5280001EB022101EB0341002384F851314FF480
:10A53800826023F0EFF9002384F83F31FEF7E8BE8C
:10A548004C4B1A68137A507992781B0403EB00235A
:10A5580013444A1C84F8512103EB0161E7E7454B9A
:10A568001A68D379107952781B0403EB002313443B
:10A57800EFE7404B1A689379D07812781B0403EB05
:10A5880000231344E5E79EF8051000293FF489AE3F
:10A5980099F8001000293FF484AE374B1B8803EB71
:10A5A80083035B004FF4116093FBF1F123F0B2F9E0
:10A5B800002384F83F31FEF7ABBEDCF800104807F3
:10A5C8007FF56FAE2D4B4FF48070196823F0A2F918
:10A5D800002384F83F31FEF79BBE9EF80510002942
:10A5E8003FF45FAE99F8000000283FF45AAE244BC0
:10A5F8005B7B002B00F081841F4B198891FBF0F1E5
:10A6080001EB810149004FF4047023F083F9002322
:10A6180084F83F31FEF77CBE84F83EA184F84031CF
:10A62800A4F84A21E9E5B4F84A21C2F1FF029342AD
:10A638007FF4E1AD84F84DA1DDE584F84CA1DCE5BB
:10A648000231DEE6012384F8503142F21071D2E67D
:10A65800C83D002035560020FC3D0020AC540020A9
:10A6680004550020CC74002067666666386C0020AC
:10A678000056002080540020D8740020B8340020F0
:10A68800107500203B685E2098473B680220984779
:10A69800FF2022F04BFE0378FF2B00F0238490F973
:10A6A80001304FEAE3785FFA88F8D8B223F0D6F998
:10A6B800404623F0D3F93B685E2098473B68032067
:10A6C8009847FF2022F032FE0378FF2B1DBFB0F918
:10A6D8000830DDB2C3F307284FF0000828469B4D29
:10A6E80023F0BCF9404623F0B9F96B79002B40F010
:10A6F800A1820AA9964823F075F93B685E2098471D
:10A708003B6813209847BDF92850E8B223F0A6F912
:10A71800C5F3072023F0A2F93B685E2098473B6801
:10A728001B209847BDF92A50E8B223F097F9C5F3E2
:10A73800072023F093F93B685E2098473B68232065
:10A7480098474E2023F08AF9002023F087F90AA9B8
:10A758007F4823F047F93B685E2098473B68122002
:10A768009847BDF92850E8B223F078F9C5F30720D7
:10A7780023F074F93B685E2098473B681A20984795
:10A78800BDF92A50E8B223F069F9C5F3072023F090
:10A7980065F93B685E2098473B682220984745202A
:10A7A80023F05CF9002023F059F93B685E209847B4
:10A7B80094F81431FEF72CBD3868F6F7E8FF002846
:10A7C8007FF419AD84F83FA117E5C4F8303184F857
:10A7D8002831604F23F0ECF894F83431FEF76FBD60
:10A7E8005D49062022F0A0FE002384F84E0184F87B
:10A7F8003F31FEF78DBD00253B68D6F8008084F810
:10A8080014515E2098473B68544C172098472846B7
:10A8180023F024F9524BA3FB08239B0BA4FB031240
:10A828005209C2EB0212A3EB8203D8B223F016F945
:10A838003B685E2098473B6818209847494BA3FB24
:10A8480008239B09A4FB03125209C2EB0212A3EBD3
:10A858008203D8B223F002F9284623F0FFF83B68B8
:10A868005E209847FEF7D7BC013B84F86331FFF7B9
:10A878009DB8013B84F86231FEF777BF0AF1FF3AD1
:10A8880084F86BA1FFF7A9BB0CF1FF3C84F86AC1FF
:10A89800FFF763B934493A2022F046FE2870FEF7E4
:10A8A8005DBD324A31681278C4F82411013A012A90
:10A8B8003FF645AC1021022299701A713FE43B68BB
:10A8C800DFF8B0A0DFF8B4905E2098473B6810200E
:10A8D8009847DAF8003089FB0312DB17C3EB6213E1
:10A8E800D8B2029323F0BAF8029BC3F3072023F0EF
:10A8F800B5F83B685E2098473B6821209847DAF80E
:10A90800003089FB0329D8176422C0EB691002FBC9
:10A9180010300028B8BF4042C0B223F09FF840462C
:10A9280023F09CF8FEF7E5BD23F032F8104B012226
:10A938001A70FEF797BC0F4B9FED0F7AD3ED007A94
:10A94800F8EEE77A67EE877AFFF718B9943D0020AA
:10A9580080969800DC76002015D9020889888888B6
:10A9680073B2E745D34D621029C401088F3D00201A
:10A9780029000020B83400200AD7233C1F85EB515A
:10A988009C4B1B88DA0513D4D80600F12783990657
:10A9980000F131835A0600F14483180700F143831C
:10A9A800D90700F1428313F0020F0CBF04270C27CC
:10A9B800914B924A1B78D27803F001030AB143F015
:10A9C80002035320029322F06DFF8D4A128802EB96
:10A9D800820202EB8202900080B222F049FF00203E
:10A9E80022F046FF874A884912882868C2EBC212BB
:10A9F800520081FB023111444FEAE279C9EB612927
:10AA08005FFA89F94946F6F7C5FE98F80020029BD7
:10AA180028681F4389EA0209002188F80090F6F7A0
:10AA2800B9FE39462868F6F7B5FE98F80030286868
:10AA38007B40DBB2194688F80030F6F7ABFE94F895
:10AA48005831002B7FF4FFAA4F2022F02BFF15F07E
:10AA58001DFF15F01BFF15F019FF01212868F6F7F7
:10AA680099FE6A4A98F800301778286807F00107B5
:10AA7800394683F0010388F80030F6F78BFE98F822
:10AA8800003028685F40394688F80070F6F782FE83
:10AA980094F85831FFF7D7BA5D4E5E4B0093002407
:10AAA800A6F13F015C4B5D4A089106F8404C5C49B1
:10AAB80009960AA8F8F722FC089E731C08933470BC
:10AAC800089B2922591C08911A70089BEA22591CD4
:10AAD80008911A70089BC822591C08910AA81A7074
:10AAE80025F040FE471C0AA93A46089826F0CEFDF4
:10AAF800089AD31901330893D455089B5A1C089215
:10AB08001C70089B5A1C08921C70089B5A1C0892BF
:10AB18001C70089B5A1C08921C70089B5A1C0892AF
:10AB28001C70089B5A1C08921C70089B5A1C08929F
:10AB38001C70089B5A1C08921C70089B5A1C08928F
:10AB48001C70089B5A1C08921C70089B5A1C08927F
:10AB58001C70089BFF22591C08911A70089B01223F
:10AB6800991812A808911A7050F8283D9B1B337049
:10AB780011F026FC2C70FEF7F1BB88468946084682
:10AB8800049105918E4606910391FEF721BE254A50
:10AB98001F4B12680B93A3F1400500202121D70019
:10ABA80003F8400CA97040F1D5811F490326114BC9
:10ABB8001B88580500F1CB81DA0700F1198203F0F0
:10ABC80002031A4A002B1CBF03261146184F3246AF
:10ABD800384626F05BFDF31912A80133B91E40F878
:10ABE800203D00225B1AF2556B7011F0E9FBFEF76D
:10ABF8006DBC00BFFC3D002035560020A43D002060
:10AC0800D87400208C3D0020030820804C39002097
:10AC18004C3E002079540020C86B0308D06B030811
:10AC2800DC6B030844390020B46B0308C46B0308C9
:10AC38000F3E0020DFF870A39AF80090B9F1000FDA
:10AC48003FF457ADC94AB4F81C8111883B68029299
:10AC58004FEA081864201FFA88F800FB01914FEAB0
:10AC68004900B1FBF0F148EA01285E20C1F3032155
:10AC78001FFA88F848EA010898473B680620984771
:10AC88005FFA88F022F0EAFE4FEA182022F0E6FE8A
:10AC9800B4F81C31029AB649B2F800804A7A0133F6
:10ACA8009BB2012A93FBF9F009FB1033A4F81C317D
:10ACB80000F0BD816E23AF4A497B03FB08F382FB9A
:10ACC8000302DB17C3EBA20321B19BB29AF8002061
:10ACD80093FBF2F33A68DFF8D4825E201FFA83F917
:10ACE80090473B683A209847A8FB09384FEA58181C
:10ACF8001FFA88FA5FFA8AF022F0B0FE4FEA1A20AB
:10AD080022F0ACFE3B685E2098473B683B209847A2
:10AD1800642303FB18939BB29748053380FB0320F9
:10AD2800DB17C3EBA000C0B222F098FE002022F08F
:10AD380095FE3B68DFF84892DFF83C825E20984732
:10AD48003B6828209847D9F8003088FB0328DB1790
:10AD5800C3EBA8085FFA88F022F080FEC8F307204A
:10AD680022F07CFE3B685E2098473B6804209847A9
:10AD78002B89002B40F04C81D9F8085085F3100539
:10AD8800E8B222F06BFEC5F3072022F067FEB0E4BC
:10AD9800C4F82CB11D70FEF765BA784A734B0B9254
:10ADA80012AEA2F13D0046F8200D1988744FA2F1A9
:10ADB800400300204FF00A0E02F8400C082283F8E6
:10ADC80001E030469A70F8F79EF93B686A49DA174D
:10ADD80081FB0313C2EBA30399B23046F8F793F94A
:10ADE80008F04EFEBF680A9B3A0C591C0A911A706B
:10ADF8000A9B3A0A591C0A911A700A9B5A1C0A9211
:10AE08001F700A9B5A1C0A921870304611F0D8FA23
:10AE1800FEF759BB5B4F9FED5C8AB7F90220574894
:10AE28000B9007EE902AF8EEE77A12AE67EE887A72
:10AE3800A0F13D01FDEEE77A46F8201D00F8403C00
:10AE48000823CDED027A00F83F3C1E23BDF8081018
:10AE580000F83E3C3046F8F756F9B7F9003007EEEF
:10AE6800903AF8EEE77A304667EE887AFDEEE77AB0
:10AE7800CDED027ABDF80810F8F745F9B7F90430B6
:10AE880007EE903AF8EEE77A304667EE887AFDEEFC
:10AE9800E77ACDED027ABDF80810F8F734F93046B4
:10AEA80011F08EFAFEF70CBB02213868F6F766FC43
:10AEB80094F83431FEF703BA1023042218460AA97D
:10AEC8008DF82A808DF82B808DF82C808DF82D80B8
:10AED8008DF828308DF8292022F0FCFC84F83F8179
:10AEE800FEF716BA4046FFF7E1BB2849881F22F053
:10AEF800BFFB84F84E01FFF7C8B91C4B1988FFF750
:10AF08007FBB234AD278002A0CBF4FF0040C4FF0C5
:10AF1800050CFEF747BF012238681A70F6F731FCB6
:10AF280005463868F6F72DFC6D067EF49BA98E2839
:10AF38007EF498A994F82831002B7EF4AFA9154B1C
:10AF4800C4F830312D2384F83431FEF792B9032642
:10AF580011493BE6114B124A1B68124903F480035E
:10AF6800834216BF11460426032620E6D874002023
:10AF780010750020310CC330676666664C3E0020B1
:10AF8800CC7400200455002058A08B41502000208C
:10AF9800A43D0020CC3E0020B86B0308386C00208C
:10AFA800B46B0308AC6B03081E7500201F85EB51BA
:10AFB8003C499A790B8803EB830303EB83034FEA3D
:10AFC80083081FFA88F8002A40D0374B1B680FFA0D
:10AFD80083FA08F055FD40B2FEF702BB3427E7E4D8
:10AFE800984699461846049305930393FEF7F0BBD9
:10AFF8002E490426EAE52427DAE44B1CDBB2042BAD
:10B0080084F851314FEA01617FF491AAFFF78CBAB5
:10B0180008F036FD22F022FD002022F01FFDFFF788
:10B0280068BB1027C4E42027C2E40827C0E43B68B3
:10B038005E2098473B68392098475FFA88F022F0ED
:10B048000DFD4FEA182022F009FD72E64FF0FF339C
:10B05800BDE7984699461846049305939E46039380
:10B06800FEF7B6BB0393FEF7B3BB98460393FEF710
:10B07800AFBB0D4B9046B3F900A06420FEF7B0BA01
:10B0880098469946184604930393FEF7A1BB984641
:10B0980099460393FEF79CBB984699461846039336
:10B0A800FEF796BBD8740020CC740020BC6B030854
:10B0B8002DE9F04F724B734A1C7893B000F59C4110
:10B0C8002031814607911160002C00F00D856E4AF1
:10B0D8001268904240F22E826C4A6D491768DFF878
:10B0E800E8B10492013C1C706A4C039107F4805744
:10B0F800002F40F02C82039B5B7D002B40F0C08426
:10B10800049B1B681D0400F11A87634B9945A378BB
:10B1180000F29D83002B40F09D83604B0593049BB8
:10B128001F6817F4805940F05584039BBBF90660EB
:10B138005B8B9E42B4BF00260126594B1B6813F057
:10B14800805300F00E82059A127812F0010200F086
:10B158000F8203985349408C91ED037A07EE900AC9
:10B16800F8EEE77AB4EEE77AF1EE10FA80F2E187CA
:10B17800002E40F004824C4D95F8A010002940F0B4
:10B18800FE814A494A480D6895F82D500021016012
:10B19800416081604749002D40F0F2810D70002A1E
:10B1A80040F0F381444B1A78002A50D10399BBF937
:10B1B80000E04F8B898BBBF90200BE45CCBF8025D0
:10B1C800002545F040038E45A8BF2B469B0843F059
:10B1D8008005B842C8BF2B4643F040058842A8BF47
:10B1E8001D46BBF904E0BBF90600AD0845F0800335
:10B1F800BE45C8BF1D4645F040038E45A8BF2B4637
:10B208009B0843F0800E284DB842C8BF734643F0F0
:10B21800400E95F8A2708842B8BF73469F4201F06D
:10B228002181A5F8A42085F8A620244985F8A23014
:10B238000F78002F01F06D805F2B01F0F8806F2BE5
:10B2480000F0CF87059B1B78DB0740F19187049BB3
:10B258001B4A1B68069203F00403002B40F0FB8492
:10B268000DF14008174D0023C8F8043005F15009C6
:10B27800109340F6330A192740F2833629E000BFBD
:10B288002C590020A057002028590020386C002095
:10B29800AC6D0020A43D0020404B4C0035560020EA
:10B2A8004439002020750020D82100208054002037
:10B2B800B038002034240020596E0020D405002026
:10B2C800A8540020343B00204C53002004354D4541
:10B2D80020D0AA78EB789A4217FB0261F6D26A78F6
:10B2E800043217FB03633BF912205245A8BF5246AC
:10B2F800B2F5617FB8BF4FF461728A42E6DD9A42C7
:10B30800E4DC29782429E1D840460435F8F780F9A7
:10B318004D45DED1B34B98E803001F78B24B83E864
:10B328000300002F00F022840121AF48F8F77FF9CD
:10B33800002840F0A681E378002B40F0A281AB4CB6
:10B3480023881DB225F00105AEB2B342268000F075
:10B358008986A74D02270E204FF014094FF0FF08E9
:10B368002F7085F8019085F8028024F053FA394649
:10B378009D482688F8F75BF9002841F0258026F0DB
:10B3880002039BB2B34223800AD0994B1421FF22B7
:10B3980002250E201D7059709A7024F03BFA2688F9
:10B3A800944BDFF89CA21978DAF804000393B507E8
:10B3B80008BF81F00201C1F34001F7F769FA2421BF
:10B3C8008948F8F734F930B9059A1378590744BF12
:10B3D80023F004031370069B1B6813F00A0F24D094
:10B3E80005218148F8F723F9002800F06F862588A1
:10B3F8006B0740F169877C480621F8F718F900289F
:10B4080000F051866F0640F17C8707217648F8F7EF
:10B418000EF950B1784B794AB3F90430784982FB78
:10B428000302DB17C3EBA2030B800C216E48F8F76D
:10B43800FEF82288002800F0408142F480739A4286
:10B44800238009D06A4B02251421FF220E201D708B
:10B4580059709A7024F0DEF96A4B1B78082B00F0BB
:10B4680038810E2B00F03581049B1B685E0544D59E
:10B47800654B1B79002B00F0E98014215A48F8F736
:10B48800D6F8002840F0E78011F00AF8012024F0EF
:10B4980003F990B3DFF8AC8100254FF0CC0902E046
:10B4A800DDB2022D29D809FB05F76B1C58F8076097
:10B4B800002EF5D1C378554A90F9020052F823308E
:10B4C8000196032200920121324623F07BFE0346B7
:10B4D80005EB450000EB0010049353B1314608EB2F
:10B4E8008000CC2228F051FB049B48F80730013536
:10B4F800EDB21DF0C7FE0028D3D1059B1B78DD07F0
:10B5080040F1FA804249434A01230B701370039BB0
:10B51800DAF80000197801F00101F7F7B9F9069B8C
:10B528001D686A0700F15881EB0600F1728113B0BB
:10B53800BDE8F08F384B394A1F68049307F48057E9
:10B548000392DFF804B1364C002F3FF4D4AD00214C
:10B558002548F8F76CF800287FF4CDAD07F0CCFB50
:10B56800C9E578023FF5EFAD059A127802F00102BD
:10B578002C4D002185F8A010002E3FF402AE2A4978
:10B5880001200870002A3FF40DAEF9067FF50AAED7
:10B59800264A1278D2063FF505AEB9F1000F7FF4BE
:10B5A80001AE002B7FF4FEAD7D023FF5FBAD204BD5
:10B5B8001B78002B01F042831E4B9B78002E41F034
:10B5C8004D833BB11C4A1D4B12681B689B1A002B0C
:10B5D800C1F2E9831020134D24F01CF9012385F8EA
:10B5E800A130DFE56F54002044390020FC3D0020E5
:10B5F80044380020305700200455002067666666EE
:10B608009C340020303B002010750020545B030858
:10B6180036560020CC340020386C0020AC6D002059
:10B62800A43D0020D8210020342400204C390020DB
:10B63800D4050020EC78002068570020A4250020BD
:10B64800345700205C4F00204C530020059B1B788A
:10B65800D8077FF519AF3C2014F074FF00283FF499
:10B668004CAF09F0BDFA3C2014F00EFF00283FF45F
:10B6780044AF09F0B5FA3C2014F006FF0028F0D1D9
:10B688003BE7069B1B689A077FF559AEAC4C2688AA
:10B69800F3073FF574AE46F001039E4223803FF462
:10B6A8006EAEA84B1421FF2202250E201D70597082
:10B6B8009A7024F0AFF8268861E622F480739BB272
:10B6C8009A4223807FF4BEAE9F4B1B78082B7FF4F1
:10B6D800C8AE228822F040039BB29A4223803FF4EE
:10B6E800C3AE984B02251421FF220E201D705970FD
:10B6F8009A7024F08FF8B7E6944B93F80090B9F15C
:10B70800000F5FD1DFF89082914F18F8030C3E7854
:10B718004146A8F1030517F0EFFC002800F0B883B4
:10B72800002E40F00A8405F10801687917F0E4FC5E
:10B73800002841F095818749A87A17F0DDFC002898
:10B7480000F0B983022E41F08F818349E87B17F01E
:10B75800D3FC002841F08C818049287D17F0CCFC6F
:10B76800002800F0B983042E41F086817C49687E68
:10B7780017F0C2FC002841F083817A49A87F17F0AE
:10B78800BBFC002800F0B983062E41F04C817649B5
:10B7980095F8230017F0B0FC002840F0158773498E
:10B7A80095F8280017F0A8FC002800F0B983082EA7
:10B7B80040F0F4866E4995F82D0017F09DFC00289E
:10B7C80040F0B9836B4B01221A7024F049FE069BA6
:10B7D8001D686A077FF5A8AE032017F0B7FC00289C
:10B7E80000F05886238813F008067FF49DAE0820E1
:10B7F80024F020F96048614B006818606049614A8C
:10B80800069D614BBBF806002D68088016601E6017
:10B818008AE6162017F09AFC002800F01D86238877
:10B8280013F400747FF483AE4FF4007024F002F92F
:10B838005148534D5149534A534BBBF80660006871
:10B848002E80086014601C6013B0BDE8F08F0BB93F
:10B858000123A3704D4B05931B201F7894F821609A
:10B8680017F074FC012E07F00109824600F0DB8511
:10B8780007F00203069394F82030DFF82081444D46
:10B88800052B00F29A80DFE813F08B004F000600CA
:10B89800D800F900BD00012E04BF052384F820302C
:10B8A800B9F1000F00F00D81039B3A4FB3F918105E
:10B8B800B8F80030002261F30F0263F31F4200233F
:10B8C80061F30F0361F31F43CBF804203968626901
:10B8D800CBF80030914200F21384012E41F0DC8154
:10B8E800032294F820300692CAE717F05BFC01287F
:10B8F80007D1284FB8F802303A68642101FB0323C6
:10B908002361BAF1000F04D098F80630002B40F0FC
:10B918008C80012E51D01F4F22693B689A42C0F09B
:10B92800F485012384F82030012E6BD098F8073075
:10B93800012B00F0CF800EF0A9FB94F820309FE790
:10B94800FC3D002044380020303B002036560020C3
:10B958002B000020D8360020DD360020E2360020FB
:10B96800E7360020EC360020F1360020F6360020BD
:10B97800FB360020CC340020B8340020B43400203A
:10B98800A8340020AC340020A43400203556002010
:10B99800C83D002068570020CE36002028380020F7
:10B9A800B9F1000FA1D14FF48060BAF1000F00F097
:10B9B800778324F03FF800232361069B002B3FF494
:10B9C800AEAB069823F026FF049B1F6817F4805936
:10B9D8003FF4ABAB1D21B248F7F729FE00287FF4EE
:10B9E800A4ABB04A039BD2881B8BBBF90660991A9B
:10B9F8008E4240F3948513449E42B4BF002601262C
:10BA0800FFF79BBBA84F3A68B8F80230642101FBE6
:10BA180003234FF480600022236184F82020E27021
:10BA280023F0F0FF94F820302AE70EF02FFB0322D2
:10BA38004FF47A7384F82020E3619B4F2B8843F0FE
:10BA480002032B8007F058F93A68E369134404228B
:10BA5800A36184F82020012E40F051853B68A2693B
:10BA68009A42AAD2914B187818B917F06FFB0028A0
:10BA7800A3D12B8823F002032B80C4E78A4FEAE77F
:10BA8800039A013BD27D3BF91330002A40F03383FF
:10BA9800A3F57A73B3F57A7FA8BF4FF47A7323EAD4
:10BAA800E37307EE903A9FED827AF8EEE77A67EE55
:10BAB800877A804AFCEEE77A17EE903A1380FFF710
:10BAC80024BB794F3B6847F230520323E26184F884
:10BAD8002030B3E70EF0DAFA032240F6B83384F8E0
:10BAE8002020E361704FA9E7734F3B78002B00F0EB
:10BAF8004F87724BDFF8D881DFF8D8B1DFF8D8A1CB
:10BB0800039345465E46049099460EE019F80410E2
:10BB18009847032C28DC88B93B782AF8020F0134AF
:10BB28009C4205F1040580F2DD80072CE1B2304625
:10BB3800DBF80430EADD984700B2EDE738F8242056
:10BB48006B88801A4FF47A719B1A01FB00F040F65B
:10BB5800CA0290FBF3F00844904240F2EE23A8BFDB
:10BB680010469842B8BF184600B2D5E7DFF86CA176
:10BB7800DFF86C81524D0AF15A064FF0010951461F
:10BB88001AF8010C17F0B8FAF8B19AF804009AF804
:10BB980002309AF803E000EB400105EB8101013B1C
:10BBA800D1F8B42003EB4303434493420DD095F8F6
:10BBB800E02081F8B0E009FA00F022EA0000C1F8BC
:10BBC800B430C1F8B87085F8E0000AF1060AB24549
:10BBD800D5D13C49344A3C4B3C4D09681B78D2F8D6
:10BBE800009008910793A5F1B00A00266B685BB333
:10BBF8001F784FB3AA68A9EB0202002A0ADB9AF859
:10BC0800E0200121B14022EA010209F5FA718AF81F
:10BC1800E020A960079ABAB12A7859780432D2B2DA
:10BC2800002940F08C8203993BF91220098B01F11D
:10BC3800C800824240F335849AF8E0109A7841FAB5
:10BC480006F3D80740F1A5840136042E05F10C054A
:10BC5800CCD1FFF769BB1A4D95F8AA3053B1059BB3
:10BC68001B78DE0706D5039BBBF906205B8B9A423F
:10BC780000F3658411210A48F7F7D9FC002800F081
:10BC8800468295F8AE302BB995F8A83013B932230F
:10BC9800A5F8AC30012385F8AE30FFF7E1BA00BF54
:10BCA800443900200C38002068570020D4050020B3
:10BCB800AAF1823F8C3D002080590020AC6D002005
:10BCC800D821002000560020853D00208822002031
:10BCD800985900202C550020D6210020E535002059
:10BCE8009C420308DDF81090C44A04921146C44AE5
:10BCF8000968A2FB092A42F201020A404FEA9A1A8D
:10BD0800059200F00082BF4DBF48C04CC04A95F86C
:10BD180000E0007884F800E01070BEF1000F04D055
:10BD2800BB4A92F800E08EF0010EBA4D0F2085F85C
:10BD38002400002B00F0FA82B74B039E0C931B786B
:10BD4800B6F826C00B931C463B78B78C039EB34AC3
:10BD5800368B0E962646A2FB0442520802EB42029C
:10BD6800B21AD2B2CDF824C001F48051089295F8E5
:10BD78002580DFF8C0B2DFF8E8C20A900AF59672AB
:10BD880076460F9105F1280400200692CDF83490EC
:10BD9800AE46002E00F03A823EF910201FFA82F9D2
:10BDA800B9454FEA400103D3099DA94540F2728283
:10BDB8005CF82020924580F032823BF90120059DF5
:10BDC800002D40F04682013098422BF8012004F102
:10BDD8000604DEDB0A98924ADDF834908EF8258056
:10BDE8000F280CBF012100218EF82400117000F0EB
:10BDF800A4828C4C8C4E8D4F35883868A168626857
:10BE0800E06045F00405401A90427F4F3580804D30
:10BE18004FF0010188BF00223970297088BF84F86B
:10BE28002120002B00F09B82049A03991768804E0A
:10BE3800B1F824C0B1F818E07E4817F480573546A9
:10BE480040F0D38239460EE06A7802EB820202EBB8
:10BE5800820202F2EE2292B20131994220F8022BBC
:10BE680005F102050ED016F81120002A00F01682FE
:10BE7800022AE9D00131028820F8022B994205F103
:10BE88000205F0D10C9A137801331370FFF730B91B
:10BE980008F10501687917F02FF900283FF44BAC39
:10BEA800012E40F0DD8505F10D01A87A17F024F97F
:10BEB800002840F0D9856049E87B17F01DF9002873
:10BEC8003FF44AAC032E40F0D3855C49287D17F037
:10BED80013F9002840F0D0855949687E17F00CF90D
:10BEE80000283FF44AAC052E40F0CA855549A87F82
:10BEF80017F002F9002840F09685534995F8230079
:10BF080017F0FAF800283FF44AAC072E40F05C839B
:10BF18004E4995F8280017F0EFF8002840F03E83C6
:10BF28004B4995F82D0017F0E7F800283FF44AAC84
:10BF3800092E3FF447AC4FF009094B4631E3354D24
:10BF4800D5F88830A9EB0303002BFFF6DEA8414A99
:10BF580095F88C30517C079AC5F8882001333E4A01
:10BF6800039E32F81120B17D03F00F0385F88C3061
:10BF78002B4492B292FBF1F283F8902095F890103E
:10BF880095F8912095F8923095F89C000A4495F818
:10BF98009310134495F89420194495F895300A4461
:10BFA80095F89610134495F89720194495F8983009
:10BFB8000A4495F89910134495F89A20194495F86D
:10BFC8009B300A44134495F89D1095F89F20184417
:10BFD80095F89E3001440B441A4442F30B12642A2C
:10BFE800F17DA8BF642213B209B1C2F1640307EE60
:10BFF800903A9FED1A7AF8EEE77A58E5386C002007
:10C00800D34D62107C5700208C070020853D00200E
:10C018008D070020D82100202D590020ABAAAAAAFC
:10C028002A550020A43D0020C83D00206857002064
:10C03800CC5900204C530020DD360020E236002089
:10C04800E7360020EC360020F1360020F6360020D6
:10C05800FB360020B4560020D056002014AE2341F1
:10C06800305900200221C648F7F7E1FA00283FF4CA
:10C0780086A92580B7073FF593A946F00203B34286
:10C0880023803FF48DA9BF4B02201421FF22187092
:10C098000E2059709A7023F0BDFB2688FFF780B9EF
:10C0A80023F0B0FC87E425F040039BB2AB42238029
:10C0B8003FF4ABA9B34B02251421FF220E201D70BB
:10C0C80059709A7023F0A6FBFFF79FB9238823F0D5
:10C0D8000405ADB2AB4225803FF48DA9A94B0225DA
:10C0E8001421FF220E201D7059709A7023F092FBC4
:10C0F8002588FFF780B9C3F53B6308331BB2C7E453
:10C1080003230693DFE4A04A92F800E005E695F8D9
:10C11800A830002B3FF4A4A8059B1B7813F001035B
:10C128007FF49EA8012285F8A83085F8A920FFF79A
:10C1380097B8964D012185F8A010FFF720BA01297C
:10C1480000F0E0839AF8E0200123B340013613435E
:10C15800042E8AF8E03005F10C057FF447ADFFF7AF
:10C16800E3B8059B8A4A1B781060D80700F1F5816F
:10C1780095F8A61000297FF46AA8B5F9A430322BE7
:10C188007FF765A895F8A2200120572A85F8A60010
:10C1980000F02E84049B1B6813F0040302D05A2A73
:10C1A80000F039855D2A00F0B1845B2A00F0D38461
:10C1B8005E2A00F0DD84562A00F01285972A00F0E6
:10C1C8001E85A72A40F06A847249049B0A781B6876
:10C1D80042F004020A70704A069203F00403FFF763
:10C1E8003CB8B2F5FA7FFFF632A895F8A620002AE7
:10C1F8007FF42DA8059B1B78012185F8A610D90787
:10C2080000F1428405F0FCFEFFF721B8002F3FD073
:10C218005CF8202092454FEA4001FFF4CEAD5F4A1A
:10C228005E4D525C05EB0109002A00F09D80022A50
:10C2380047D199F8012002EB820202EB820202F256
:10C24800EE2292B2032833DD059D12B2002D3FF491
:10C25800BAAD089D24F81520B8F1000F03D10B9D45
:10C26800022D7FF6B0AD2288B4F80290B4F80480AD
:10C278004A4490444A4A0FFA88F882FB0852494DCA
:10C28800A2EBE87225F8018012B24FF001089AE596
:10C298003A464100069D4CF8205090E5CAB2022A61
:10C2A80004D9032A7FF4E6AD6246D5E57246D3E5A4
:10C2B800012505FA00F90A9D25EA090512B20A9531
:10C2C8007DE53BF80120BDE745F004039D4223804E
:10C2D8000AD02C4B02251421FF220E201D70597004
:10C2E8009A7023F097FA25882F4B304AB3F9043017
:10C2F8002F4982FB0302DB17C3EBA2030B80FFF776
:10C308007AB845F04003AB4223807FF4D3AEFFF701
:10C318007CB839461A48F7F78AF900283FF421AF64
:10C3280085F8A77005F06CFEFEF78CBF2149224AFC
:10C338000C91DFF890B0012111701B211048059372
:10C34800F7F775F9059B00287FF453AD1B4C1C4F7C
:10C35800E2683B68A3609B1AC82B00F23B83049BEE
:10C368001F6807F480578DE5C2B2022A40F2C882DE
:10C37800032AA6D10E9A0F9D002D08BF3A4661E701
:10C388004439002044380020853D0020D821002071
:10C39800A82500204C390020A8540020CC590020A2
:10C3A8005655555548220020045500206766666694
:10C3B800883400202D5900202A550020A43D002053
:10C3C800685700204C53002026F001039BB2B3426B
:10C3D80023803FF44FAE0E202F7085F8019085F82A
:10C3E800028023F017FA268844E600210FE06A78D5
:10C3F80002EB820202EB820202F2EE2292B20131D9
:10C40800994220F8022B05F102053FF43BAD16F8DE
:10C4180011201AB1022AEAD00288F0E7CAB2032A28
:10C42800FAD87246EBE700230693FFF724BAB2F571
:10C43800FA7FFEF60CAF95F8A630002B7EF407AF16
:10C44800059B1B7801210B4085F8A61000F0A482FB
:10C4580006F052FCFEF7FBBE4FF4007023F0D2FA50
:10C46800FFF765B8BE4ABF491068B5F9A420C76987
:10C4780081FB07018911FF17781A00F5FF407F300B
:10C4880082423EF7D2AEC91B0A4412B2A5F8A420D4
:10C49800FEF7CBBE082023F0B5FA069B1D68FFF710
:10C4A80043B8C8398A423DDA9AF8E0109A7841FAD6
:10C4B80006F3D9073FF5C8AB52420120099223F091
:10C4C80089FA7B1E099A162B00F2C280DFE813F066
:10C4D800B001C6019701EF01DC01030282016D0181
:10C4E800560131011A01C000EF0105010302820162
:10C4F8006D01EF00D900C300AE00960080003A68D5
:10C50800E3691344A361FFF758BA0DF0BFFD032296
:10C5180040F6B83384F82020E361FFF78FBA01268C
:10C52800FEF70BBE9AF8E0300122B24023EA02037C
:10C5380009F5FA728AF8E030AA60FFF785BB002196
:10C548008948F7F774F800287FF494AB322385F80C
:10C55800AA00A5F8AC30FFF78DBB844B1B78002BE5
:10C568003EF475AEE378002B7EF471AE95F8A730F3
:10C578000133DBB2032B85F8A7307EF668AE7C4B1F
:10C588005B7813B9002E7EF462AE06F0B5FBFEF7B9
:10C5980059BE002A0CBF012002208FE74FF008097E
:10C5A8004B4603EB83031D4487F80090A97868780D
:10C5B80015F0D8F9059B6F4A1B7801211170D9072E
:10C5C8007FF503A9FEF7A3BF4FF007094B46E8E73D
:10C5D800DAF8E400DFF8A08190F8361098F8023015
:10C5E80011446429A8BF642121EAE17180F836105A
:10C5F800002B40F08B8320F00FFAA3E5DAF8E40073
:10C60800DFF8748190F8371098F802301144FE2949
:10C61800A8BFFE2121EAE17180F83710002BEAD08B
:10C62800162016F0F1FDDAF8E400E4E70898DFF8E0
:10C63800488141781144B1F5967FA8BF4FF49671AF
:10C6480021EAE171417098F80230002B40F05883DC
:10C65800DAF8E400CFE7DAF8E400DFF81C81817843
:10C668001144C829A8BFC82121EAE171817098F84E
:10C678000230002BBFD0142016F0C6FDDAF8E40013
:10C68800B9E7DAF8E400DFF8F08041781144C82906
:10C69800A8BFC82121EAE171417098F80230002B47
:10C6A800A9D0132016F0B0FDDAF8E400A3E7DAF811
:10C6B800E400DFF8C48001781144C829A8BFC82164
:10C6C80021EAE171017098F80230002B93D0122012
:10C6D80016F09AFDDAF8E4008DE7DFF89C800898F8
:10C6E80098F80230417911446429A8BF642121EAED
:10C6F800E1714171002BABD00E2016F085FDDAF800
:10C70800E40078E7DAF8E400DFF86C80017A98F85A
:10C7180002301144C829A8BFC82121EAE171017279
:10C72800002B3FF468AF0B2016F06EFDDAF8E4003A
:10C7380061E7DAF8E400DFF84080C17998F8023060
:10C748001144C829A8BFC82121EAE171C171002B91
:10C758003FF451AF0A2016F057FDDAF8E4004AE733
:10C7680040400020D34D621044390020853D002010
:10C77800EC780020CC340020365B0020DAF8E400A6
:10C78800DFF87885817998F802301144C829A8BF64
:10C79800C82121EAE1718171002B3FF42CAF0920F7
:10C7A80016F032FDDAF8E40025E7DAF8E400DFF8FD
:10C7B8004C85417998F802301144C829A8BFC8218E
:10C7C80021EAE1714171002B40F05382112F7FF46F
:10C7D80046AF10E7DAF8E400DFF82085017998F829
:10C7E80002301144C829A8BFC82121EAE1710171AA
:10C7F800002B40F0D082102F7FF447AFFBE608995A
:10C80800DFF8F8840F791744642FA8BF642727EA54
:10C81800E7770F7116F012FD98F80230002B3FF4FD
:10C8280017AF0320394616F0EFFCDAF8E400E2E629
:10C838000898DFF8C88401781144FA29A8BFFA21BA
:10C8480021EAE171017098F80230002B3FF400AF43
:10C85800012016F0D9FCDAF8E400CCE60898DFF8F5
:10C868009C84817811446429A8BF642121EAE1717C
:10C87800817098F80230002B3FF4EAAE022016F0DF
:10C88800C3FCDAF8E400B6E60898DFF87084C179EA
:10C8980098F80230114481F30801C171002B3FF46C
:10C8A800D7AE052016F0B0FCDAF8E400A3E6089B42
:10C8B800DFF84884997998F8020011446429A8BFE0
:10C8C800642121EAE1719971002840F0DA810D2F85
:10C8D8007FF405AFBCE6DAF8E400DFF82084C1781D
:10C8E80098F802301144C829A8BFC82121EAE1718B
:10C8F800C170002B40F05F820F2F7FF4DCAE7AE628
:10C908000E9A9FE43BF912209978B2F5617F4FF4B3
:10C91800966393FBF1F332DB40F633019142A8BFF3
:10C9280011460C2FA1F5617191FBF3F100F0F9802C
:10C93800182F7FF407ACC9B2C8290B46A8BFC82373
:10C94800DAF8E400C27DDFB297423FF4FBAB9A1AF3
:10C95800DFF8A883C77548BF0732D71098F80230A8
:10C968000137FFB23BB9002F3FF4ECAB384623F058
:10C9780031F8FFF7E7BB182016F046FCF3E70C2F59
:10C9880000F0E680182F7FF4DDAB00210B46D7E7D7
:10C99800C34A0392FFF7A8B9C249096811F40031E4
:10C9A80040F0EA800B46C048C65C0F2E03F10C032A
:10C9B8003DD001311529F7D1049BBC491B6806916C
:10C9C800FA3AA5F8A420002203F0040385F8A6206B
:10C9D800FEF743BCB64A049B1F68138823F0040380
:10C9E8001380012307F4805784F82130FFF74ABAEF
:10C9F800AE4AB04B069210461A68AF494FF47A73A4
:10CA0800B3FBF2F3C3EB431203EB82030268DB00D0
:10CA18005707A1F8B43000F1A280049B1B6803F00B
:10CA28000403FEF71ABC4FF006094B46B9E5A34EBE
:10CA3800D6F800E04B00BEF1000F07D05F1800EBFE
:10CA480087079EF801E07F787745B5D20B449C4F65
:10CA58009C4900EB8300002330603B800B60ABE710
:10CA68004FF001094B469CE54FF002094B4698E50B
:10CA78004FF003094B4694E54FF004094B4690E507
:10CA88004FF005094B468CE5049B8F491B680A60EB
:10CA9800864A069203F00403FEF7DFBB0021BB2A97
:10CAA800109100F09880B72A00F09180BE2A00F01B
:10CAB8009580BD2A67D0792A00F05A817A2A00F039
:10CAC80050819E2A00F047819D2A00F03D81AE2AC0
:10CAD80000F03381AD2A00F02981EF2A00F020818F
:10CAE800FD2A00F01781FB2A00F04F81FE2A00F092
:10CAF8004681F72A00F067817B2A7EF4A8AB4FF4C1
:10CB0800FA61022006F0CEFEFEF7A1BB6F4B0022B1
:10CB180001206F4D6F492A700B6022F05BFFFEF712
:10CB280096BBCFB26A4B09915B78BB423FF40AAB24
:10CB3800DFF8C881384606F08FFF98F80230099967
:10CB48001BB1C9B20C2016F05FFB0137FFB20AE730
:10CB580000273946E6E7604B01220220D9E7049B0B
:10CB68005E4A1B680A21118003F00403FEF775BBB7
:10CB78005B4B02220320CCE75A490978032900F0CD
:10CB8800868019460FE74FF6FE73574A474896893D
:10CB98000690D089334401449381D18119F0C0FAB9
:10CBA800F6F790F819F0A4FAF9F754FF012022F0EB
:10CBB80011FF049BB5F8A4201B68FA3A0021A5F8D8
:10CBC800A42003F0040385F8A610FEF746BB0B4625
:10CBD8004FF6FE71D9E70B460221D6E70223D4E7C8
:10CBE80019F09EFAF6F76EF819F082FAF9F732FFA3
:10CBF800012022F0EFFE95F8A220FFF7DFBA049B90
:10CC08003A4A1B684FF4C8711180284A069203F00B
:10CC18000403FEF722BB95F8A820002A40F0DE8026
:10CC280095F8AA3083F0010385F8AA30002B40F06C
:10CC3800D0800C2022F0EEFDFEF709BB002E3EF45A
:10CC4800C9AC2B4D95F8A130002B3EF4ABAA22F0CD
:10CC5800C5FD002385F8A130FEF7A4BA002BF0D05B
:10CC68002449254A09684FF47A7000FB03131360BE
:10CC7800E7E71120099216F0C7FADAF8E400099AF2
:10CC8800A4E50D20099216F0BFFA099A1FE622F0D2
:10CC9800A5FDB5F9A4208FE603230693FEF791BE00
:10CCA800AC6D0020D835002058590308A85400203E
:10CCB800C83D0020286C0020BC5F0020E423002031
:10CCC8007E24002080240020A82500201A5A002055
:10CCD8007454002080540020685A0020E678002010
:10CCE800B65A00208F3D0020F4450020E878002047
:10CCF800D821002068570020A4250020365B00209A
:10CD0800152016F081FADAF8E40074E4172016F01A
:10CD18007BFA9DE40021012006F0C4FDFEF797BAD6
:10CD28000021084606F0BEFDFEF791BAFF2100205B
:10CD380024F062FC95F8A220CFE60121002024F01F
:10CD48005BFC95F8A220C5E60021FF2024F054FCE6
:10CD580095F8A220BBE6012024F04EFC95F8A2200D
:10CD6800B2E6224A137A43F001031372FEF76FBA50
:10CD78001E4A137A23F001031372FEF768BA0021E2
:10CD8800032006F08FFDFEF762BA0021022006F0AC
:10CD980089FDFEF75CBA1020099216F035FADAF828
:10CDA800E400099A27E5124D05F0A6FF002385F84F
:10CDB800A130FEF7F7B90F20099216F025FADAF834
:10CDC800E400099A98E50021042006F06BFDFEF7BF
:10CDD8003EBA0B2022F01EFDFEF739BA054A85F847
:10CDE800A81085F8A9000692FEF737BA105500205A
:10CDF800D8210020A85400202DE9F0478C4B1B783F
:10CE0800DB07074644D58B4B8B4D1C788B4E012C8A
:10CE180059D01CD3022C07D189498A4A098812881B
:10CE2800914201D901241C70EB7AE3B12B89D3B16B
:10CE3800854B1B78BBB106F023FE002800F09B80D1
:10CE48002B7B83422CBF0121002131700CE07C49EF
:10CE58007E4A098810886A7B801A8842E2DAEB7A6F
:10CE68000024002BE2D131782A79632A06D8022CD3
:10CE7800774E00F0BA803378002B5DD1754AAB7AD3
:10CE88008C4238BF0C461470002B4CD1BDE8F0879B
:10CE98006B4B694D19885B88E878CB1A83EAE37293
:10CEA8008142A2EBE3721DD32B788B421AD3614BDC
:10CEB8001C78E01E012861D96749097802294FD0FA
:10CEC800012C5E4EA5D15F4A5D491288687B0988AE
:10CED800121A914239DD5D4A12888A42A4D200248E
:10CEE8001C70A1E7B1EB400FE1DC524B1C78E11E4E
:10CEF800012940F29480022ADEDC57494F4E087817
:10CF0800DFF84481DFF844C1DFF838E10021032469
:10CF1800022834701C7088F80010ACF80010AEF8C5
:10CF2800001081D11FE0012C71D0022C0BD10720F9
:10CF3800BDE8F04722F06EBC7068381A474B98423B
:10CF480058DD72709AE7BDE8F08702241C706BE721
:10CF5800022AD2DD4049097802294FF0040464D13D
:10CF68003949364E09783E48022ACCBF00220122B0
:10CF7800C28081804BE70221317075E7022A9BDC71
:10CF880095F800C091FBFCFC0CF1010CBCF1080FFA
:10CF9800DFF8B4A0304EA87895F801E096F8008044
:10CFA8002A4CDFF8A090254EA8BF4FF0080C8AF84D
:10CFB80000C01FFA8CFA10FB0AF01EFB0AFE80B2B2
:10CFC800DFF88CA02080A9F800E000244FF0640E60
:10CFD800B8F1020F34701C70CAF804408AF801E0F6
:10CFE8007FF439AF0FFA8CF1BDE73078A0B901238F
:10CFF80077603370C2F164021A4B00FB02F083FBC6
:10D008000023C017A0EBA3506430707036E70820E7
:10D01800BDE8F04722F0FEBB7368F81A8EE7032CD0
:10D0280096D10D49097802299AD0044EFCE600BF32
:10D038003556002054260020943D00205A26002012
:10D04800D8740020582600201E750020562600207F
:10D05800943400208F3D0020207400207F96980093
:10D06800247400206BCA5F6B2DE9F04F2DED0C8BFB
:10D07800414B1B7897B0012B039001F0F681DFF844
:10D0880004B19BF80021002A41F0FE81072B01F032
:10D0980005824FF00009DFF8F0A0DAF804305046B6
:10D0A8009847002800F06A81BAF8B45000228AF83C
:10D0B8005520002D41F0A380BAF93C40DAF824103D
:10D0C800BAF93E00DAF82820BAF94030611ACAF8ED
:10D0D80030102A490191821ADAF82C00CAF8342053
:10D0E8000C461B1A9AF85610CAF838300AF1300064
:10D0F80011F0EEF82368990040F1E580DAED0D5A59
:10D10800DAED0C7A1E4A9BED416ADBED426A9BED33
:10D11800437ADBF810311268B8EEE58ADAED0E5A78
:10D12800F8EEE77AF8EEE58A013377EE867A38EE9C
:10D13800268A78EE878A9342CBED417A8BED428A34
:10D14800CBED438ACBF8103101F088850A4B1D7866
:10D15800142D03F091800023DBF818410293062C6C
:10D1680000F2A480DFE814F06816281708163917AB
:10D1780012001118AE1700BF20740020386C002070
:10D188004C420020C0220020BC5F0020D84B1A78F7
:10D19800DBF81C61D74F9FEDD87AF0003B1883ED80
:10D1A800007A002A78D0D549B0EE476AF0EE476A8F
:10D1B8000023F1EC017A013367EEA77A05EE903A85
:10D1C800B4EEE77AF1EE10FAF8EEE55AB8BFB0EE31
:10D1D800677A9A4276EEA76AA7EEA56AE9D1F5EED4
:10D1E800C06A3B18F1EE10FA83ED007A54DDC6EE02
:10D1F800265AC34BC34A1288F7EE007A75EEE75AEF
:10D20800D3ED007A65EEA77AFDEEE77A17EE903A4D
:10D21800812B43F3EB879342A8BF134607EE903A5E
:10D22800F8EEE77AB84B811903EB810393ED057AA1
:10D23800D3ED003A93ED066A93ED014AD3ED046A03
:10D24800D3ED034A93ED025AA3EEA77AA4EE276A18
:10D2580066EEC76AA7EE646ABDEEC77AE5EE276A8E
:10D2680017EE101A812983ED056AC3ED066A43F3A8
:10D27800BA878A42A8BF0A4607EE902AF8EEE77AEC
:10D28800FCEEE77ACDED047ABDF810303A189380B9
:10D2980016B9132D04F00683152D42F0C0853844C5
:10D2A8009A4F838827F81630DBF81841984B0134D9
:10D2B80083FB04231A19E317C3EBA203C3EBC303CD
:10D2C800E41ACBF81841934B1B78002B01F07282BB
:10D2D800914CCDF80890914FDFF83082DDF804903A
:10D2E80004F5BC7600258E4BDAED087A1B78172BEF
:10D2F80001F0768794ED007AB8EEC78A082B28EEFD
:10D30800278A07D1B0EE480A019324F033FB019B2A
:10D3180028F81500D9F8002092000BD5002D04F04C
:10D32800CD83B0EE480ADAF8143206F17000984757
:10D33800B0EE408AB0EE480ADAF83431A6F170004F
:10D348009847DAF8A43130469847754B1B78032B79
:10D35800B0EE408A01F03E87D4F8F800DAF8B83029
:10D36800B0EE480A98470135032D06F12406A7ECCC
:10D37800010A04F10404B6D1DDF80890684B1E7860
:10D38800072E00F0FA879BF828310493002B41F010
:10D398000080644B5B79002B40F02B870123604AA7
:10D3A8008BF828311278072A02F03283002305937C
:10D3B8005D4B9BED4C9A93ED007A5C4BDBED4BCAD1
:10D3C800D3F800905A4B0293F7EE007A37EEC9CAA9
:10D3D80000242CEE07CA574BDFF89881DFF898A194
:10D3E800DFED558A9FED55AADFED43BADFED549A7C
:10D3F8009FED54BADFED54AA544F554E0193B4EE45
:10D40800E7CAF1EE10FA88BFB0EE67CA2546514B5D
:10D4180098ED008A2344D3ED007AF5EE407AF1EED8
:10D4280010FA17D04C4B234493ED007A78EE476AF4
:10D43800B0EEE66AF4EEC67AF1EE10FA08D5F5EE2B
:10D44800C06AF1EE10FACCBF37EE878A37EE678AEA
:10D4580083ED008A414B1A88930739D0022D37D0C3
:10D4680099F82E103E4B07EE901A234493ED007A5C
:10D478004B42F8EEE76A07EE903A26EE877AF8EE26
:10D48800E77AB4EEE77AF1EE10FA0AD407EE901ACA
:10D49800F8EE677AF4EEC77AF1EE10FA88BFF0EE8C
:10D4A800477A304B304903EB450331F91500B3F99E
:10D4B8000C30C01A07EE100AB8EEC77AD007E7EEAC
:10D4C800687A40F16E87294B93ED008A27EE888AA7
:10D4D800029B9BF864212344D3ED01DA38EE6DDA20
:10D4E800002A00F08680224BDBF8682146E000BF66
:10D4F800524200207044002000000000C02200209A
:10D508005442002050420020884400202474002007
:10D518009324499249420020EC5F00202C6C0020A3
:10D5280020740020146C00209C720020805400207D
:10D53800286C0020A4380020CDCCCC3DAE47813FDC
:10D548000000C84200003443610BB63BBC380020E1
:10D55800B03800209072002000240020FC3D0020FC
:10D568000C240020F4450020045500207872002087
:10D57800A4720020F42300208471002003991B6802
:10D588008A1A9A4235DD99F84830022B02F07482E3
:10D59800022D04F0AE82D34B1B68990741F1F1804C
:10D5A800D14BD249DFF8C0E331F915C09EED008AAE
:10D5B800DFF8B8E3C6ED00BA03EB450028EE288A89
:10D5C800B0F90C00A0EB0C0007EE900AF8EEE77A31
:10D5D800DEF8000027EE888A904238EE6DDAC1F254
:10D5E8001283F7EE007AB4EEE79AF1EE10FA01F141
:10D5F800E182BF4B234493ED000A019B2CEE800A85
:10D60800022D20EE0D0AA3EC010A019304F0148206
:10D61800B84B9AED007AD3ED007AB74BD6ED006A95
:10D6280093ED006AB54B67EE277A234427EE8C7A90
:10D63800D3ED007A67EE277AF0EE665AEDEE275AB8
:10D64800B1EE467AF4EEC75AF1EE10FA08D4F4EEC9
:10D65800C65AF1EE10FA8CBFB0EE467AB0EE657A93
:10D668009BED4C6AF7EE007AB4EEE76AF1EE10FA39
:10D67800ACBF0123002343B1F0EEE66AF0EEC77AAF
:10D68800F4EEE67AF1EE10FA01D586ED007A022D75
:10D6980004F0CB819A4A9B4B52F825001B68B0EEE8
:10D6A8006D0A9847984A994B52F825001B68984785
:10D6B80099F8373023B1964B1B88002B00F0F3867E
:10D6C800B0EE6B8A934B9AED007A38EE400A234409
:10D6D80093ED008A83ED000A99F8483030EE480A45
:10D6E800C0EE077A2BB38C4B1B78D80721D5B7EE41
:10D6F800007AB4EEC79AF1EE10FA04DB9BF86431B5
:10D70800002B01F01681DBF86831039AD31A834A9B
:10D7180012689A420DDD824B93ED007AB0EECDDAB5
:10D72800B4EEC7DAF1EE10FA41F1898200238BF8E2
:10D7380064317C4B9BF87421234493ED007A2CEEE2
:10D74800877A67EE277AC7ED007A32B9019BC6ED72
:10D7580000BA43ED01BAC7ED00BA0135032D08F14F
:10D76800040807F1040706F1040604F104047FF431
:10D778004EAE6D4B1B78072B01F0EC86012B02F0A7
:10D788004C81002302939BF87C31002B40F0CC861F
:10D79800664B1A46664B10681B6810F4805E93F857
:10D7A8002C3041F02F80634A634992ED006A498B1F
:10D7B800624A8BED636A92ED007A614A8BED647A76
:10D7C80007EE901AF8EEE76AD2ED037A5D4A8BED20
:10D7D800616A37EE467A77EEE67AD2ED006A8BED2B
:10D7E800607A01228BF89421C7EEA65A5649574A07
:10D7F80091ED005A56499FED576A91ED004A5649F6
:10D80800DFED566AD1ED004A92ED007A35EE045A02
:10D81800F7EE007AF4EEE75A35EE245AF1EE10FAF4
:10D8280088BFF0EE675A25EE065AF4EEE65AB1EED6
:10D83800476AF1EE10FAB4EEC65AB8BFF0EE665A6F
:10D84800F1EE10FACBED665A01F13F84B4EEC75AF7
:10D85800F1EE10FA88BFB0EE475A3B4ADFED3D6A59
:10D86800D2ED017A3A4A92ED014A3B4A77EE847A40
:10D87800D2ED014A77EEA47A67EEA67AB4EEE76AAB
:10D88800F1EE10FA08DCB4EEE77AF1EE10FA8CBF8C
:10D89800B0EE676AB0EE476A2B4ADFED2E6AD2ED2A
:10D8A800027A2B4AD2ED024A2D4A77EEA47A92EDFB
:10D8B800007A67EEA67AF1EE473AF4EEE37AF1EEF3
:10D8C80010FA08D4F4EEC77AF1EE10FA8CBFF0EE35
:10D8D800473AF0EE673A234A5278002A48D1F1EEE7
:10D8E800633A45E0A8540020F44500200455002080
:10D8F8004C7200202C000020C072002058720020BA
:10D908008C71002088710020E0710020DC710020FB
:10D91800FC3D00202C24002035560020A472002055
:10D92800B07200206472002020740020386C00203F
:10D938008054002068390020AC6D00200038002099
:10D948002075002014380020A4380020C47200205C
:10D95800B03800206F12833ABC3800200000000065
:10D96800C8720020303B002078720020A07200208E
:10D97800002B41F00B86B7EE004ADFF89CA39AF81B
:10D988000020002A03F08581E14CDFEDE27AD4ED36
:10D99800024AD4ED016A94ED037A66EE244AE5EE74
:10D9A800264AE3EE874A64EE244AF4EEE74AF1EEAB
:10D9B80010FAB4BFB0EE677AB0EE647A98BFF0EEB2
:10D9C800647A012ACDED0A4A03F07C8194ED063A87
:10D9D800D4ED052AD4ED076A26EE033AA5EE223ADD
:10D9E800A3EEA63A24EE033AB4EEE73AF1EE10FAC3
:10D9F800B4EEC73A8CBFF0EE676AF0EE436AF1EE18
:10DA080010FA88BFF0EE676AB4BFF0EE477AF0EE1E
:10DA1800437A022A8DED0B3A00F0808194ED0A7A60
:10DA2800D4ED092A94ED0B3A26EE077AA5EE227A70
:10DA3800A3EE837A24EE077AB4EEE67AF1EE10FAD2
:10DA4800B4EEE77A8CBFB0EE663AB0EE473AF1EE44
:10DA580010FA8DED0C7A98BFF0EE436AB8BFB0EEBD
:10DA6800677A032A01F0C983D4ED0E7AD4ED0D2A22
:10DA780094ED0F3A66EE277AE5EE227AE3EE837AA2
:10DA880064EE277AF4EEE67AF1EE10FAF4EEC77A4D
:10DA98008CBFB0EE663AB0EE673AF1EE10FACDED13
:10DAA8000D7A98BFF0EE436AB8BFF0EE477A042AC1
:10DAB80000F0348194ED127AD4ED112A94ED133AE2
:10DAC80026EE077AA5EE227AA3EE837A24EE077A69
:10DAD800B4EEE67AF1EE10FAB4EEE77A8CBFB0EE67
:10DAE800663AB0EE473AF1EE10FA8DED0E7A98BF2D
:10DAF800F0EE436AB8BFB0EE677A052A01F07D837D
:10DB0800D4ED167AD4ED152A94ED173A66EE277AF5
:10DB1800E5EE227AE3EE837A64EE277AF4EEE67A8B
:10DB2800F1EE10FAF4EEC77A8CBFB0EE663AB0EEBA
:10DB3800673AF1EE10FACDED0F7A98BFF0EE436A2E
:10DB4800B8BFF0EE477A062A00F0E88094ED1A7A1A
:10DB5800D4ED192A94ED1B3A26EE077AA5EE227A1F
:10DB6800A3EE837A24EE077AB4EEE67AF1EE10FAA1
:10DB7800B4EEE77A8CBFB0EE663AB0EE473AF1EE13
:10DB880010FA8DED107A98BFF0EE436AB8BFB0EE88
:10DB9800677A072A01F03183D4ED1E7AD4ED1D2A65
:10DBA80094ED1F3A66EE277AE5EE227AE3EE837A61
:10DBB80064EE277AF4EEE67AF1EE10FAF4EEC77A1C
:10DBC8008CBFB0EE663AB0EE673AF1EE10FACDEDE2
:10DBD800117A98BFF0EE436AB8BFF0EE477A082A88
:10DBE80000F09C8094ED227AD4ED212A94ED233A1A
:10DBF80026EE077AA5EE227AA3EE837A24EE077A38
:10DC0800B4EEE67AF1EE10FAB4EEE77A8CBFB0EE35
:10DC1800663AB0EE473AF1EE10FA8DED127A98BFF7
:10DC2800F0EE436AB8BFB0EE677A092A01F0E582E0
:10DC3800D4ED267AD4ED252A94ED273A66EE277A94
:10DC4800E5EE227AE3EE837A64EE277AF4EEE67A5A
:10DC5800F1EE10FAF4EEC77A8CBFB0EE663AB0EE89
:10DC6800673AF1EE10FACDED137A98BFF0EE436AF9
:10DC7800B8BFF0EE477A0A2A50D094ED2A7AD4ED4C
:10DC8800292A94ED2B3A26EE077AA5EE227AA3EEFE
:10DC9800837A24EE077AB4EEE67AF1EE10FAB4EE5F
:10DCA800E77A8CBFB0EE663AB0EE473AF1EE10FA7A
:10DCB8008DED147A98BFF0EE436AB8BFB0EE677A7C
:10DCC8000B2A01F09A82D4ED2E7AD4ED2D2A94ED08
:10DCD8002F3A66EE277AE5EE227AE3EE237A67EEAC
:10DCE800847AF4EEE67AF1EE10FAF4EEC77A8CBF95
:10DCF800B0EE666AB0EE676AF1EE10FACDED157A0D
:10DD080098BFF0EE466AB8BFF0EE477A06E000BF6B
:10DD180040370020000000000174002077EEE67A0A
:10DD2800F7EE006AF4EEE67AF1EE10FACBED4C7AF3
:10DD380043F3608286EEA77A022ADDED0B7A64EE61
:10DD4800874A67EE877ACDED0A4ACDED0B7A4DD03A
:10DD5800DDED0C7A67EE877A032ACDED0C7A45D093
:10DD6800DDED0D7A67EE877A042ACDED0D7A3DD088
:10DD7800DDED0E7A67EE877A052ACDED0E7A35D07D
:10DD8800DDED0F7A67EE877A062ACDED0F7A2DD072
:10DD9800DDED107A67EE877A072ACDED107A25D067
:10DDA800DDED117A67EE877A082ACDED117A1DD05C
:10DDB800DDED127A67EE877A092ACDED127A15D051
:10DDC800DDED137A67EE877A0A2ACDED137A0DD046
:10DDD800DDED147A67EE877A0B2ACDED147A05D03B
:10DDE800DDED157A27EE877A8DED157AE54B1C68FF
:10DDF80014F0805401F00982F6EE005ACBED665A11
:10DE0800002A02F04087E04B9BF99411DD78DBEDA6
:10DE1800644ADE4B9BED636ADFF88CC3DC4EDD4F52
:10DE28009CED005A3F78B6F906C0DBED606ADBED81
:10DE3800617A07EE101AFDEEE44A1978D64BB3F86A
:10DE48001A8014EE903AFDEEC64A01F0010900F07E
:10DE58001006B8EEC77A14EE901A00F48000002D70
:10DE680041F0CE83002E41F0DD81CC4C9DED0A5A65
:10DE780094ED006ACA4825EE866AA5EE076AB0EEF8
:10DE8800675AA6EE265ABDEEC56A16EE106A16EE59
:10DE9800105A9E42A8BF1D46B142C8BF0D4606EEA5
:10DEA800105AB8EEC66A012A80ED006A00F0608157
:10DEB80094ED046A9DED0B5A25EE866AA5EE076A75
:10DEC800B0EE675AA6EE265ABDEEC56A16EE106A7F
:10DED80016EE105A9E42A8BF1D46B142C8BF0D4655
:10DEE80006EE105AB8EEC66A022A80ED016A00F002
:10DEF8003F8194ED086A9DED0C5A25EE866AA5EEE1
:10DF0800076AB0EE675AA6EE265ABDEEC56A16EE47
:10DF1800106A16EE105A9E42A8BF1D46B142C8BFED
:10DF28000D4606EE105AB8EEC66A032A80ED026A5C
:10DF380000F01E8194ED0C6A9DED0D5A25EE866A5F
:10DF4800A5EE076AB0EE675AA6EE265ABDEEC56A78
:10DF580016EE106A16EE105A9E42A8BF1D46B14230
:10DF6800C8BF0D4606EE105AB8EEC66A042A80ED00
:10DF7800036A00F0FD8094ED106A9DED0E5A25EEBF
:10DF8800866AA5EE076AB0EE675AA6EE265ABDEE77
:10DF9800C56A16EE106A16EE105A9E42A8BF1D46B4
:10DFA800B142C8BF0D4606EE105AB8EEC66A052A39
:10DFB80080ED046A00F0DC8094ED146A9DED0F5A40
:10DFC80025EE866AA5EE076AB0EE675AA6EE265ACF
:10DFD800BDEEC56A16EE106A16EE105A9E42A8BF2C
:10DFE8001D46B142C8BF0D4606EE105AB8EEC66AC5
:10DFF800062A80ED056A00F0BB8094ED186A9DED55
:10E00800105A25EE866AA5EE076AB0EE675AA6EEA4
:10E01800265ABDEEC56A16EE106A16EE105A9E42D2
:10E02800A8BF1D46B142C8BF0D4606EE105AB8EE4D
:10E03800C66A072A80ED066A00F09A8094ED1C6A89
:10E048009DED115A25EE866AA5EE076AB0EE675A6D
:10E05800A6EE265ABDEEC56A16EE106A16EE105ADE
:10E068009E42A8BF1D46B142C8BF0D4606EE105AD3
:10E07800B8EEC66A082A80ED076A79D094ED206A5E
:10E088009DED125A25EE866AA5EE076AB0EE675A2C
:10E09800A6EE265ABDEEC56A16EE106A16EE105A9E
:10E0A8009E42A8BF1D46B142C8BF0D4606EE105A93
:10E0B800B8EEC66A092A80ED086A59D094ED246A38
:10E0C8009DED135A25EE866AA5EE076AB0EE675AEB
:10E0D800A6EE265ABDEEC56A16EE106A16EE105A5E
:10E0E8009E42A8BF1D46B142C8BF0D4606EE105A53
:10E0F800B8EEC66A0A2A80ED096A39D094ED286A12
:10E108009DED145A25EE866AA5EE076AB0EE675AA9
:10E11800A6EE265ABDEEC56A16EE106A16EE105A1D
:10E128009E42A8BF1D46B142C8BF0D4606EE105A12
:10E13800B8EEC66A0B2A80ED0A6A19D094ED2C6AEB
:10E148009DED155A65EE865AE7EE055AE6EEA57A74
:10E15800FDEEE77A17EE904AA342A8BF2346A142F4
:10E16800C8BF0B4607EE903AF8EEE77AC0ED0B7A97
:10E17800B9F1000F00F0A4870A4B1B68002B40F090
:10E18800128413E044390020A43D002035560020B5
:10E198004C530020A8670020AC6D002040370020B9
:10E1A800043900207C7100200C370020CB4B1B78F1
:10E1B80093B19AF8000060B1C94DCA4E0024E0B28C
:10E1C8003368B5EC010A98479AF800000134844294
:10E1D800F5DBC54B1B689847C44B1B78072B01F030
:10E1E800B18101238BF8003117B0BDEC0C8BBDE871
:10E1F800F08FBF4B1B78013BDBB2FFF7D0B8BD49AE
:10E20800BD4B91F80180B94902930E781B68BB4F4A
:10E218004FF47A71B1FBF3F3C3EB431403EB8403BC
:10E22800DC00A4B2A542B7F9060002F0C182DAF810
:10E238008810BAF93CE0DAF86C304A1C07EE90EA2C
:10E248007344012ACAF88820CAF86C30F8EEE77AD5
:10E2580002F0BB82DAED1E5ADAED206A07EE102AC8
:10E2680037EEE56AB8EEC75A012D86EE057A37EE25
:10E27800257A77EEC77A8AED1F7AE7EE866A8AED05
:10E288001E7AF0EE667ACAED216ACAED206A02F0BB
:10E298003585DAF89C10BAF93EE0DAF870304A1C95
:10E2A80007EE90EA7344012ACAF89C20CAF8703035
:10E2B800F8EEE77A02F0A482DAED235ADAED256A5D
:10E2C80007EE102A37EEE56AB8EEC75A012D86EE3A
:10E2D800057A37EE257A77EEC77A8AED247AE7EE63
:10E2E800866A8AED237AF0EE667ACAED266ACAED66
:10E2F800256A02F02C85DAF8B010BAF940E0DAF8AD
:10E3080074304A1C07EE90EA7344012ACAF8B02018
:10E31800CAF87430F8EEE77A02F08D82DAED285AFE
:10E32800DAED2A6A07EE102A37EEE56AB8EEC75A20
:10E33800012D86EE057A37EE257A77EEC77A8AEDD3
:10E34800297AE6EE276A8AED287AF0EE667ACAED2F
:10E358002B6ACAED2A6A02F02385F880BAF8B4302D
:10E36800624A013B1678AAF8B43002990023072EB6
:10E378004B608B60CB607FF406A8F8F751FE5F4FC7
:10E388009BF828310493A0EB09003880002B3FF458
:10E3980000A8013B8BF8283117B0BDEC0C8BBDE809
:10E3A800F08F9BED567AB1F90000DBED576AB1F9B1
:10E3B80002E0534AF4EEC76A80EAE0738EEAEE712F
:10E3C800A3EBE073F1EE10FAA1EBEE71B8BFF0EE3B
:10E3D800476A8B42B8BF0B4607EE103A1378B8EE7F
:10E3E800C77A27EE287A002B40F07482454B93EDCC
:10E3F800006AB4EECA6AF1EE10FA41F10483F7EE4E
:10E40800005A75EEC65A3BEE477A65EEAA5A3E4B5D
:10E41800A7EE256A93ED007A26EE076AB5EEC06A84
:10E42800F1EE10FA40F2ED86C9EE865AB7EE007AA0
:10E43800B0EE476AA6EEE56AF0EE466AF4EEC76A01
:10E44800F1EE10FA88BFF0EE476AF5EEC06AF1EE19
:10E4580010FAB8BFF0EE6B6A2C4B93ED007A67EEBA
:10E46800877AA7EEA68AFFF733B8294BDFF8B4B04E
:10E478001968284A214F9BF80031C96912883980E8
:10E488007A80002B3EF405AE07F006FF00238BF8D8
:10E498000031164B1B78072B7EF4FBADF8F7C0FD57
:10E4A8008146FEF7F8BD1C4B1C4A234493ED007AC5
:10E4B800D2ED007A1A4B67EE277AF7EE006AF4EE8F
:10E4C800E67AF1EE10FA93ED007A88BFF0EE667AFC
:10E4D80067EE877A27EE888AFFF7F4B8106C002079
:10E4E800043900209C670020A467002020740020C5
:10E4F80048720020146C0020286C0020247400202E
:10E50800847200208C720020807200207C720020AF
:10E518004040002078330020182400207472002026
:10E5280070720020C0220020D84BDFF8A4A31B780B
:10E53800D90740F129829AF80030002B3FF41CAE2D
:10E54800DBED573A9BED564ADBED617AD04A9BEDFD
:10E55800606A92ED007ADBED544A9BED535ACD4C3C
:10E56800CD48F4EEC43AF3EE045AF1EE10FA77EE21
:10E57800A56A01F1928294ED025A25EE645AB0EE32
:10E58800674AA5EE064AB4EEE64A34EE655AF1EE5D
:10E5980010FA48BFB0EE475A012B80ED005A3FF4FD
:10E5A800EBAD94ED065A25EE645AB0EE674AA5EE37
:10E5B800064AB4EEE64A34EE655AF1EE10FA48BF60
:10E5C800B0EE475A022B80ED015A3FF4D5AD94EDD9
:10E5D8000A5A25EE645AB0EE674AA5EE064AB4EE2A
:10E5E800E64A34EE655AF1EE10FA48BFB0EE475AE3
:10E5F800032B80ED025A3FF4BFAD94ED0E5A25EE81
:10E60800645AB0EE674AA5EE064AB4EEE64A34EE1E
:10E61800655AF1EE10FA48BFB0EE475A042B80ED68
:10E62800035A3FF4A9AD94ED125A25EE645AB0EEA0
:10E63800674AA5EE064AB4EEE64A34EE655AF1EEAC
:10E6480010FA48BFB0EE475A052B80ED045A3FF444
:10E6580093AD94ED165A25EE645AB0EE674AA5EECE
:10E66800064AB4EEE64A74EE655AF1EE10FA48BF6F
:10E67800F0EE475A062BC0ED055A3FF47DADD4EDB8
:10E688001A5A65EEE45AB0EE674AA5EE864AB3EE2A
:10E69800045AB4EEE64A74EE455AF1EE10FA48BF51
:10E6A800F0EE475A072BC0ED065A3FF465ADD4ED9E
:10E6B8001E5A65EEE45AB0EE674AA5EE864AB4EEF5
:10E6C800E64A74EE455AF1EE10FA48BFF0EE475AA2
:10E6D800082BC0ED075A3FF44FADD4ED225A65EE32
:10E6E800E45AB0EE674AA5EE864AB4EEE64A74EEFE
:10E6F800455AF1EE10FA48BFF0EE475A092BC0ED23
:10E70800085A3FF439ADD4ED265A65EEE45AB0EE16
:10E71800674AA5EE864AB4EEE64A74EE455AF1EE2B
:10E7280010FA48BFF0EE475A0A2BC0ED095A3FF4D9
:10E7380023ADD4ED2A5A65EEE45AB0EE674AA5EE49
:10E74800864AB4EEE64A74EE455AF1EE10FA48BF2E
:10E75800F0EE475A0B2BC0ED0A5A3FF40DADD4ED3D
:10E768002E5A65EEE44AE4EE867AF4EEE76A77EE2E
:10E77800C57AF1EE10FAC8BFF0EE477AC0ED0B7A11
:10E78800FAE4464BC6ED00BA1B689342BEF629AFC1
:10E79800434B1A8800238BF86431002A41F0FE8726
:10E7A800404A414B1178186881F00101F4F770F87C
:10E7B800FEF71FBF3D4D3E4F05F5F47405F5157680
:10E7C800F5EC017A9AED080ADAF81432F8EEE77AED
:10E7D800204627EE800A9847A4F1E000DAF83431A1
:10E7E8009847A4F17000DAF8A4319847D5F8F400F6
:10E7F800DAF8B83098472434A642A7EC010ADFD1EA
:10E80800FEF7BCBD214A1278D20703D4294A128BDD
:10E81800ABF88821284A2949128891ED037A07EE36
:10E82800902AF8EEE77AB4EEE77AF1EE10FA41F2C0
:10E838003B822349098807EE901AF8EEE77AB4EE8E
:10E84800E77AF1EE10FAC1F2F8801E491E4AD1EDBE
:10E85800006A92ED006A1D49CBED636ABCEEC75AA7
:10E8680076EE665A15EE102ACBED616ACBED605A4A
:10E878008BED646AABF888210122D1ED006A8BF830
:10E88800942177EE677AFEF7AFBF00BF35560020B8
:10E898000C3700204037002004390020A0720020E7
:10E8A800405700204257002044570020EC5F0020CA
:10E8B8002C6C0020AC6D002018380020207500203A
:10E8C8001A380020043800200038002020380020A2
:10E8D80001740020A64B93ED005AB5EEC05AF1EE34
:10E8E80010FA40F38E84A34BD3ED004AF5EEC04AEC
:10E8F800F1EE10FA40F3858434EEC77A66EEE95AF1
:10E9080087EE246AC5EE856AB7EE007AB4EEC76A68
:10E91800F1EE10FA88BFB0EE476AB5EEC06AF1EEC4
:10E9280010FA76EE876AB8BFB0EE6B6A66EE266AB2
:10E9380084E5914A92ED007AF0EEE76AF4EEC76A50
:10E94800F1EE10FA7EF7DFAE8C4A92ED007AF0EE27
:10E95800CD6AF4EEC76AF1EE10FA7EF7D4AE884AB3
:10E9680098ED007AD2ED006AB0EEC77AB4EEE67A96
:10E97800F1EE10FA7EF5C7AE01220399CBF86811C3
:10E988008BF86421FEF7C3BE9AF80020002A3FF4F2
:10E99800F3AB92007B497C4822F078FE7B4B1B68E6
:10E9A800002B3FF403AC7A4B1B78192B07D80121B5
:10E9B800784A01FA03F31A40002A42F0FD81764BA7
:10E9C800764D774E01931B689C061BD5F37AFF2B77
:10E9D80004D0744A12789A4201F24984B6F9087050
:10E9E800F37D2F80FF2B04D06E4A12789A4201F2F1
:10E9F8003984B6F914406C80082014F0A7FB00286D
:10EA080041F07981B6F90600B5F900E0B5F9027070
:10EA1800B6F91210B6F91E20B5F90440B6F904305B
:10EA2800B5F906C07045A8BF7046B942A8BF3946B7
:10EA3800A242A8BF22469E45A8BF03462B80B6F92E
:10EA48001030B5F908009F42B8BF1946B6F92A3008
:10EA58006980B6F91C10B6F934706345A8BF6346DF
:10EA68008C42B4BF0C461446B6F93620AC80B6F9D1
:10EA78002840B5F90A108242A8BF0246A445ACBF97
:10EA88009C46A446B6F94230B5F90C40A5F806C034
:10EA98008B42A8BF0B46B842ACBF10463846B6F901
:10EAA8004E202881B6F94000B5F90E70A242A8BFE1
:10EAB80022468842C8BF0346B6F95A00B6F94C1038
:10EAC8006B81B842B6F95830374EA8BF38469F42D6
:10EAD800A8BF0346A142D8BF1146A981EB81B389DB
:10EAE80023B3324FDFF8C890DFF8B48007F1100481
:10EAF800B7F9023000EE103A4846B8EEC00AF1F70E
:10EB080095FD22F037FFB8F90430B8F9062000B2B5
:10EB1800984209F1240908F10C0803DB82421346E4
:10EB2800A8BF034627F8023FA742E1D1184B1B783C
:10EB3800013B182B00F22A83DFE813F016032803A1
:10EB48002803CB02280328032803C10B2803280322
:10EB5800280328032803B00B2803280328032803C5
:10EB68002803CB02CF0B28032803B00B160300BFE2
:10EB78008072002088720020B4720020B0720020D9
:10EB8800B872002010370020043900207C71002062
:10EB98008071002032413003386C0020F4380020A6
:10EBA800307300202C550020D0620020F23800205D
:10EBB800786F002002996F4BD1ED017A93ED007ABE
:10EBC800F0EEE77AF4EEC77AF1EE10FA7EF511ADC1
:10EBD800D1ED027AF0EEE77AB4EEE77AF1EE10FAC8
:10EBE8007EF707ADD1ED037AF0EEE77AB4EEE77A77
:10EBF800F1EE10FA7EF7FDAC5F4B1B689B077FF5C3
:10EC0800C7AD5E495E4BB3F90C20B1F900E05D4831
:10EC1800AEEB020E00688EEAEE72A2EBEE72824252
:10EC2800BEF6E7ACB3F90E30B1F90220D21A82EA87
:10EC3800E273A3EBE27398427EF7DBACA8E5524B94
:10EC480098ED007AD3ED006AB0EEC77AB4EEE67AB2
:10EC5800F1EE10FA7EF76DADFEF768BD07EE103ADB
:10EC68004A4B4B4F1B78CBF81051B8EEC77AF7EEEA
:10EC7800006A132B86EE879AB7F90400BBF8144193
:10EC88009AED080A01F01685424B434A93ED001AA3
:10EC980093ED053A93ED122A93ED176AD3ED091A0D
:10ECA80093ED0E4AD3ED015AD3ED063A93ED0A7A65
:10ECB80093ED0F5AD3ED132AD3ED186AD3ED044A16
:10ECC800D3ED030A67EE897A69EE288A29EE088A65
:10ECD800A1EE273A02EB84050021A2EE286ACBF8C0
:10ECE8000411CBF80811A1EE884AE5EEA73AA7EE81
:10ECF800085A93ED167AD3ED0D5A93ED021AD3ED17
:10ED08000C1A85ED003AE2EEA86A64EEC34A27EED3
:10ED1800467A93ED0B2AD3ED152A85ED204AE0EECD
:10ED2800C33A65EEC45A93ED143AC3ED053AE1EEE1
:10ED3800274AF0EE477AA1EEC45AE2EE085AE2EE0C
:10ED4800C66AE3EE287AC3ED064A83ED0E5AC3ED90
:10ED58000F5A85ED406AC3ED176AC3ED187ACBF8F0
:10ED68000C11631C03F01F03ABF81431B880FEF7D5
:10ED7800EDB900BFAC720020A85400200455002053
:10ED8800F4450020A8720020B872002020740020EA
:10ED980024740020F444002070420020B9F1000FD0
:10EDA80041F09085E24C002F42F0668294ED006AB3
:10EDB800DDED0A4ADF4825EE866ABDEEC55AA4EEA7
:10EDC800876A15EE101AB0EE675AA6EE265ABDEEFF
:10EDD800C56A16EE106A16EE105A9E42A8BF1D4666
:10EDE800B142C8BF0D4606EE105AB8EEC66A012AEF
:10EDF80080ED006A3FF4CDAD94ED046A9DED0B5AA9
:10EE080025EE866AA5EE076AB0EE675AA6EE265A80
:10EE1800BDEEC56A16EE106A16EE105A9E42A8BFDD
:10EE28001D468E42B8BF0D4606EE105AB8EEC66AA9
:10EE3800022A80ED016A3FF4ACAD94ED086A9DEDBD
:10EE48000C5A25EE866AA5EE076AB0EE675AA6EE5A
:10EE5800265ABDEEC56A16EE106A16EE105A9E4284
:10EE6800A8BF1D468E42B8BF0D4606EE105AB8EE32
:10EE7800C66A032A80ED026A3FF48BAD94ED0C6AF2
:10EE88009DED0D5A25EE866AA5EE076AB0EE675A23
:10EE9800A6EE265ABDEEC56A16EE106A16EE105A90
:10EEA8009E42A8BF1D468E42B8BF0D4606EE105AB8
:10EEB800B8EEC66A042A80ED036A3FF46AAD94EDA1
:10EEC800106A9DED0E5A25EE866AA5EE076AB0EE29
:10EED800675AA6EE265ABDEEC56A16EE106A16EEF9
:10EEE800105A9E42A8BF1D468E42B8BF0D4606EE78
:10EEF800105AB8EEC66A052A80ED046A3FF449AD97
:10EF080094ED146A9DED0F5A25EE866AA5EE076A00
:10EF1800B0EE675AA6EE265ABDEEC56A16EE106A1E
:10EF280016EE105A9E42A8BF1D468E42B8BF0D4627
:10EF380006EE105AB8EEC66A062A80ED056A3FF456
:10EF480028AD94ED186A9DED105A25EE866AA5EE57
:10EF5800076AB0EE675AA6EE265ABDEEC56A16EEE7
:10EF6800106A16EE105A9E42A8BF1D468E42B8BFC0
:10EF78000D4606EE105AB8EEC66A072A80ED066AF4
:10EF88003FF407AD94ED1C6A9DED115A25EE866A93
:10EF9800A5EE076AB0EE675AA6EE265ABDEEC56A18
:10EFA80016EE106A16EE105A9E42A8BF1D468E42F3
:10EFB800B8BF0D4606EE105AB8EEC66A082A80EDAC
:10EFC800076A3FF4E6AC94ED206A9DED125A25EEEF
:10EFD800866AA5EE076AB0EE675AA6EE265ABDEE17
:10EFE800C56A16EE106A16EE105A9E42A8BF1D4654
:10EFF8008E42B8BF0D4606EE105AB8EEC66A092A08
:10F0080080ED086A3FF4C5AC94ED246A9DED135A6F
:10F0180025EE866AA5EE076AB0EE675AA6EE265A6E
:10F02800BDEEC56A16EE106A16EE105A9E42A8BFCB
:10F038001D468E42B8BF0D4606EE105AB8EEC66A97
:10F048000A2A80ED096A3FF4A4AC94ED286A9DED84
:10F05800145A25EE866AA5EE076AB0EE675AA6EE40
:10F06800265ABDEEC56A16EE106A16EE105A9E4272
:10F07800A8BF1D468E42B8BF0D4606EE105AB8EE20
:10F08800C66A0B2A80ED0A6A3FF483AC94ED2C6AB9
:10F098009DED155A65EE865AE7EE055AE6EEA57A15
:10F0A800FDEEE77A17EE904AA342A8BF2346A14295
:10F0B800D8BF194607EE901AF8EEE77AC0ED0B7A3A
:10F0C800002A7FF466ACFFF757B8B0EE465AFEF751
:10F0D800C4BB194BB5F908101A6802B111609B69D5
:10F0E800B5F90A2003B11A60019B1B689A0602F160
:10F0F800748002220492D9027FF558A8F57B112D5D
:10F108003FF654A80D4BDDF810801F4633F9153033
:10F1180000EE103A4046B8EEC00A6C1C05F10E0627
:10F1280003F038FF4346E4B25D1BF6B2B84608E088
:10F138004037002004390020E06200204C530020B2
:10F148003C46671C6019122CFFB2C0B23FF42EA8CF
:10F1580038F9143000EE103AB8EEC00A03F01AFF7E
:10F16800B742EDD1FFF722B8B37B002B42F06C8297
:10F17800284B1B7813F0010342F06682264A126876
:10F18800002A02F03B84136001230493019B1B684F
:10F19800980603D4214A1278052AACD1049A13465A
:10F1A8000233541CDBB21046E4B20493B5F90030C4
:10F1B80000EE103AB8EEC00A03F0ECFEB5F90230E2
:10F1C80000EE103A2046B8EEC00A03F0E3FE019BB9
:10F1D8001B6890E722F0CEFB28F81500FEF7BCB8B4
:10F1E80094ED007A0AEB4502B8EEC78A928F28F8A8
:10F1F800152028EE278AFEF78DB8F0EE477AFEF73D
:10F208008DBDDFED076AFFF727B947023EF5F4AD7C
:10F21800FEF7F6BD35560020E06200208071002020
:10F2280000000000B9F1000F41F0A083D34C9DED20
:10F238000A5A94ED006AD24825EE866AA5EE076A56
:10F24800B0EE675AA6EE265ABDEEC56A16EE106AEB
:10F2580016EE105A9E42A8BF1D46B142C8BF0D46C1
:10F2680006EE105AB8EEC66A012A80ED006A3FF42D
:10F2780090AB94ED046A9DED0B5A25EE866AA5EED7
:10F28800076AB0EE675AA6EE265ABDEEC56A16EEB4
:10F29800106A16EE105A9E42A8BF1D46B142C8BF5A
:10F2A8000D4606EE105AB8EEC66A022A80ED016ACB
:10F2B8003FF46FAB94ED086A9DED0C5A25EE866A13
:10F2C800A5EE076AB0EE675AA6EE265ABDEEC56AE5
:10F2D80016EE106A16EE105A9E42A8BF1D46B1429D
:10F2E800C8BF0D4606EE105AB8EEC66A032A80ED6E
:10F2F800026A3FF44EAB94ED0C6A9DED0D5A25EE73
:10F30800866AA5EE076AB0EE675AA6EE265ABDEEE3
:10F31800C56A16EE106A16EE105A9E42A8BF1D4620
:10F32800B142C8BF0D4606EE105AB8EEC66A042AA6
:10F3380080ED036A3FF42DAB94ED106A9DED0E5AF3
:10F3480025EE866AA5EE076AB0EE675AA6EE265A3B
:10F35800BDEEC56A16EE106A16EE105A9E42A8BF98
:10F368001D46B142C8BF0D4606EE105AB8EEC66A31
:10F37800052A80ED046A3FF40CAB94ED146A9DED08
:10F388000F5A25EE866AA5EE076AB0EE675AA6EE12
:10F39800265ABDEEC56A16EE106A16EE105A9E423F
:10F3A800A8BF1D46B142C8BF0D4606EE105AB8EEBA
:10F3B800C66A062A80ED056A3FF4EBAA94ED186A3E
:10F3C8009DED105A25EE866AA5EE076AB0EE675ADB
:10F3D800A6EE265ABDEEC56A16EE106A16EE105A4B
:10F3E8009E42A8BF1D46B142C8BF0D4606EE105A40
:10F3F800B8EEC66A072A80ED066A3FF4CAAA94EDF9
:10F408001C6A9DED115A25EE866AA5EE076AB0EED4
:10F41800675AA6EE265ABDEEC56A16EE106A16EEB3
:10F42800105A9E42A8BF1D46B142C8BF0D4606EEFF
:10F43800105AB8EEC66A082A80ED076A3FF4A9AAEE
:10F4480094ED206A9DED125A25EE866AA5EE076AAC
:10F45800B0EE675AA6EE265ABDEEC56A16EE106AD9
:10F4680016EE105A9E42A8BF1D46B142C8BF0D46AF
:10F4780006EE105AB8EEC66A092A80ED086A3FF40B
:10F4880088AA94ED246A9DED135A25EE866AA5EEA6
:10F49800076AB0EE675AA6EE265ABDEEC56A16EEA2
:10F4A800106A16EE105A9E42A8BF1D46B142C8BF48
:10F4B8000D4606EE105AB8EEC66A0A2A80ED096AA9
:10F4C8003FF467AA94ED286A9DED145A25EE866AE2
:10F4D800A5EE076AB0EE675AA6EE265ABDEEC56AD3
:10F4E80016EE106A16EE105A9E42A8BF1D46B1428B
:10F4F800C8BF0D4606EE105AB8EEC66A0B2A80ED54
:10F508000A6A3FF446AA94ED2C6A9DED155A65EEF9
:10F51800865AE7EE055AE6EEA57AFDEEE77A17EE8B
:10F52800904AA342A8BF2346A142C8BF0B4607EE94
:10F53800903AF8EEE77AC0ED0B7A002A7FF429AA10
:10F54800FEF71ABEF7F76CFD029A0E4B801AD880A8
:10F55800FEF747BEF7F764FD0B4B059A1B78094F7A
:10F56800801A012B788000F05982072B7EF409A9B4
:10F57800F7F756FD0290FEF706B900BF40370020A6
:10F58800043900202474002020740020184B5A7974
:10F59800002A3EF4F0A9174A1278002A3EF4EBA993
:10F5A8001B78DFED154A07EE903A144BB8EE677AF0
:10F5B8001B8807EE902A06EE903AF8EEE77AF8EE06
:10F5C800666A67EE277AB7EE007A87EEA64AB4EE47
:10F5D800E44AF1EE10FA88BFB0EE644AB4EEC74AC6
:10F5E800F1EE10FAB8BFB0EE474AFEF7C6B900BF51
:10F5F800943D00201E750020713DAA3FD87400205C
:10F60800002E7FF4CBABEC4C002F00F09386D4EDAA
:10F61800004A9DED0A4AE94865EEA44AFDEEC53A5E
:10F62800E4EE074AB0EE674AA4EEA64A13EE901A33
:10F63800B4EEC46AF1EE10FAF0EE444A88BFF0EE78
:10F64800454AFDEEE44A14EE906A14EE905A9E4242
:10F65800A8BF1D46B142C8BF0D4604EE905AF8EE49
:10F66800E44A012AC0ED004A3EF482ADD4ED044AD2
:10F678009DED0B4A65EEA44AE4EE074AB0EE674AF0
:10F68800A4EEA64AB4EEC46AF1EE10FAF0EE444ACB
:10F6980088BFF0EE454AFDEEE44A14EE906A14EE97
:10F6A800905A9E42A8BF1D468E42B8BF0D4604EE32
:10F6B800905AF8EEE44A022AC0ED014A3EF458ADE9
:10F6C800D4ED084A9DED0C4A65EEA44AE4EE074ADB
:10F6D800B0EE674AA4EEA64AB4EEC46AF1EE10FA98
:10F6E800F0EE444A88BFF0EE454AFDEEE44A14EED7
:10F6F800906A14EE905A9E42A8BF1D468E42B8BF2B
:10F708000D4604EE905AF8EEE44A032AC0ED024A88
:10F718003EF42EADD4ED0C4A9DED0D4A65EEA44A9B
:10F72800E4EE074AB0EE674AA4EEA64AB4EEC46A0D
:10F73800F1EE10FAF0EE444A88BFF0EE454AFDEECD
:10F74800E44A14EE906A14EE905A9E42A8BF1D46F1
:10F758008E42B8BF0D4604EE905AF8EEE44A042AE9
:10F76800C0ED034A3EF404ADD4ED104A9DED0E4AB7
:10F7780065EEA44AE4EE074AB0EE674AA4EEA64A4C
:10F78800B4EEC46AF1EE10FAF0EE444A88BFF0EE27
:10F79800454AFDEEE44A14EE906A14EE905A9E42F1
:10F7A800A8BF1D468E42B8BF0D4604EE905AF8EE2B
:10F7B800E44A052AC0ED044A3EF4DAACD4ED144A12
:10F7C8009DED0F4A65EEA44AE4EE074AB0EE674A9B
:10F7D800A4EEA64AB4EEC46AF1EE10FAF0EE444A7A
:10F7E80088BFF0EE454AFDEEE44A14EE906A14EE46
:10F7F800905A9E42A8BF1D468E42B8BF0D4604EEE1
:10F80800905AF8EEE44A062AC0ED054A3EF4B0AC38
:10F81800D4ED184A9DED104A65EEA44AE4EE074A75
:10F82800B0EE674AA4EEA64AB4EEC46AF1EE10FA46
:10F83800F0EE444A88BFF0EE454AFDEEE44A14EE85
:10F84800906A14EE905A9E42A8BF1D468E42B8BFD9
:10F858000D4604EE905AF8EEE44A072AC0ED064A2F
:10F868003EF486ACD4ED1C4A9DED114A65EEA44ADF
:10F87800E4EE074AB0EE674AA4EEA64AB4EEC46ABC
:10F88800F1EE10FAF0EE444A88BFF0EE454AFDEE7C
:10F89800E44A14EE906A14EE905A9E42A8BF1D46A0
:10F8A8008E42B8BF0D4604EE905AF8EEE44A082A94
:10F8B800C0ED074A3EF45CACD4ED204A9DED124AF7
:10F8C80065EEA44AE4EE074AB0EE674AA4EEA64AFB
:10F8D800B4EEC46AF1EE10FAF0EE444A88BFF0EED6
:10F8E800454AFDEEE44A14EE906A14EE905A9E42A0
:10F8F800A8BF1D468E42B8BF0D4604EE905AF8EEDA
:10F90800E44A092AC0ED084A3EF432ACD4ED244A50
:10F918009DED134A65EEA44AE4EE074AB0EE674A45
:10F92800A4EEA64AB4EEC46AF1EE10FAF0EE444A28
:10F9380088BFF0EE454AFDEEE44A14EE906A14EEF4
:10F94800905A9E42A8BF1D468E42B8BF0D4604EE8F
:10F95800905AF8EEE44A0A2AC0ED094A3EF408AC87
:10F96800D4ED284A9DED144A65EEA44AE4EE074A10
:10F97800B0EE674AA4EEA64AB4EEC46AF1EE10FAF5
:10F98800F0EE444A88BFF0EE454AFDEEE44A14EE34
:10F99800906A14EE905A9E42A8BF1D468E42B8BF88
:10F9A8000D4604EE905AF8EEE44A0B2AC0ED0A4AD6
:10F9B8003EF4DEAB04E000BF4037002004390020ED
:10F9C800D4ED2C4A9DED154A65EEA45AE7EE045A8B
:10F9D800E6EEA57AB4EEE76AF1EE10FAC8BFF0EEEB
:10F9E800457AFDEEE77A17EE904AA342A8BF234670
:10F9F800A142D8BF194607EE901AF8EEE77AC0ED93
:10FA08000B7AFEF7B5BBCC4B93ED006AFEF706BD4B
:10FA1800F7F706FB0590FDF7CBBCC84FF7F700FBDF
:10FA2800C74ADBF8783112680290C31A9A1ACBF8E1
:10FA38007801BB80FA80FDF7A6BEBBF88811914219
:10FA480040F2F485BF49C04AD1ED007A92ED007AC0
:10FA5800BE49CBED637A77EE676ACBED617A012216
:10FA6800CBED606A8BED647AD1ED006ADFEDB87A90
:10FA78008BF89421FDF7B8BEB64B1B88002B40F0DD
:10FA8800F485B54AB54B11781868F2F701FFDBF831
:10FA98006821039B9A1AFDF77BBDD4ED014A64EEF9
:10FAA800C54AB0EE674AA4EE864AB4EEE64A74EE5A
:10FAB800654AF1EE10FA48BFF0EE474A012BC0ED57
:10FAC800004A3EF459ABD4ED054A64EEC54AB0EE9F
:10FAD800674AA4EE864AB4EEE64A74EE654AF1EE49
:10FAE80010FA48BFF0EE474A022BC0ED014A3EF437
:10FAF80043ABD4ED094A64EEC54AB0EE674AA4EEBA
:10FB0800864AB4EEE64A74EE654AF1EE10FA48BF4A
:10FB1800F0EE474A032BC0ED024A3EF42DABD4ED7C
:10FB28000D4A64EEC54AB0EE674AA4EE864AB4EEC2
:10FB3800E64A74EE654AF1EE10FA48BFF0EE474A1D
:10FB4800042BC0ED034A3EF417ABD4ED114A64EE22
:10FB5800C54AB0EE674AA4EE864AB4EEE64A74EEA9
:10FB6800654AF1EE10FA48BFF0EE474A052BC0EDA2
:10FB7800044A3EF401ABD4ED154A64EEC54AB0EE32
:10FB8800674AA4EE864AB4EEE64A74EE655AF1EE88
:10FB980010FA48BFF0EE475A062BC0ED055A3EF45E
:10FBA800EBAAD4ED195A65EEC55AB0EE674AA5EE30
:10FBB800864AF3EE044AB4EEE64A74EE645AF1EE6D
:10FBC80010FA48BFF0EE475A072BC0ED065A3EF42C
:10FBD800D3AAD4ED1D5A65EEC55AB0EE674AA5EE14
:10FBE800864AB4EEE64A74EE645AF1EE10FA48BF5B
:10FBF800F0EE475A082BC0ED075A3EF4BDAAD4EDE3
:10FC0800215A65EEC55AB0EE674AA5EE864AB4EEAB
:10FC1800E64A74EE645AF1EE10FA48BFF0EE475A1D
:10FC2800092BC0ED085A3EF4A7AAD4ED255A65EE73
:10FC3800C55AB0EE674AA5EE864AB4EEE64A74EEB7
:10FC4800645AF1EE10FA48BFF0EE475A0A2BC0ED9D
:10FC5800095A3EF491AAD4ED295A65EEC55AB0EE78
:10FC6800674AA5EE864AB4EEE64A74EE645AF1EEA7
:10FC780010FA48BFF0EE475A0B2BC0ED0A5A3EF473
:10FC88007BAAD4ED2D5A25EEC55AE5EE067AF4EE98
:10FC9800E67A77EEE47AF1EE10FAB8BFF0EE477A3A
:10FCA800C0ED0B7AFEF768BA2D4A2E49D2ED006AEC
:10FCB8002D4A91ED006A1278CBED636A8BED646A88
:10FCC800002A40F0E88276EEC65AF0EE466ABCEEAC
:10FCD800C76A2649CBED605A16EE102ACBED616A49
:10FCE800ABF88821FF22D1ED006A8BF8942177EEDA
:10FCF800C77AFDF779BD9BF8BC31012B01F01C8553
:10FD08001B4B96F916005A8896F90AE01B88194980
:10FD180010FB03F31EFB02F281FB020C81FB0301C3
:10FD2800D217DB17C2EB2C12C3EB21133A441C4445
:10FD38002A806C80FEF766BE807200202474002042
:10FD4800143B002004380020003800202038002010
:10FD58000000000040570020425700204457002070
:10FD68006839002008380020A86700201C380020C7
:10FD7800045500201F85EB51CB4EDBED017A9BED3E
:10FD8800006A3088736977EEA77AF0EE006AB0EE01
:10FD9800677AA6EE267A01380BEBC002D6EE267AF1
:10FDA800083A1033F6EE003A27EE237A67EEA37A84
:10FDB8008BED207ACBED217ADFF8F8B25E460BF1B5
:10FDC800800192ED027A92ED036AD6ED036AD6EDD0
:10FDD800027A53ED014A13ED025A37EE674A76EE7E
:10FDE800C65A77EE277AE4EE845A0138A2F108025F
:10FDF800E5EE047A06F1080603F1080336EE267AE2
:10FE080001F10801E4EE877AE5EE475A67EEA37A36
:10FE180025EEA37AC1ED007A81ED017AD1D1142DB6
:10FE28007DF444AAF7F7FCF8029BA04FC01A78802B
:10FE3800DBF81841FDF73ABA9B4E3588D6F804E04E
:10FE48004FEA550C4FEA8C020BEB8507ED080BEBDC
:10FE5800020300F09F8010320135954803EB051529
:10FE68003A4410330EF1100407F1100151ED032A42
:10FE780051ED043A10ED043A10ED032A51ED026AEF
:10FE880011ED016A50ED020A10ED010A12ED044A63
:10FE980012ED035A53ED044A53ED035A13ED027A57
:10FEA80053ED017A12ED021A52ED011A73EE238A0C
:10FEB80032EE228A40ED048A00ED038A70EEA68AAB
:10FEC80030EE068A40ED028A00ED018A74EE848ADB
:10FED80035EE858A43ED048A03ED038A77EE018ABD
:10FEE80037EEA18A43ED028A03ED018A73EE633A85
:10FEF80075EE655A14ED035A32EE623A74EE644AAE
:10FF080025EE638A14ED044A23EE052A64EE652A79
:10FF1800A3EE048A10339D4224EE843AA3EE842A89
:10FF280000F1100004F11004A5EE853A01F110016A
:10FF380002F11002E4EE852A01ED078A01ED082A94
:10FF480002ED073A42ED082A54ED055A14ED065A17
:10FF580070EEE66A30EE466A31EE477A71EEE77A7D
:10FF680026EE253A65EEE63A25EE674A67EE054A3B
:10FF7800E6EE053AA6EE853AA7EE254AE7EEA54A4B
:10FF880001ED063A41ED053A02ED064A42ED054A11
:10FF98007FF46CAF1FFA8CF472462146454818F07E
:10FFA80091FE21467268384618F08CFE424B1B7849
:10FFB800142B7FF43DAF35E73B4E3E48B268B1891C
:10FFC80020F070FB3C4B1D78142D01F0D684DBF833
:10FFD80018410134CBF81841CFE6DFF8E48098F8EF
:10FFE80000205FEA920E01F00D85344F0EF10100FA
:08FFF80040013E1807F120034F
:020000040801F1
:10000000A7F1700113ED076A53ED056A13ED037A4A
:1000100053ED017A53ED025A13ED084A53ED064AA7
:1000200013ED045A26EE066A66EEA66A27EE077AF4
:1000300067EEA77AA4EE046A20339E42E4EEA46A37
:1000400001F11001A5EE057AE5EEA57AF1EEC65AAA
:10005000B1EEE66AF1EEC76AB1EEE77A41ED085A11
:1000600001ED076A41ED066A01ED057ACAD1203833
:1000700007440BEB0E1112F0030318BF08370FD023
:1000800057ED017A17ED027A67EEA77A013BE7EEAA
:10009000077A07F10807B1EEE77AA1EC017AEFD110
:1000A000142D01F0A1840134CBF81841FDF774B888
:1000B0005842002024740020D0220020C0220020BA
:1000C000207400204023002052420020DBF81CE175
:1000D000BBF814C18A4BCCF120085FFA88F80CEB0E
:1000E0004E1603EB86065FEA980301F0EB830133BB
:1000F00018018449844A371806F1100313ED024AA7
:1001000013ED035A13ED016A13ED047A51ED024A1F
:1001100051ED035A51ED016A51ED047A64EE244A1F
:1001200065EE255A66EE266A67EE277A1033BB42E3
:1001300042ED024A42ED035A42ED016A42ED047A71
:1001400001F1100102F11002D8D17049A0F11002A2
:1001500016448F185A4418F0030309D0B6EC017AFC
:10016000F7EC017A67EE277A013BE2EC017AF5D1F0
:10017000BCF1000F41F09082142D7DF49BA8F6F79E
:1001800053FF029B624FDBF81841C01A7880FDF7DD
:1001900091B8DBF81C615F4B5F4ADFED607AD2ED0E
:1001A000008A5F4FF1000B44F8EE688A9B8809EEE5
:1001B000103A643BC82BA8BFC82368EEA78AF8EEA4
:1001C000497A782BB8BF782368EEA78A07EE903A71
:1001D0003144B0EE680A07EB8107B8EEE78A21F0F8
:1001E00019FCB8EEC99AF0EE409AB0EE680A21F018
:1001F00073FB38EE097A79EE487A28EE098A67EEC1
:10020000877AB7EE006A88EE277A142DF8EE007A26
:1002100077EE076A60EE277A89EEA67A77EE065ABD
:1002200036EE477AC6EE256A67EEA67A27EE267A7C
:10023000C7ED006A87ED047AC7ED026AC7ED017A5F
:10024000C7ED037A01F09183364B374A013683FBC1
:10025000063EAEEBE67E0EEB4E0E0134A6EB0E0E26
:100260001578CBF81841CBF81CE131E72F4A32F969
:100270001340FEF7C4BB2D4A32F91370FEF7B4BB2E
:10028000F6F7D2FE284B02901D78142D05BF204FA3
:10029000DBF81841DBF818413C80FCF764BF76EED0
:1002A000665A18E5224F002437F9023F00EE103A53
:1002B000E0B2B8EEC00A013402F070FE062CF3D1B1
:1002C0000494FEF767BF1B4BB5F906101A6802B11C
:1002D00011609B69B5F90820002B7EF408AFFEF78A
:1002E00007BF154F002437F9023B00EE103AE0B289
:1002F000B8EEC00A013402F051FE042CF3D1DFE75E
:100300007042002000440020D0220020F043002052
:100310002474002070440020286C002027D4D2369A
:10032000D461002056555555207400204C530020B0
:10033000F6380020E0620020FA38002094ED006AD0
:10034000DDED0A4AD44825EE866ABDEEC55AA4EE14
:10035000876A15EE101AB0EE675AA6EE265ABDEE61
:10036000C56A16EE106A16EE105A9E42A8BF1D46C8
:10037000B142C8BF0D4606EE105AB8EEC66A012A51
:1003800080ED006A3DF4F8AE94ED046A9DED0B5AE1
:1003900025EE866AA5EE076AB0EE675AA6EE265AE3
:1003A000BDEEC56A16EE106A16EE105A9E42A8BF40
:1003B0001D468E42B8BF0D4606EE105AB8EEC66A0C
:1003C000022A80ED016A3DF4D7AE94ED086A9DEDF6
:1003D0000C5A25EE866AA5EE076AB0EE675AA6EEBD
:1003E000265ABDEEC56A16EE106A16EE105A9E42E7
:1003F000A8BF1D468E42B8BF0D4606EE105AB8EE95
:10040000C66A032A80ED026A3DF4B6AE94ED0C6A2A
:100410009DED0D5A25EE866AA5EE076AB0EE675A85
:10042000A6EE265ABDEEC56A16EE106A16EE105AF2
:100430009E42A8BF1D468E42B8BF0D4606EE105A1A
:10044000B8EEC66A042A80ED036A3DF495AE94EDD9
:10045000106A9DED0E5A25EE866AA5EE076AB0EE8B
:10046000675AA6EE265ABDEEC56A16EE106A16EE5B
:10047000105A9E42A8BF1D468E42B8BF0D4606EEDA
:10048000105AB8EEC66A052A80ED046A3DF474AECF
:1004900094ED146A9DED0F5A25EE866AA5EE076A63
:1004A000B0EE675AA6EE265ABDEEC56A16EE106A81
:1004B00016EE105A9E42A8BF1D468E42B8BF0D468A
:1004C00006EE105AB8EEC66A062A80ED056A3DF4BB
:1004D00053AE94ED186A9DED105A25EE866AA5EE8E
:1004E000076AB0EE675AA6EE265ABDEEC56A16EE4A
:1004F000106A16EE105A9E42A8BF1D468E42B8BF23
:100500000D4606EE105AB8EEC66A072A80ED066A56
:100510003DF432AE94ED1C6A9DED115A25EE866ACB
:10052000A5EE076AB0EE675AA6EE265ABDEEC56A7A
:1005300016EE106A16EE105A9E42A8BF1D468E4255
:10054000B8BF0D4606EE105AB8EEC66A082A80ED0E
:10055000076A3DF411AE94ED206A9DED125A25EE26
:10056000866AA5EE076AB0EE675AA6EE265ABDEE79
:10057000C56A16EE106A16EE105A9E42A8BF1D46B6
:100580008E42B8BF0D4606EE105AB8EEC66A092A6A
:1005900080ED086A3DF4F0AD94ED246A9DED135AA8
:1005A00025EE866AA5EE076AB0EE675AA6EE265AD1
:1005B000BDEEC56A16EE106A16EE105A9E42A8BF2E
:1005C0001D468E42B8BF0D4606EE105AB8EEC66AFA
:1005D0000A2A80ED096A3DF4CFAD94ED286A9DEDBD
:1005E000145A25EE866AA5EE076AB0EE675AA6EEA3
:1005F000265ABDEEC56A16EE106A16EE105A9E42D5
:10060000A8BF1D468E42B8BF0D4606EE105AB8EE82
:10061000C66A0B2A80ED0A6A3DF4AEAD94ED2C6AF1
:100620009DED155A65EE865AE7EE055AE6EEA57A77
:10063000FFF7DBB9194A1A49D2ED007A194A91ED50
:10064000007A1278CBED637A8BED647A002A01F0A0
:10065000CC8077EE676A1449CBED617ACBED606AA6
:10066000FF22D1ED006ADFED117A8BF89421FDF7BE
:10067000BFB80F494B69002B3CF48EAF0D480E4BB1
:10068000008893FBF0F00B684FF0010E186081F8C2
:1006900011E0FCF781BF00BF043900206839002059
:1006A00008380020A86700201C3800200000000047
:1006B000485700206057002020A10700A34DA44EFA
:1006C00095ED004A95ED057AD5ED014A95ED066A5E
:1006D000D5ED046A95ED035AD5ED025A67EE897A95
:1006E00006EB8403A4EE277AA4EEA76A66EEC76A37
:1006F000A5EE476AE5EEA76A20EE070A85ED056AD2
:10070000C5ED066A83ED007A29EE088A21F036F9F4
:1007100069EE288AD5ED0E5AD5ED176A95ED091ABE
:10072000D5ED121A95ED0F5A95ED187A95ED0A2A26
:10073000D5ED132A95ED0D6AD5ED167A95ED0C3AA7
:10074000D5ED0B3A95ED154AD5ED144AE1EE085A70
:10075000002206EB8403E8EEA16A00B2CBF8042184
:10076000A2EE085ACBF80821CBF80C21A8EEA27A09
:1007700026EE656A67EEE67AA3EE655AA3EE886A0E
:10078000A6EEC47AE8EEA47A85ED0E5AC3ED205A9F
:1007900085ED0F6AC3ED406A85ED177AC5ED187ACD
:1007A000FEF7E3BA6B494A69002A3CF426AF0A68AF
:1007B00013604B74FCF721BFBAF93C30CAF824200F
:1007C00007EE903A0122F8EEE77ACAF86C30CAF8E0
:1007D00088200023012DCAED1F7ACAED1E7ACAF8BF
:1007E000803001F05B80A5427DF457ADBAF93E3010
:1007F000CAF8703007EE903A00220123F8EEE77A4B
:10080000CAF82820CAF89C300023012DCAED247AAA
:10081000CAED237ACAF8943001F04480A5427DF4F1
:100820006EADBAF94030CAF8743007EE903A002243
:100830000123F8EEE77ACAF82C20CAF8B03000237A
:10084000012DCAED297ACAED287ACAF8A8307DF4BC
:1008500088AD9FED418A032E71D0B8F1000F09D009
:1008600007EE908AF8EEE77AF4EEC87AF1EE10FA25
:1008700001F1D180394ADAF8743012689BF82011FE
:10088000F88003EB540393FBF4F40023CAF82C40E4
:1008900093621363D36231B1314B1B8823F400633D
:1008A000002B7DF45FAD2F4B1B6813F4003340F039
:1008B000A2872D491A46C85C012803F10C0300F0F9
:1008C000B0840132152AF6D1FDF74CBDBEF1000F00
:1008D00000F0FD87FDEEC54A0AA8244C244D14EE15
:1008E000901A00EB8202D4ED004AF0EC013A65EE7A
:1008F000A44A04EE101AE3EE874A1034F0EE673A89
:10090000E4EEA63AF0EE634A37B1F4EE463AF1EE81
:1009100010FA48BFF0EE454AFDEEE44A14EE906A44
:100920008E4204DB9E42A8BF1E4604EE106AB8EE5B
:10093000C44A8242A5EC014AD5D1FDF721BCB0EEF4
:10094000480A21F01BF800B287E700BFF4440020FA
:100950007042002048570020000000004040002066
:10096000C83D0020D83500205859030840370020E2
:1009700004390020BEF1000F00F00387DC4C9DED30
:100980000A5A94ED006ADB4825EE866AA5EE076AEE
:10099000B0EE675AA6EE265ABDEEC56A16EE106A8C
:1009A00016EE105A9E42A8BF1D46B142C8BF0D4662
:1009B00006EE105AB8EEC66A012A80ED006A3DF4D0
:1009C000DFAB94ED046A9DED0B5A25EE866AA5EE29
:1009D000076AB0EE675AA6EE265ABDEEC56A16EE55
:1009E000106A16EE105A9E42A8BF1D46B142C8BFFB
:1009F0000D4606EE105AB8EEC66A022A80ED016A6C
:100A00003DF4BEAB94ED086A9DED0C5A25EE866A66
:100A1000A5EE076AB0EE675AA6EE265ABDEEC56A85
:100A200016EE106A16EE105A9E42A8BF1D46B1423D
:100A3000C8BF0D4606EE105AB8EEC66A032A80ED0E
:100A4000026A3DF49DAB94ED0C6A9DED0D5A25EEC6
:100A5000866AA5EE076AB0EE675AA6EE265ABDEE84
:100A6000C56A16EE106A16EE105A9E42A8BF1D46C1
:100A7000B142C8BF0D4606EE105AB8EEC66A042A47
:100A800080ED036A3DF47CAB94ED106A9DED0E5A47
:100A900025EE866AA5EE076AB0EE675AA6EE265ADC
:100AA000BDEEC56A16EE106A16EE105A9E42A8BF39
:100AB0001D46B142C8BF0D4606EE105AB8EEC66AD2
:100AC000052A80ED046A3DF45BAB94ED146A9DED5C
:100AD0000F5A25EE866AA5EE076AB0EE675AA6EEB3
:100AE000265ABDEEC56A16EE106A16EE105A9E42E0
:100AF000A8BF1D46B142C8BF0D4606EE105AB8EE5B
:100B0000C66A062A80ED056A3DF43AAB94ED186A90
:100B10009DED105A25EE866AA5EE076AB0EE675A7B
:100B2000A6EE265ABDEEC56A16EE106A16EE105AEB
:100B30009E42A8BF1D46B142C8BF0D4606EE105AE0
:100B4000B8EEC66A072A80ED066A3DF419AB94ED4B
:100B50001C6A9DED115A25EE866AA5EE076AB0EE75
:100B6000675AA6EE265ABDEEC56A16EE106A16EE54
:100B7000105A9E42A8BF1D46B142C8BF0D4606EEA0
:100B8000105AB8EEC66A082A80ED076A3DF4F8AA42
:100B900094ED206A9DED125A25EE866AA5EE076A4D
:100BA000B0EE675AA6EE265ABDEEC56A16EE106A7A
:100BB00016EE105A9E42A8BF1D46B142C8BF0D4650
:100BC00006EE105AB8EEC66A092A80ED086A3DF4AE
:100BD000D7AA94ED246A9DED135A25EE866AA5EEF8
:100BE000076AB0EE675AA6EE265ABDEEC56A16EE43
:100BF000106A16EE105A9E42A8BF1D46B142C8BFE9
:100C00000D4606EE105AB8EEC66A0A2A80ED096A49
:100C10003DF4B6AA94ED286A9DED145A25EE866A35
:100C2000A5EE076AB0EE675AA6EE265ABDEEC56A73
:100C300016EE106A16EE105A9E42A8BF1D46B1422B
:100C4000C8BF0D4606EE105AB8EEC66A0B2A80EDF4
:100C50000A6A3DF495AA94ED2C6A9DED155A65EE4D
:100C6000865AE7EE055AE5EEA67AFDEEE77A17EE2C
:100C7000902A9342A8BF13469142D8BF194607EE67
:100C8000901AF8EEE77AC0ED0B7AFDF779BA1A4BB5
:100C9000197801F00109FDF76FBA184BDFED187AEA
:100CA0001C68CBED4C7A14F0805400F0D282B7EE81
:100CB000007A77EE677AF4EEE75AF1EE10FA88BF21
:100CC000F0EE675ACBED665AFDF79EB877EE677A7D
:100CD000B7EE007AF4EEC77AF1EE10FACBED4C7A6B
:100CE00040F38C8284EEA77A8DED0A7AFDF782B804
:100CF00040370020043900203556002044390020B8
:100D000000000080012A40F3C98507EE101AB8EEF2
:100D1000C77AC7EE876AB1EEE68A032E15D0B8F11E
:100D2000000F09D007EE908AF8EEE77AF4EEC87A61
:100D3000F1EE10FA00F16F86DAF86C3003EB540331
:100D400093FBF4F3CAF824304DE5B0EE480A20F0E6
:100D500015FE00B2E3E7012A40F3A48507EE101A5E
:100D6000B8EEC77AC7EE876AB1EEE68A032E15D0D1
:100D7000B8F1000F09D007EE908AF8EEE77AF4EEAA
:100D8000C87AF1EE10FA00F14686DAF8703003EB1B
:100D9000540393FBF4F3CAF828303FE5B0EE480A59
:100DA00020F0ECFD00B2E3E7012A7FF752AD07EE39
:100DB000101AB8EEC77AC7EE876AB1EEE68A4AE53E
:100DC000914B1B88DE0540F11E85904B904A93EDB8
:100DD000017AD3ED006AD3ED027A8E4B0793BDEE14
:100DE000C77AB3F906708C4B0193FDEEE66A17EEF5
:100DF000103AFDEEE77A118BADF82A3016EE902A04
:100E000017EE903AADF82820ADF82C30834A84488C
:100E1000B2F90230B2F90020824CD0ED007A9FED99
:100E2000827A82484FF47A7503F5E16305FB03F398
:100E300002F5E16205FB02F284FB03651D44DB174A
:100E400084FB0264C3EBE52377EEC77A079D007845
:100E50002E8806901444D2172846C2EBE422FDEEF9
:100E6000E77A2C466D88A4888646A3F5FA736D1A36
:100E70000089ADF8403017EE903AA2F5FA72ADF85D
:100E80003250BEF80E50ADF84220641A401ABEF837
:100E90000A20ADF82E30BEF80C30ADF83440ADF875
:100EA00038006C1A0698624DADF83E407F1A761AEB
:100EB000521A5B1A0021ADF83670ADF83060ADF80B
:100EC0003A20ADF83C3029606960A960E9600028EB
:100ED00000F0A685574FDFF86881574ECDF820B057
:100EE0008946CDF824A03DE016AB03EB440030F971
:100EF000300CA8F8000097F902C001238E4403FAD1
:100F000004F44E4B56F82EE01CFB00F083FB003C33
:100F1000C017039B14EA0E0FC0EB6C100CBF01242A
:100F20004FF0FF3498420EDB059B02FB03F2434B6C
:100F300083FB02E3D217C2EB6313A3EB0A031BB2DA
:100F40008342A8BF034635F8112003FB042325F88C
:100F50001130069B09F10109994507F1070708F1CE
:100F600002086FDAB879002837D1397897F9052067
:100F700005924FEA410E0EEB010006EB800097F957
:100F80000430C288808897F803C07C78121A92B225
:100F90002A4802FB03F380FB03A0DB17C3EB6013BB
:100FA0004FEA520AA3EB0A031BB20393BCF1000FF2
:100FB0009AD016AB03EB440BB8F900003BF930BCF8
:100FC000584513DA8444604503DCE3455846A8BF1E
:100FD000604600B2A8F800008DE71630C0B212F0EB
:100FE000B9F80028C1D1A8F80000B2E783DDA0EB72
:100FF0000C0CDC4503DB6045A8BF604683460FFA56
:101000008BF0A8F8000076E7FC3D0020207500205A
:10101000AC6D00204C530020386C0020045500209B
:1010200004390020C5B3A2910080BB4408710020A0
:10103000F43800200C710020307300201F85EB5124
:101040005C240020DDF820B0DDF824A096F90A0029
:101050002B88874A874910FB03F3F07A097882FBD3
:101060000342FF284FEAE373C3EB621200F01183DF
:10107000814240F20E83079B33F9100096F9164027
:101080006B88104428807A4AF07D14FB03F382FBBE
:101090000342FF284FEAE373C3EB621200F0F682CB
:1010A000814240F2F382079B33F9100096F9224007
:1010B000AB88104468806E4A96F8230014FB03F353
:1010C00082FB0342FF284FEAE373C3EB621200F096
:1010D000DA82814240F2D782079B33F9100096F9F9
:1010E0002E40EB881044A880614A96F82F0014FB2C
:1010F00003F382FB0342FF284FEAE373C3EB621260
:1011000000F0BE82814240F2BB82079B33F910009F
:1011100096F93A402B891044E880554A96F83B00EE
:1011200014FB03F382FB0342FF284FEAE373C3EB94
:10113000621200F0A282814240F29F82079B33F943
:10114000100096F946406B8910442881484A96F869
:10115000470014FB03F382FB0342FF284FEAE373CB
:10116000C3EB621200F08682814240F28382079BC9
:1011700033F9100096F95240AB89104468813C4A1B
:1011800096F8530014FB03F382FB0342FF284FEA57
:10119000E373C3EB621200F06A82814240F267821D
:1011A000079B33F9100096F95E40EB891044A88143
:1011B0002F4A96F85F0014FB03F382FB0342FF28DB
:1011C0004FEAE373C3EB621300F04E82884280F073
:1011D0004B82079A32F910201344EB81019BFDF7F3
:1011E000F6BB0423032404930220FDF7E3BF82230C
:1011F000FCF750B8DFED207AFCF718B81F4B1C68DD
:1012000014F0805425D0B6EE007A67EE877AF4EEBB
:10121000E75AF1EE10FA48BFF0EE675A3FF552ADCB
:1012200045E5DBF8244153003CB1981801EB800000
:1012300064784078A042BDF495A8134401EB830183
:101240000023CBF82411ABF8BE31CBF8C031FDF749
:1012500089B810F4800401D00024D4E7B6EE007AF7
:10126000F4EEC75AF1EE10FACDDCFCF7CDBD00BFAD
:101270001F85EB512C55002000000243443900200B
:10128000D4ED004A9DED0A4AF04865EEA44AFDEE11
:10129000C53AE4EE074AB0EE674AA4EEA64A13EE5A
:1012A000901AB4EEC46AF1EE10FAF0EE444A88BF28
:1012B000F0EE454AFDEEE44A14EE906A14EE905AC0
:1012C0009E42A8BF1D46B142C8BF0D4604EE905ACB
:1012D000F8EEE44A012AC0ED004A3DF45EABD4EDDD
:1012E000044A9DED0B4A65EEA44AE4EE074AB0EECF
:1012F000674AA4EEA64AB4EEC46AF1EE10FAF0EE24
:10130000444A88BFF0EE454AFDEEE44A14EE906A86
:1013100014EE905A9E42A8BF1D468E42B8BF0D469D
:1013200004EE905AF8EEE44A022AC0ED014A3DF478
:1013300034ABD4ED084A9DED0C4A65EEA44AE4EEC8
:10134000074AB0EE674AA4EEA64AB4EEC46AF1EECC
:1013500010FAF0EE444A88BFF0EE454AFDEEE44A4A
:1013600014EE906A14EE905A9E42A8BF1D468E421B
:10137000B8BF0D4604EE905AF8EEE44A032AC0EDD9
:10138000024A3DF40AABD4ED0C4A9DED0D4A65EEE0
:10139000A44AE4EE074AB0EE674AA4EEA64AB4EEC9
:1013A000C46AF1EE10FAF0EE444A88BFF0EE454A06
:1013B000FDEEE44A14EE906A14EE905A9E42A8BFE5
:1013C0001D468E42B8BF0D4604EE905AF8EEE44A30
:1013D000042AC0ED034A3DF4E0AAD4ED104A9DED85
:1013E0000E4A65EEA44AE4EE074AB0EE674AA4EE60
:1013F000A64AB4EEC46AF1EE10FAF0EE444A88BF91
:10140000F0EE454AFDEEE44A14EE906A14EE905A6E
:101410009E42A8BF1D468E42B8BF0D4604EE905AAC
:10142000F8EEE44A052AC0ED044A3DF4B6AAD4ED2C
:10143000144A9DED0F4A65EEA44AE4EE074AB0EE69
:10144000674AA4EEA64AB4EEC46AF1EE10FAF0EED2
:10145000444A88BFF0EE454AFDEEE44A14EE906A35
:1014600014EE905A9E42A8BF1D468E42B8BF0D464C
:1014700004EE905AF8EEE44A062AC0ED054A3DF41F
:101480008CAAD4ED184A9DED104A65EEA44AE4EE0C
:10149000074AB0EE674AA4EEA64AB4EEC46AF1EE7B
:1014A00010FAF0EE444A88BFF0EE454AFDEEE44AF9
:1014B00014EE906A14EE905A9E42A8BF1D468E42CA
:1014C000B8BF0D4604EE905AF8EEE44A072AC0ED84
:1014D000064A3DF462AAD4ED1C4A9DED114A65EE20
:1014E000A44AE4EE074AB0EE674AA4EEA64AB4EE78
:1014F000C46AF1EE10FAF0EE444A88BFF0EE454AB5
:10150000FDEEE44A14EE906A14EE905A9E42A8BF93
:101510001D468E42B8BF0D4604EE905AF8EEE44ADE
:10152000082AC0ED074A3DF438AAD4ED204A9DEDC3
:10153000124A65EEA44AE4EE074AB0EE674AA4EE0A
:10154000A64AB4EEC46AF1EE10FAF0EE444A88BF3F
:10155000F0EE454AFDEEE44A14EE906A14EE905A1D
:101560009E42A8BF1D468E42B8BF0D4604EE905A5B
:10157000F8EEE44A092AC0ED084A3DF40EAAD4ED7B
:10158000244A9DED134A65EEA44AE4EE074AB0EE04
:10159000674AA4EEA64AB4EEC46AF1EE10FAF0EE81
:1015A000444A88BFF0EE454AFDEEE44A14EE906AE4
:1015B00014EE905A9E42A8BF1D468E42B8BF0D46FB
:1015C00004EE905AF8EEE44A0A2AC0ED094A3DF4C6
:1015D000E4A9D4ED284A9DED144A65EEA44AE4EE50
:1015E000074AB0EE674AA4EEA64AB4EEC46AF1EE2A
:1015F00010FAF0EE444A88BFF0EE454AFDEEE44AA8
:1016000014EE906A14EE905A9E42A8BF1D468E4278
:10161000B8BF0D4604EE905AF8EEE44A0B2AC0ED2E
:101620000A4A3DF4BAA9D4ED2C4A9DED154A65EE5F
:10163000A45AE7EE045AE6EEA57AB4EEE76AF1EEB4
:1016400010FAC8BFF0EE457AFDF72EBD0439002030
:10165000D14BB5F90A201B68002B00F0D3811A602A
:1016600001230493FDF796BDB6F95C20B4E5B6F905
:10167000500098E5B6F944007CE5B6F9380060E51D
:10168000B6F92C0044E5B6F9200028E5B6F91400B7
:101690000CE5B6F90800F1E4C04B4FEA88065FEAB2
:1016A0009C0201EB060703EBCE1E5E4400F0BF81F7
:1016B00001324FEA02180EEB08000EF1100307F199
:1016C000100106F1100213ED024A13ED035A13ED57
:1016D000016A13ED047A51ED024A51ED035A51EDBE
:1016E000016A51ED047A64EE244A65EE255A66EEED
:1016F000266A67EE277A1033984242ED024A42ED9D
:10170000035A42ED016A42ED047A01F1100102F13F
:101710001002D8D1A8F110029644BB1816441CF050
:10172000030C3EF429ADBEEC017AF3EC017A67EECE
:10173000277ABCF1010CE6EC017AF4D1FEF71CBD6E
:10174000974996F916E00B8896F90A20B1F902003C
:1017500094491EFB03F3524200FB02F081FB03E2BB
:10176000121181FB00E1DB17C017C0EB2110991AA1
:10177000D31A01440344791A1C4429806C80FDF774
:1017800045B90AAD884E894F05EB8202814604E0D7
:10179000AA42A7EC016A3CF4F3AC96ED006AF5ECC2
:1017A000014A019125EE866AA7EE246AF0EE674AA7
:1017B000E6EE264ABDEEE46A16EE10EA714505DC57
:1017C00016EE100A9E45A8BF184601909DED016ACD
:1017D0001036B8EEC66A002CDAD1B9F1000FD7D1B5
:1017E000C445B8BFB0EE456AD2E777EEC76AF0EEFF
:1017F000477AFEF730BF6E4B1B78032B00F0138146
:101800000023FFF756B86B4B9FED6B6A93ED007AA0
:101810006A4BD3ED003A674BD3ED017A674B93EDFA
:10182000014A644BD3ED026A644BD3ED024A644B28
:1018300037EE237A93ED005AD3ED015A614B0193B1
:1018400077EE847A37EE057A76EEA46A77EEA57A9B
:1018500027EE067A66EE866A67EE867A1946BDEE50
:10186000C77AFDEEE66AFDEEE77A17EE102A096800
:10187000CDED036A17EE903AADF82820CD04BDF9FE
:101880000C20ADF82A30ADF82C2060D44E4A4F4BD6
:101890000792198BB2F90670FFF7B8BA9FED4C8A20
:1018A000FFF73BBA9FED4A8AFFF760BA9FED490AFE
:1018B000494F25EE800A20F061F8DBF81841F880E6
:1018C000FBF7F8BC4549464A0F46FEF744BCFDEE1F
:1018D000C54A0AAD344EDFF8D4E014EE901A05EB99
:1018E000820206E0AA42EEEC014A06F110063CF440
:1018F00047ACD6ED004AB5EC014A65EEA44AE7EEE6
:10190000044AB0EE674AA6EEA44AF0EE444A37B164
:10191000B4EE446AF1EE10FAC8BFF0EE454AFDEEAF
:10192000E44A14EE909A494504EE901A04DC994575
:10193000A8BF994604EE909AF8EEE44A002CD1D163
:101940000028CFD1C445B8BFF0EE454ACAE71E4BC8
:10195000079319461D4BB1F90670198B8F42BCBF16
:101960005242ADF82C20FFF751BAF5F75DFB029B10
:10197000194FDBF81C61DBF81841C01A7880FEF7BC
:1019800063BCF5F751FB174B134F1D78029BC01A30
:101990007880FEF720BB00BFE0620020704200208C
:1019A000045500201F85EB514037002004390020EA
:1019B0008F3D0020A43800203333333FB03800205F
:1019C000BC380020386C00204C530020AC6D002047
:1019D000000000000000C84224740020F0430020F2
:1019E000C022002020740020F5F71EFB514B524FFF
:1019F0001D78029B98F80020DBF81841C01AB880C7
:101A0000FEF751BB01230493FDF7C4BB4B4901F121
:101A10008007FEF730BBF880AAF8B440FCF7A9BCF9
:101A2000474EFFF713BB1DF0DDFEFCF79BBC3B46AA
:101A300075E69BF87431002B7BF49FAEFBF78ABEF2
:101A4000404A414B10681B689847404B9AED007A1A
:101A5000D3ED007A3E4BD6ED006A83ED020A3D4B92
:101A600067EE277A234427EE8C7AD3ED007A3A4B3F
:101A700067EE277AF0EE665AEDEE275A93ED006A8C
:101A8000B1EE467AF4EEC75AF1EE10FA08D4F4EE4D
:101A9000C65AF1EE10FA8CBFB0EE467AB0EE657A17
:101AA0002E4B1B78012B02D0192B7BF4DDADDFED23
:101AB0002C7AB4EEE7DAF1EE10FACCBF0123002362
:101AC000FBF7DDBD132B05D1B0EE480A1FF056FF22
:101AD000A8F80000B0EE480ADAF814322148984716
:101AE000144B1B78132BB0EE408A7BF427AC1FF00D
:101AF00045FFA8F80200FBF721BC1B4BD3ED007A91
:101B0000B1EE677AB4EEC7DAF1EE10FA0FD4B4EEA4
:101B1000E7DAF1EE10FA88BFB0EE67DA134BC6EDE4
:101B200000BA1B689342BBF660ADFDF769B8B0EE32
:101B300047DAF3E72074002024740020C02200203C
:101B40003073002030720020447200202C000020EE
:101B5000A438002058720020C0720020807100203C
:101B600000009642D4610020BC720020A0720020C8
:101B7000704700BF10F8113C0133DBB20A2B00F8AC
:101B8000113C07D9044A10F8131C002322F8113025
:101B900000F8113C704700BF84570020F0B55C4F3F
:101BA0005C4B3C785C4A0134A2FB040293E8600081
:101BB000120902EB8202D86BA4EB8202A9423A70AE
:101BC00001EB000233D293F84500002855D053486A
:101BD00002F580320478B2FBF4F2964230D3901BC7
:101BE0004FF4803595FBF4F42044986040F68C2443
:101BF0000025A04283E8060083F8455028D993F8D1
